:100000000C94A5210C94D6210C94D6210C94D621C5
:100010000C94D6210C94D6210C94D6210C94D62184
:100020000C94D6210C94D6210C94D6210C94D62174
:100030000C94D6210C94338C0C94D6210C94D6219C
:100040000C94D6210C94E1750C94D6210C94D621F5
:100050000C94D6210C94D6210C9487CB0C94E98B6C
:100060000C94D6210C94983F0C948E3F0C94D6217E
:100070000C94D6210C94D6210C94D6210C94D62124
:100080000C94D6210C94D6210C94D6210C94D62114
:100090000C94D6210C94D6210C94D6210C94D62104
:1000A0000C94D6210C94D6210C94D6210C94D621F4
:1000B0000C94D6210C94D6210C94D6210C94D621E4
:1000C0000C94D6210C94D6210C94D6210C94D621D4
:1000D0000C94D6210C94D6210C94D6210C94D621C4
:1000E0000C94D6213D4BAC49E549794BE549E549AE
:1000F000E549E549E549E549E549E549E549E54990
:10010000E549E549E549E549E549E549E549E5497F
:10011000E549E549E549E549E549E549E549E5496F
:10012000734BE549E549E549E549E549E549E549CF
:10013000E5494C4BE549E549E549E549E549E549E6
:10014000E549E549E549E549904BE249C763B063B4
:10015000D663B363AD63D963B663C263B963D46373
:10016000BC63BF6360F663F652F656F65CF69AF629
:1001700067F66BF671F675F679F67FF683F687F615
:100180009AF68DF691F695F6BBF9C0F9C5F9CFF957
:10019000D9F952FAE3F9EBF9F3F9FDF907FA11FA93
:1001A00020FA2AFA52FA34FA3EFA48FA084AD73BB9
:1001B0003BCE016E84BCBFFDC12F3D6C74319ABD36
:1001C00056833DDA3D00C77F11BED9E4BB4C3E915A
:1001D0006BAAAABE000000803F05A84CCDB2D44E49
:1001E000B93836A9020C50B9918688083CA6AAAA4B
:1001F0002ABE000000803F000D94B0140C94CC6225
:100200000C94A1D60C94BBF90C942D490C94E3806A
:100210000C9452FA0D94A4390C94CFD60C94C2636A
:100220000C9411FA0D9495110C9448600C94A2FF53
:100230000D9471110C9447FD0C94BC630C943C60BC
:100240000C94B78E0C94904B0C9483C30C94B663AF
:100250000C94A4DC0D948F0F0C94E2490C941B8D2C
:100260000C94734B0C9434FA0C94608D0C94C5D898
:100270000C94D4630D9430000D94A8140C9487F65C
:100280000C94508D0D9402100C94125C0C9463F637
:100290000C9461440C94596A0C94EBDD0C94794BEA
:1002A0000D9489110C94BE8E0C9460F60C94E4CCE1
:1002B0000C9456F60C94EFDD0C94D1900C94E54917
:1002C0000C9407FA0C949DFF0C9477510C947FF6D4
:1002D0000D9434100D940A110C94D75C0C94F9FC15
:1002E0000C9498FF0C94D4D80C9442FD0C94B24713
:1002F0000C94A1D70C946BF60C94CEFF0C94B0DC4C
:100300000D9453100C943E8D0D9472100C94214951
:100310000C9424490C94BF630C9462600C94D963D0
:100320000D9419110D948F110C941B5C0C944CFDC1
:100330000C942AFA0D94BF140C9436660C94755DD7
:100340000C948FCC0C94FDF90C943DFD0C94BB9255
:100350000C94F9CC0C94C7630C94BC8B0D94FB10DB
:100360000C94DF3F0C9462670C9489660C941566BC
:100370000C9420FA0C94A1510C94235C0C94E6D8B4
:100380000C944E600C94AB410C94C8FF0C9438FD57
:100390000C94BCFF0C9488D70C949DD80C943EFA16
:1003A0000D94D6010D94A80F0C9456600D947D11F8
:1003B0000C9467F60C94B0630C94628D0C94F3F972
:1003C0000C94DAD80C94584D0C945E600C94D9F9C6
:1003D0000C94B3630C94F3DD0C94FDCC0C94A0D876
:1003E0000D9483110C94E13F0C94E0CC0C94E33F0A
:1003F0000C9483F60C94AD630D949B110D94C30F74
:100400000C94C2FF0C94648D0C94A6D80C94D66303
:100410000D94AC140C94E73F0C9476510D94280085
:100420000C94F35B0C94F5CC0D9486390C9471F616
:100430000C94E3F90D9459110C94E53F0C94F7DDFD
:100440000C94CFF90D9477110C94B9630C94DC6380
:100450000C9454DA0D94F5100C94C5F90C94416683
:100460000C94E0D80C9475F60C94EA630C949AF60C
:100470000C94B2D80C94DE5B0C94E68B0C947A51FD
:100480000C94CB650C940E5E0C9495F60C9479F656
:100490000C944A670C9466600C946E8E0C94866F74
:1004A0000D94D4100C943D4B0C94A3D80D940901D9
:1004B0000C945A600C9448FA0C94EBF90D94D60FF6
:1004C0000C94B5650C9491F60C9452600C94C0F9A0
:1004D0000C942F940C948DF60C94AC490C945CF60F
:1004E0000C9403520D941B100C943C490C945B9497
:1004F0000D94AA140C94478D0C94F15B0D94621129
:100500000D94E90F0D94AE140C94D4FF0C94BAD74B
:100510000C94E75E0C9475D70C94FE650D94B112A3
:100520000C944C4B0C9452F64E414E494E49545942
:10053000494E46CDCCCC3D0AD7233C17B7D13877AE
:10054000CC2B329595E6241FB14F0A0000204100C4
:1005500000C84200401C4620BCBE4CCA1B0E5AAE0E
:10056000C59D7400407A10F35A00A0724E1809001D
:1005700010A5D4E80000E87648170000E40B540208
:100580000000CA9A3B000000E1F505000080969843
:1005900000000040420F000000A086010000001093
:1005A0002700000000E803000000006400000000D5
:1005B000000A00000000000100000000002C76D8B6
:1005C00088DC674F0823DFC1DFAE59E1B1B796E59C
:1005D000E3E453C63AE651997696E8E6C28426EB00
:1005E000898C9B62ED407C6FFCEFBC9C9F40F2BA13
:1005F000A56FA5F490055A2AF75C936B6CF9676DAB
:10060000C11BFCE0E40D47FEF520E6B500D0ED90FF
:100610002E0300943577050080841E080000204ECC
:100620000A000000C80C333333330F986E12831165
:1006300041EF8D2114893BE65516CFFEE6DB18D13C
:10064000844B381BF77C1D901DA4BBE4242032840E
:10065000725E228100C9F124ECA1E53D27434F4D94
:100660004D554E49434154494F4E004452595255FD
:100670004E004552524F525300494E464F0045439B
:10068000484F0047322F4733206261642070617207
:10069000616D65746572730A0057617274656E2EC0
:1006A0002E2E004D65736820706F696E74206F7513
:1006B00074206F662072616E67650A004B6C696317
:1006C0006B207A756D20466F72747365747A656EEF
:1006D0000046616C736368657220447275636B6574
:1006E00072004D6F746F72656E20616E6765736323
:1006F00068616C74657400456E642066696C652081
:100700006C6973740A00426567696E2066696C657E
:10071000206C6973740A00286E6F2066696C652905
:100720000043757272656E742066696C653A2000CC
:100730005344207072696E74696E672062797465C3
:1007400020004E6F74205344207072696E74696E7D
:10075000670A005072696E742074696D653A2000F2
:10076000496E76616C69642050696E204D6F6465D6
:100770000A000A53746174733A2046696C616D65AE
:100780006E7420757365643A20002C204C6F6E6780
:10079000657374206A6F623A2000546F74616C2034
:1007A00074696D653A20002C204661696C65643A75
:1007B00020002C2046696E69736865643A200050F9
:1007C00072696E74733A200053746174733A200036
:1007D00045202553006F66660044454255473A0060
:1007E0004D3131322053687574646F776E004D312E
:1007F000313320530042657474206BC3BC686C7441
:100800002E2E2E0042657474206865697A742E2E2F
:100810002E00534F564F4C2053563031204F4646F2
:100820002E002F2F20004D31343520533C696E644B
:1008300065783E206F7574206F662072616E676503
:100840002028302D31290A00416363656C6572618F
:1008500074696F6E3A2050003F4A206F7574206FA4
:10086000662072616E67652028302E303120746FEB
:1008700020302E33290A0046523A0020466C6F770A
:100880003A200050726F7465637465642050696E1D
:100890000A004D424C2041646A757374205A00204E
:1008A000643A0020693A0020703A0064697300439A
:1008B000290A0061626C656420286D696E20746588
:1008C0006D702000436F6C64206578747275646588
:1008D0007320617265200046696C616D656E7420DD
:1008E00072756E6F75742000486F6D6576657273F2
:1008F00061747A20616B746976004572723A205493
:100900006F6F206661722100546F6F2066617220E4
:1009100066726F6D207265666572656E63652070C4
:100920006F696E740A00454550524F4D204F4B0A77
:1009300000506F7765722D6C6F7373207265636FF3
:10094000766572792000446F6E65207072696E74EE
:10095000696E672066696C650A004D3737004D3354
:1009600031007E06790672066B065D064572726F6F
:10097000722077726974696E6720746F20454550E4
:10098000524F4D210A004D343130004D313132008B
:100990004D31303800414E474548414C54454E009A
:1009A0005072696E7465722073746F707065642024
:1009B00064756520746F206572726F72732E2046A5
:1009C000697820746865206572726F7220616E6448
:1009D00020757365204D39393920746F2072657325
:1009E000746172742E202854656D7065726174751F
:1009F00072652069732072657365742E2053657467
:100A00002069742061667465722072657374617206
:100A100074696E67290A004E6F20436865636B73C3
:100A2000756D2077697468206C696E65206E756DD0
:100A30006265722C204C617374204C696E653A209B
:100A400000636865636B73756D206D69736D6174A8
:100A500063682C204C617374204C696E653A2000E9
:100A60004C696E65204E756D626572206973206EEB
:100A70006F74204C617374204C696E65204E756DE7
:100A80006265722B312C204C617374204C696E6549
:100A90003A20004D313130005344207265616420AA
:100AA0006572726F720A002121204B494C4C206301
:100AB0006175736564206279204B494C4C206275E6
:100AC00074746F6E2F70696E0A002121204B494C9F
:100AD0004C2063617573656420627920746F6F20A8
:100AE0006D75636820696E616374697665207469E9
:100AF0006D65202D2063757272656E7420636F6D55
:100B00006D616E643A2000627573793A2070617588
:100B100073656420666F7220696E7075740A006276
:100B20007573793A2070617573656420666F722001
:100B3000757365720A00627573793A2070726F631B
:100B4000657373696E670A004D656469756D20652C
:100B50006E746665726E74004D656469756D2065AE
:100B6000726B616E6E74004D313030302053004D29
:100B700036303000363726033C3D380E2E303E12DC
:100B80001A1C180AFF430809084400014C616465F7
:100B90006E206D6D00456E746C6164656E206D6DC8
:100BA0000046696C616D656E7464757263686D652D
:100BB00073736572004520696E206D6DC2B30020AD
:100BC000082046616B746F72002008206D61780008
:100BD0002008206D696E004175746F2054656D703A
:100BE0006572617475720056206D696E204C656582
:100BF0007266616872740056206D696E200056201E
:100C00006D617820450056206D6178205A0056208D
:100C10006D617820590056206D6178205800412080
:100C20006D617820450041206D6178205A00412097
:100C30006D617820590041206D6178205800412075
:100C40004C656572666168727400412045696E7A10
:100C5000756700476568C3A47573650025697920C9
:100C6000256964202569682025696D202569730040
:100C700023646566696E652044454641554C545F62
:100C8000004B6420004B6920004B70200050494409
:100C9000204175746F74756E652066696E6973683E
:100CA0006564212050757420746865206C617374CC
:100CB000204B702C204B6920616E64204B642063B4
:100CC0006F6E7374616E74732066726F6D206265EF
:100CD0006C6F7720696E746F20436F6E66696775FD
:100CE000726174696F6E2E680A0050494420417524
:100CF000746F74756E65206661696C65642120741B
:100D0000696D656F75740A000A20436C61737369BD
:100D10006320504944200A00204B643A2000204BB5
:100D2000693A2000204B703A20002054753A200088
:100D3000204B753A2000206D61783A2000206D69C3
:100D40006E3A200020643A200020626961733A20E4
:100D500000504944204175746F74756E652073743A
:100D60006172740A00504944204175746F74756E45
:100D700065206661696C6564212054656D706572DB
:100D8000617475726520746F6F20686967680A0006
:100D9000504944204175746F74756E650050494424
:100DA000204175746F74756E65206661696C656449
:100DB0002120426164206578747275646572206ECA
:100DC000756D6265720A004572723A2075746638F4
:100DD00020666F6E74206E6F7420696E697469612D
:100DE0006C697A65642E00000C0F00FE0702260372
:100DF000BC01FFFE0AFE08FE05080806000040F0E0
:100E0000C88888987810050808060000C0F8888807
:100E1000888888F80505050600012030F83020058F
:100E200008080600002070F820202020E0050909AD
:100E30000600FF2070A8A8B888887020050606065E
:100E40000001E08CEA8C8A0A0509090600FFF8A86F
:100E50008888888888A8F8050A0A0600FE2050506D
:100E6000505088A8A8887003030306000340A040E0
:100E7000FFFFFFFFFFFFFFFFFFFFFFFFFFFFFFFF82
:100E8000FFFFFFFFFFFF0000000605FF0107070649
:100E9000020080808080800080030303060105A09B
:100EA000A0A005060606000050F85050F8500509AD
:100EB000090600FF2070A8A07028A8702005070769
:100EC000060000C8C81020409898050707060000D3
:100ED00040A0A040A890680103030602058080801E
:100EE0000309090601FF2040408080804040200324
:100EF00009090601FF80404020202040408005076E
:100F00000706000020A8702070A82005050506002F
:100F1000012020F820200203030601FFC0408005C5
:100F20000101060003F8020202060100C0C0050725
:100F30000706000008101020404080050707060043
:100F400000708898A8C8887003070706010040C091
:100F500040404040E0050707060000708808102068
:100F600040F8050707060000F808103008887005EB
:100F7000070706000010305090F81010050707060C
:100F80000000F880F00808887005070706000030A8
:100F90004080F0888870050707060000F8081010E8
:100FA0002020200507070600007088887088887058
:100FB000050707060000708888780810600205059C
:100FC000060100C0C000C0C00206060601FFC0C086
:100FD00000C0408003050506010120408040200537
:100FE0000303060002F800F803050506010180402E
:100FF0002040800507070600007088102020002090
:101000000507070600007088B8A8B88070050707B4
:10101000060000708888F8888888050707060000A1
:10102000F04848704848F0050707060000708880BF
:1010300080808870050707060000F0484848484847
:10104000F0050707060000F88080F08080F80507AB
:1010500007060000F88080F0808080050707060002
:1010600000708880809888700507070600008888CF
:1010700088F8888888030707060100E04040404060
:1010800040E00507070600003810101010906005BA
:1010900007070600008890A0C0A0908805070706F3
:1010A0000000808080808080F805070706000088A7
:1010B000D8A8888888880507070600008888C8A8F7
:1010C00098888805070706000070888888888870D7
:1010D000050707060000F08888F080808005070774
:1010E00006000070888888A8906805070706000039
:1010F000F08888F0A09088050707060000708880B7
:1011000070088870050707060000F82020202020BE
:1011100020050707060000888888888888700507EA
:1011200007060000888888885050200507070600B9
:101130000088888888A8A8500507070600008888C6
:101140005020508888050707060000888850202016
:101150002020050707060000F80810204080F8034B
:1011600009090601FFE080808080808080E005071B
:1011700007060000804040201010080309090601FE
:10118000FFE020202020202020E0050303060005AA
:101190002050880501010600FEF80303030601053F
:1011A000804020050505060000700878887805074E
:1011B000070600008080F0888888F0050505060095
:1011C000007080808870050707060000080878888E
:1011D0008888780505050600007088F0807005078E
:1011E00007060000304840E0404040050707060081
:1011F000FE708888887808700507070600008080E0
:10120000F0888888880307070601004000C0404036
:1012100040E00409090601FE100030101010109083
:101220006005070706000080808890E0908803072B
:1012300007060100C04040404040E00505050600AB
:1012400000D0A8A8A8A8050505060000B0C8888891
:101250008805050506000070888888700507070660
:1012600000FEF0888888F080800507070600FE7879
:10127000888888780808050505060000B0C88080C1
:101280008005050506000078807008F00507070650
:1012900000002020F8202020180505050600008801
:1012A000888898680505050600008888885020050C
:1012B00005050600008888A8A85005050506000059
:1012C00088502050880507070600FE88888850202F
:1012D0004080050505060000F8102040F8030909C4
:1012E0000601FF204040408040404020010909069F
:1012F00002FF808080808080808080030909060151
:10130000FF8040404020404040800503030600022B
:1013100048A890FFFFFFFFFFFFFFFFFFFFFFFFFF5A
:10132000FFFFFFFFFFFFFFFFFFFFFFFFFFFFFFFFCD
:10133000FFFFFFFF0000000605FF01070706020090
:10134000800080808080800507070600FF2070A84D
:10135000A0A87020050707060000304840E040487C
:10136000B0050505060000A8508850A80507070627
:1013700000008850F820F8202001070706020080AE
:1013800080800080808004080806010070806090E2
:10139000906010E0030101060107A00607070600A0
:1013A000007884B4A4B4847803050506010460A021
:1013B0006000E00505050600002850A05028050340
:1013C00003060001F80808030101060103E006070F
:1013D000070600007884B4A4A484780501010600FF
:1013E00007F80404040601056090906005070706ED
:1013F00000002020F8202000F80305050601044025
:10140000A02040E0030505060104C0204020C003E1
:1014100003030601052040800507070600FE8888B3
:101420008898E8808005080806000078E8E8E86801
:10143000282828020202060203C0C0030202060195
:10144000FE20C003050506010440C04040E003053E
:101450000506010540A04000E0050505060000A0C6
:10146000502850A0050A0A06000040C048506050AD
:10147000B0507810050A0A06000040C0485060507D
:10148000A8081038050A0A060000C0204830E050BD
:10149000B050781005070706000020002020408883
:1014A00070050A0A060000402000708888F88888C5
:1014B00088050A0A060000102000708888F88888CD
:1014C00088050A0A060000205000708888F888887D
:1014D00088050A0A06000068B000708888F88888C5
:1014E000880509090600005000708888F8888888F7
:1014F000050A0A060000205020708888F88888882D
:1015000005070706000078A0A0F0A0A0B80509090B
:101510000600FE708880808088701060050A0A06C8
:101520000000402000F88080F08080F8050A0A065C
:101530000000102000F88080F08080F8050A0A067C
:101540000000205000F88080F08080F8050909062E
:1015500000005000F88080F08080F8030A0A06013D
:1015600000804000E04040404040E0030A0A06019D
:1015700000204000E04040404040E0030A0A0601ED
:101580000040A000E04040404040E003090906015F
:1015900000A000E04040404040E005070706000092
:1015A000704848E8484870050A0A06000068B0001C
:1015B0008888C8A8988888050A0A06000040200084
:1015C00070888888888870050A0A06000010200044
:1015D00070888888888870050A0A060000205000F4
:1015E00070888888888870050A0A06000068B0003C
:1015F0007088888888887005090906000050007086
:101600008888888888700505050600018850205064
:10161000880509090600FF087098A8A8A8C8708066
:10162000050A0A060000402000888888888888709B
:10163000050A0A06000010200088888888888870BB
:10164000050A0A060000205000888888888888706B
:101650000509090600005000888888888888700578
:101660000A0A06000010200088885020202020044C
:10167000070706010080E0909090E08005070706CC
:101680000000708890A09088B0050808060000400F
:1016900020007008788878050808060000102000EF
:1016A0007008788878050808060000205000700847
:1016B00078887805080806000068B0007008788807
:1016C000780507070600005000700878887805083C
:1016D0000806000020502070087888780505050667
:1016E0000000702870A0780507070600FE7088804B
:1016F000887010600508080600004020007088F01F
:1017000080700508080600001020007088F08070C6
:101710000508080600002050007088F0807005075A
:101720000706000050007088F0807003080806016A
:1017300000804000C0404040E0030808060100204F
:101740004000C0404040E003080806010040A000FF
:10175000C0404040E0030707060100A000C0404031
:1017600040E0050909060000502050087888888864
:101770007005080806000068B000B0C888888805B1
:101780000808060000402000708888887005080856
:101790000600001020007088888870050808060080
:1017A00000205000708888887005080806000068CE
:1017B000B000708888887005070706000050007028
:1017C000888888700505050600012000F8002005BE
:1017D00005050600007898A8C8F00508080600006E
:1017E00040200088888888700508080600001020BE
:1017F0000088888888700508080600002050008846
:101800008888887005070706000050008888888847
:1018100070050A0A0600FE102000888888502040C3
:10182000800509090600FE8080F0888888F08080A5
:101830000509090600FE5000888888502040805322
:101840004F564F4C205356303100576965646572CE
:10185000682E206E2E205374726F6D612E004B6FB8
:101860006E66696775726174696F6E00256C642EAF
:1018700025696D00476573616D74204578747275D4
:101880006469657274004CC3A46E67737465204408
:101890007275636B7A656974003E200047657361F9
:1018A0006D746520447275636B7A656974004B6F63
:1018B0006D706C6574746520447275636B65004768
:1018C0006573616D746520447275636B65003132B8
:1018D00035004245443A4550434F53203130304B58
:1018E0000052756E617761792057617463683A20A0
:1018F0004F4E004D61782054656D700032373500D1
:101900004D696E2054656D700045313A2045504355
:101910004F53203130304B004E65747A7465696CDA
:10192000004D45414E2057454C4C0050726F746F2E
:101930006B6F6C6C00312E300042617564726174A3
:1019400065003131353230300052414D5053203135
:101950002E33004E65747A2D4E6976656C6C696520
:1019600072756E6700323032302D30382D323800CB
:10197000447275636B65722D537461746973746915
:101980006B00546865726D6973746F72656E0042A6
:101990006F6172642D496E666F00447275636B658A
:1019A000722D496E666F004D313030300053442D3A
:1019B000447275636B2061626272656368656E0074
:1019C00053442D447275636B20666F727473657433
:1019D0007A656E0053746F70004D656469756D2093
:1019E000676574617573636874004D323100C39C20
:1019F0006265722064656E20447275636B65720067
:101A00004B65696E204D656469756D004A75737428
:101A1000696572756E670053442D447275636B205F
:101A200070617573696572656E004B6E6F706620CC
:101A30006472C3BC636B656E20756D0044C3BC7378
:101A400065206175667A756865697A656E0000461D
:101A5000696C616D656E742065696E6C6567656E35
:101A600000756E64204B6E6F7066206472C3BC6339
:101A70006B656E00756D20666F72747A7573657430
:101A80007A656E00576172746520617566004C61FD
:101A900064656E206465730046696C616D656E7483
:101AA000732E2E2E004B6E6F7066206472C3BC6363
:101AB0006B656E20756D00447275636B20666F7286
:101AC000747A757365747A656E0000576172746517
:101AD0002061756600466F72747365747A656E2056
:101AE00064657300447275636B732E2E2E0057610C
:101AF0007274652061756600456E746C6164656E14
:101B0000206465730046696C616D656E74732E2E7A
:101B10002E004E6976656C6C696572656E2066652F
:101B20007274696721004EC3A46368737465204BA7
:101B30006F6F7264696E617465002569202F2025BE
:101B40007500473239205331004B6C69636B207A42
:101B5000756D205374617274656E00486F6D696EA7
:101B6000672058595A0045636B656E206E6976652B
:101B70006C6C696572656E00417573626C656E644C
:101B800068C3B668650042657474206E6976656CDA
:101B90006C696572656E00556E526574205600550D
:101BA0006E526574206D6D005A2D537072756E679C
:101BB000206D6D00562045696E7A75670045696E27
:101BC0007A7567206D6D004175746F6D2E204569C3
:101BD0006E7A7567001FE020102010201010201072
:101BE000202010201030300840048003001FE03F08
:101BF000F03FF03FF01FE01FE03FF03FF03FF00FFD
:101C0000C0078003003FFFF038007030FC3020FC3C
:101C1000102078102030102C00D02E31D02F7BD007
:101C20002F7BD02E31D02C00D020301020781020E7
:101C3000FC1030FC303800703FFFF03FFFF0380000
:101C4000703186302387102787902F87D02F03D0BD
:101C50002030102078102078102030102F03D02F43
:101C600087D02787902387103186303800703FFF58
:101C7000F01FFFF81FFFF8041040020820020820A0
:101C8000041040082080104100104100082080040A
:101C900010400000001FFFF81FFFF81EF79C043FD4
:101CA000633E0C6363633C6063630C6063630C3C82
:101CB00063630C1E36630C0336630C0336630C63DC
:101CC0001C630C7E1C3E3F3C081C3F2568753A2572
:101CD000303268750025303268753A2530326875C3
:101CE00000202020202020200020520020204D36DF
:101CF0003033200020204D34313220530046696CAF
:101D0000616D656E742072756E6F75742073656E8B
:101D1000736F723A0020550046696C616D656E7490
:101D2000206C6F61642F756E6C6F6164206C656EE2
:101D3000677468733A0020204D32303920530041D7
:101D400075746F2D526574726163743A20533D301F
:101D500020746F2064697361626C652C203120747B
:101D60006F20696E7465727072657420452D6F6E98
:101D70006C79206D6F766573206173207265747263
:101D80006163742F7265636F7665720020204D3237
:101D900030382053005265636F7665723A20533CA9
:101DA0006C656E6774683E20463C756E6974732F6F
:101DB0006D3E0020570020204D3230372053005216
:101DC0006574726163743A20533C6C656E67746825
:101DD0003E20463C756E6974732F6D3E205A3C6CF4
:101DE0006966743E0020204D343133205300506F1B
:101DF0007765722D4C6F7373205265636F766572D1
:101E0000793A0020204D3330312050005049442091
:101E100073657474696E67733A0020460020480049
:101E200020204D3134352053004D61746572696155
:101E30006C2068656174757020706172616D657485
:101E40006572733A002020473239205334205A00FB
:101E5000202047323920533320490020204D34328E
:101E6000302053004D65736820426564204C6576D0
:101E7000656C696E673A0020204D3230362058007C
:101E8000486F6D65206F66667365743A00204A007E
:101E900020204D323035204200416476616E63650A
:101EA000643A20423C6D696E5F7365676D656E7460
:101EB0005F74696D655F75733E20533C6D696E5F3D
:101EC00066656564726174653E20543C6D696E5F41
:101ED00074726176656C5F66656564726174653E97
:101EE000204A3C6A756E635F6465763E002054004C
:101EF00020204D323034205000416363656C6572A0
:101F00006174696F6E2028756E6974732F7332293E
:101F10003A20503C7072696E745F616363656C3E19
:101F200020523C726574726163745F616363656CB7
:101F30003E20543C74726176656C5F616363656CCE
:101F40003E0020204D3230312058004D6178696DBF
:101F5000756D20416363656C65726174696F6E2095
:101F600028756E6974732F7332293A0020204D3220
:101F700030332058004D6178696D756D2066656558
:101F80006472617465732028756E6974732F732988
:101F90003A0053746570732070657220756E6974B1
:101FA0003A0020440020204D32303020530020449D
:101FB000697361626C65640A0046696C616D656E87
:101FC000742073657474696E67733A0020204D3114
:101FD00034392043203B20556E69747320696E208C
:101FE00043656C736975730A0020286D6D290020A4
:101FF00020473231202020203B20556E6974732009
:10200000696E206D6D0024F4D43050C38E20C2A2BE
:102010004017828B7011127A910D816CD90AA861D8
:10202000E108C7586607615143061E4B5D05C1456F
:10203000A7041A411104093D980371393103403650
:10204000DB0265339102D4305402802E1D02632CD2
:10205000EE01752AC501B028A001102781018F2546
:1020600064012B244B01E0223401AC211F018D209F
:102070000D01801FFC00841EED00971DDF00B81CC1
:10208000D200E61BC600201BBC00641AB200B219C5
:10209000A8000A19A0006A189900D11791004017EA
:1020A0008B00B516840031167E00B31579003A1501
:1020B0007300C7146F0058146A00EE13660088138B
:1020C000630025135E00C7125B006C1257001512E7
:1020D0005400C111510070114F0021114B00D61056
:1020E00049008D1047004610440002104200C00F06
:1020F0004000800F3E00420F3C00060F3B00CB0E1D
:102100003800930E37005C0E3500270E3400F30DB7
:102110003200C10D3100900D3000600D2E00320DE7
:102120002D00050D2C00D90C2B00AE0C2900850CC0
:1021300029005C0C2700350C27000E0C2600E80B4C
:102140002400C40B2400A00B23007D0B23005A0B9A
:102150002100390B2100180B2000F80A1F00D90AB2
:102160001E00BB0A1E009D0A1D00800A1D00630A96
:102170001C00470A1B002C0A1B00110A1A00F70951
:102180001A00DD091900C4091900AB0919009209E8
:1021900017007B091800630917004C09160036095F
:1021A0001600200916000A091500F5081500E008B8
:1021B0001400CC081400B8081400A40814009008F7
:1021C00013007D0812006B0813005808120046081F
:1021D0001200340811002308110012081100010830
:1021E0001100F0071000E0071000D0071000C00732
:1021F0001000B0070F00A107100091070E00830721
:102200000F0074070F0065070E0057070E004907FF
:102210000E003B070D002E070E0020070D001307D0
:102220000D0006070D00F9060C00ED060D00E00696
:102230000C00D4060C00C8060C00BC060C00B0064E
:102240000C00A4060B0099060C008D060B008206FC
:102250000B0077060B006C060B0061060A005706A0
:102260000B004C060A0042060A0038060A002E0639
:102270000A0024060A001A060A00100609000706CA
:102280000A00FD050900F4050900EB050900E20557
:102290000900D9050900D0050900C7050900BE05D8
:1022A0000900B5050800AD050800A50509009C0555
:1022B0000800940508008C050800840508007C05CA
:1022C0000800740508006C050700650508005D0539
:1022D0000700560508004E050700470507004005A2
:1022E000080038050700310507002A050700230507
:1022F00007001C050600160507000F050700080566
:10230000060002050700FB040600F5040700EE04C2
:102310000600E8040600E2040700DB040600D5041A
:102320000600CF040600C9040600C3040600BD046D
:102330000600B7040600B1040500AC040600A604BC
:102340000600A00405009B04060095040500900407
:1023500006008A04050085040500800406007A044E
:10236000050075040500700405006B040500660493
:102370000500610405005C040500570405005204D3
:1023800005004D04050048040500430405003E0413
:1023900004003A04050035040500300404002C0450
:1023A000050027040400230405001E0404001A0489
:1023B000040016040500110404000D0404000904BF
:1023C00005000404040000040400FC030400F803F6
:1023D0000400F4030400F0030400EC030400E80329
:1023E0000400E4030400E0030400DC030400D80359
:1023F0000400D4030400D0030400CC030400C80389
:102400000300C503030024F404D9201BC40C5C0E94
:102410009804C4095F0265077101F405F900FB0423
:10242000B30048048700C103690058035500030343
:102430004500BE023A008402310053022A002902FC
:10244000250004022000E4011C00C8011900AF01AE
:10245000170098011400840113007101100061013C
:10246000100051010E0043010D0036010B002B013D
:102470000B0020010B00150109000C0109000301EC
:102480000800FB000800F3000800EB000700E40070
:102490000600DE000600D8000600D2000600CC00D0
:1024A0000500C7000500C2000500BD000400B9001A
:1024B0000400B5000400B1000400AD000400A90050
:1024C0000400A5000300A20003009F0004009B007D
:1024D00003009800030095000200930003009000A1
:1024E00003008D0002008B000300880002008600BC
:1024F000020084000300810002007F0002007D00D2
:1025000002007B00020079000200770001007600E3
:1025100002007400020072000100710002006F00EE
:1025200002006D0001006C0002006A0001006900F9
:102530000200670001006600010065000100640000
:1025400002006200010061000100600001005F0004
:1025500002005D0001005C0001005B0001005A0008
:102560000100590001005800010057000100560009
:102570000100550001005400010053000000530009
:1025800001005200010051000100500001004F0005
:1025900001004E0000004E0001004D0001004C0003
:1025A00001004B0000004B0001004A0001004900FF
:1025B00001004800000048000100470001004600FB
:1025C00000004600010045000000450001004400F5
:1025D00001004300000043000100420000004200EF
:1025E00001004100000041000100400001003F00E7
:1025F00000003F0001003E0000003E0001003D00E1
:1026000000003D0001003C0000003C0000003C00D8
:1026100001003B0000003B0001003A0000003A00CE
:1026200001003900000039000100380000003800C6
:1026300000003800010037000000370001003600BC
:1026400000003600000036000100350000003500B3
:1026500000003500010034000000340000003400A8
:10266000010033000000330000003300010032009D
:102670000000320000003200010031000000310093
:102680000000310001003000000030000000300088
:1026900001002F0000002F0000002F0000002F007D
:1026A00001002E0000002E0000002E0001002D0071
:1026B00000002D0000002D0000002D0001002C0066
:1026C00000002C0000002C0000002C0001002B005A
:1026D00000002B0000002B0000002B0001002A004E
:1026E00000002A0000002A0000002A000100290042
:1026F0000000290000002900000029000000290036
:102700000100280000002800000028000000280028
:10271000000028000100270000002700000027001B
:10272000000027000000270001002600000026000E
:102730000000260000002600000026000100250001
:1027400000002500000025000000250000002500F5
:1027500000002500010024000000240000002400E7
:1027600000002400000024000100230000002300DA
:1027700000002300000023000000230000002300CD
:1027800000002300010022000000220000002200BF
:1027900000002200000022000000220001002100B1
:1027A00000002100000021000000210000002100A5
:1027B0000000210000002100010020000000200096
:1027C0000000200000002000000020000000200089
:1027D000000020000000200001001F0000001F007A
:1027E00000001F0000001F0000001F0000001F006D
:1027F00000001F0001001E0000001E0000001E005F
:1028000000001E000000043700001E290000511BBC
:1028100000005810000010090000CC0400007802ED
:102820000000410100006F70656E00545249474737
:10283000455245440066696C616D656E74007A5F4F
:102840006D696E00795F6D696E00785F6D696E000D
:102850005265706F7274696E6720656E6473746F11
:1028600070207374617475730A00486F6D696E67C8
:102870002067657363686569746572740057617277
:102880006E696E673A20486F6D696E672042756D9C
:10289000702044697669736F72203C20310A000011
:1028A000004842000048420000804002020400004C
:1028B000A0400000A04000000040FFFFFF02000019
:1028C0000000000000000000000000000000000008
:1028D00000000000000000000000000000000000F8
:1028E00000000000000000000000000000000000E8
:1028F00000000000000000000000000000000000D8
:1029000000000000000000000000000000000000C7
:1029100000000000000000000000000000000000B7
:1029200000000000000000000000000000000000A7
:102930000000000000000000000000000000000097
:102940000000000000000000000000000000000087
:10295000000000000000000000000000000001FF77
:10296000FE001E7807E0003E00F3C003C00007FF32
:10297000FE00FE7F07E0003E07F3F803C0000FFFF4
:10298000FE01FE7F03F0007E0FF3FC03C0001FFF7B
:10299000FE03FE7F83F0007E1FF3FE03C0001FFFD7
:1029A000FE07FE7FC1F800FC3FF3FF03C0003F803D
:1029B000000FE007E1F800FC7F003F83C0003F000C
:1029C000000FE007E0FC01F87F003F83C0003F00FC
:1029D000000FC003E0FC01F87E001F83C0003F0031
:1029E000000FC003E07C01F07E001F83C0003F8029
:1029F000001F8001F07E03F0FC000FC3C0003FE029
:102A0000001F8001F07E03F0FC000FC3C0001FFF19
:102A1000F81F8001F03E03E0FC000FC3C00007FF79
:102A2000FE1F8001F01F07C0FC000FC3C00003FFA2
:102A3000FF1F8001F01F8FC0FC000FC3C00000000B
:102A40007F9F8001F01F8FC0FC000FC3C0000000FB
:102A50003F9F8001F00F8F80FC000FC3C00000007B
:102A60001F9FC003F00FDF80FE001FC3C0000000E7
:102A70001F8FC003E007DF007E001F83C00000003F
:102A80001F8FE007E007FF007F003F83E0000000AA
:102A90003F8FE007E003FE007F003F83E0001FFF61
:102AA000FF07FE7FC003FE003FF3FF03FFFC1FFF95
:102AB000FF03FE7F8003FE001FF3FE03FFFC1FFFEA
:102AC000FE01FE7F0001FC000FF3FC01FFFC1FFF75
:102AD000FC00FE7F0001FC0007F3F800FFFC1FFF75
:102AE000F0001E780000F80000F3C0003FFC00007A
:102AF00000000000000000000000000000000000D6
:102B000000000000000000000000000000000000C5
:102B100000000000000000000000000000000000B5
:102B20000000101000A34001080000000000000099
:102B300000001010008400010800000000000000E8
:102B400000001830008400010800000000000000B0
:102B5000000014538FA7471F0F91000000000000D2
:102B60000000145450A448A10851000000000000C7
:102B70000000129450A44FA1085100000000000072
:102B80000000111450A4482108510000000000006A
:102B90000000111450A448A1084A000000000000E1
:102BA000000010138FA4471F0F84000000000000D6
:102BB000000000000000000000080000000000000D
:102BC00000000000000000000010000000000000F5
:102BD00000000000000000000000000000000000F5
:102BE00000000000000000000000000000000000E5
:102BF0000210000003E000000000000000000000E0
:102C0000022000000410000000100000000000007E
:102C1000024000000400000000100000000000005E
:102C20000381CB8F84039EE7C859CE70000000005B
:102C300002822C508404511428522888000000007D
:102C40000243E850840451142853E8600000000057
:102C50000222085084045114285208100000000079
:102C6000021228518414511428D228880000000030
:102C70000209C84E83E39117C749C87000000000DD
:102C800000000000800000040000000000000000C0
:102C90000000001F00000004000000000000000011
:102CA0000000000000000000000000000000000024
:102CB000000000000000000000000000000001FF14
:102CC000FFFFFFFFFFFFFFFFFFFFFFFF0FFFFFFF04
:102CD000FFFFFFFFFFFFFFFFFFFF1E0000000000E0
:102CE000000000000007FFFF3800000000000000A7
:102CF00000000003FFFF7000000000000000000063
:102D00000001FFFF60000000000000000000000064
:102D1000FFFF6000000000000000000000007FFFD7
:102D2000C000000000000000007800003FFFC00F5E
:102D3000C0FC00000000007818001FFFC03FE1FF4A
:102D40000000000000783C000FFFC07FF3FF800010
:102D5000000000783C0007FFC0FFFFFFC00000003C
:102D600000783C0003FFC1F87F87E0000000007896
:102D7000000001FFC1F03F03E00000000078000008
:102D800000FFC1E01E01E01F0003E0783C03F07F7C
:102D9000C1E01E01E07FC00FF8783C07FC3FC1E0B6
:102DA0001E01E1FFE01FFC783C0FFE1FC1E01E0189
:102DB000E3FFF03FFE783C1FFE0FC1E01E01E3F38E
:102DC000F83F3E783C3F3F07C1E01E01E7E0FC7C56
:102DD0001F783C3E1F07C1E01E01E7C07C7C0F78D6
:102DE0003C3C0F03C1E01E01E7807C780F783C3C3F
:102DF0000F03C1E01E01E7803C7800783C3C0F03E4
:102E0000C1E01E01E7803C7800783C3C0F03C1E044
:102E10001E01E7803C7800783C3C0F03C1E01E01B6
:102E2000E7C03C7800783C3C0F03C1E01E01E3E0C2
:102E30003C78007C3C3C0F03C1E01E01E3FF3FF8FF
:102E4000007FBC3C0F03C1E01E01E1FF3FF8003FE3
:102E5000BFFC0F03C1E01E01E0FF3FF8001FBFFCF5
:102E60000F03C1E01E01E07F3FF8000FBFFC0F031E
:102E7000600000000000000000000000000760008B
:102E800000000000000000000000000670000000CC
:102E90000000000000000000000E380000000000EC
:102EA000000000000000001C1E00000000000000E8
:102EB0000000000000780FFFFFFFFFFFFFFFFFFF94
:102EC000FFFFFFF001FFFFFFFFFFFFFFFFFFFFFF1F
:102ED000FF8070012C0190012701B0012201C00187
:102EE0001D01F00118011002130130020E016002F1
:102EF000090190020401C002FF000003FA00400330
:102F0000F5008003F000D003EB002004E60070041D
:102F1000E100E004DC004005D700C005D200400617
:102F2000CD00D006C8008007C3003008BE00F008FE
:102F3000B900C009B400B00AAF00B00BAA00D00CB1
:102F4000A500000EA000500F9B00C010960050126C
:102F5000910000148C00C0158700B0178200B019D2
:102F60007D00D01B7800001E730040206E00902270
:102F70006900F024640040275F0090295A00E02B8C
:102F80005500102E500020304B0010324600E03328
:102F9000410090353C001037370070383200A039BE
:102FA0002D00B03A2800A03B2300603C1E00103DDD
:102FB0001900903D1400103E0F00703E0A00C03E04
:102FC0000500003F0000403FFBFF803FF6FFC03F91
:102FD000F1FF68747470733A2F2F6D61726C696EB3
:102FE00066772E6F726700322E302E362E3100201B
:102FF00020506C616E6E65724275666665724279CC
:103000007465733A20002046726565204D656D6FCA
:1030100072793A2000436F6D70696C65643A205391
:10302000657020323520323032300A00204C617316
:103030007420557064617465643A20323032302DEA
:1030400030382D3238207C20417574686F723A20F8
:10305000284B656E6720436F6D7075746572732CB5
:1030600020574B290A00322E302E362E310A004DC1
:1030700061726C696E0020536F66747761726520AF
:1030800052657365740A00205761746368646F67E2
:103090002052657365740A002042726F776E206F4C
:1030A00075742052657365740A00204578746572E2
:1030B0006E616C2052657365740A00506F7765729B
:1030C00055700A006175746F25632E6700473238AA
:1030D0005859004D31303031006572726F7220776F
:1030E000726974696E6720746F2066696C650A0086
:1030F000446F6E6520736176696E672066696C65E2
:103100002E0A004D323900456E6473746F70700082
:103110002553202563202563202563202563006532
:103120006E6473746F7073206869743A20004CC3C6
:10313000BC667465720044C3BC73650042657474F8
:10314000205A0048617570746D656EC3BC00242000
:10315000457874722E20566F7277C3A4726D656EB7
:103160000024204265747420566F7277C3A4726D78
:10317000656E0041626BC3BC686C656E0042616243
:103180007973746570205A00466C7573737261743C
:1031900065004765736368772E002053697A653A46
:1031A000200043616E6E6F74206F70656E207375C2
:1031B000626469722000534420496E69742046613C
:1031C000696C0053442063617264206F6B0A006F66
:1031D00070656E526F6F74206661696C65640A0079
:1031E000766F6C756D652E696E6974206661696CA9
:1031F00065640A004E6F20534420636172640A00C4
:103200004D3234004D32332025730046696C652001
:1032100073656C65637465640A0046696C65206F4C
:1032200070656E65643A2000454E44205355425205
:103230004F5554494E450A002220706F73002220DA
:10324000706172656E743A2200535542524F555464
:10325000494E452043414C4C207461726765743A75
:10326000220053756263616C6C204F766572666CE8
:103270006F77004578636565646564206D617820CB
:10328000535542524F5554494E45206465707468F9
:103290003A310A0044656C6574696F6E2066616935
:1032A0006C65642C2046696C653A200046696C6543
:1032B0002064656C657465643A0057726974696E60
:1032C0006720746F2066696C653A200066726573CA
:1032D0006800646F696E67004E6F77200047323672
:1032E0002044C3BC7365206175666865697A656E44
:1032F00000473236206865697A742042657474002C
:1033000057616974696E6720666F722068656174C1
:1033100075702E0A004665737465204CC3A46E67F1
:1033200065205072696D65005072696D696E672025
:10333000666572746967004D616E75616C207072AC
:10334000696D696E672E2E2E0047323620766572C3
:103350006C617373656E003F537065636966696580
:103360006420582C5920636F6F7264696E617465B4
:10337000206F7574206F6620626F756E64732E0AFD
:10338000003F28522965706561742076616C75650F
:10339000206E6F7420706C61757369626C653B2080
:1033A0006D757374206265206174206C656173743F
:1033B00020312E0A003F5370656369666965642099
:1033C0006E6F7A7A6C652074656D70657261747564
:1033D0007265206E6F7420706C61757369626C65C4
:1033E0002E0A003F537065636966696564206669EB
:1033F0006C616D656E742073697A65206E6F7420E0
:10340000706C61757369626C652E0A003F5370655C
:10341000636966696564207072696D65206C656EAC
:10342000677468206E6F7420706C61757369626C6C
:10343000652E0A003F537065636966696564206E96
:103440006F7A7A6C652073697A65206E6F7420706C
:103450006C61757369626C652E0A003F5265747207
:10346000616374696F6E204D756C7469706C696509
:1034700072206D7573742062652073706563696670
:103480006965642E0A003F53706563696669656407
:103490002052657472616374696F6E204D756C742F
:1034A00069706C696572206E6F7420706C617573E1
:1034B00069626C652E0A003F5370656369666965D1
:1034C00064206C6179657220686569676874206E34
:1034D0006F7420706C61757369626C652E0A0043AD
:1034E000292E0A003F53706563696669656420622E
:1034F00065642074656D7065726174757265206EA7
:103500006F7420706C61757369626C65202834304B
:103510002D00473236207374617274696E672E2EE7
:103520002E0A0020746F6F206C6F6E6720657874B0
:10353000727573696F6E2070726576656E746564FE
:103540000A0020636F6C6420657874727573696F0C
:103550006E2070726576656E7465640A00DB0FC953
:103560003F45BCDA3F8FB30240FCF02740569461E0
:1035700040FE4B9B4084A5D840E0231841346A5656
:1035800041E859974164DBD5416E271742B4B755DE
:1035900042CE1A9742C8AED542B5885A43D4068463
:1035A000BFA65FA7BF7443E0BF10B11AC01C2C5860
:1035B000C0E8F697C0B849D6C04E4E17C124D355BF
:1035C000C1802497C1A0B5D5C1121A17C244AE5507
:1035D000C2781797C26CACD5C267885AC37C3C3E90
:1035E0005E2B3D3F2F5B5D3B2C2A225C00496E76B3
:1035F000616C69642065787472756465720A002074
:103600000820C39C42455253434852495454454EA6
:10361000004D415854454D5020747269676765727A
:10362000656400200820554E544552534348524982
:103630005454454E004D494E54454D5020747269C6
:1036400067676572656400202F002042403A0020C1
:10365000403A0020573A003F005765726B73656926
:103660006E7374656C6C756E67656E00447275631D
:103670006B206162676562726F6368656E004D32D0
:10368000350050617573652E2E2E00454550524F02
:103690004D2056657273696F6E204572726F7200AD
:1036A000454550524F4D20496E64657820457272F1
:1036B0006F7200454550524F4D2043524320457292
:1036C000726F720049676E6F726500526573657440
:1036D000656E004B6F6E6669672E206C6164656E67
:1036E000004B6F6E6669672E20737065696368654D
:1036F000726E004572772E2045696E7374656C6C2E
:10370000756E67656E0061757300616E0046494CA9
:10371000414D454E5420454E544C4144454E004683
:10372000494C414D454E54204C4144454E0046497C
:103730004C414D454E54205745434853454C00534A
:1037400074616E646172647765727465206C616423
:10375000656E00242045696E7374656C6C756E67C8
:10376000656E0052756E6F75742D53656E736F7252
:10377000004D37303220542564004D363030204221
:103780003020542564004D373032203B2564004DF5
:1037900037303120542564004D373032004D3730FA
:1037A00031004D36303020423000447275636B205A
:1037B000776569746572004D65687220656E746C1A
:1037C0006164656E00464F5254532E204F50544949
:1037D0004F4E454E3A00445255434B2050415553AD
:1037E0004945525400202044C3BC73653A2000442C
:1037F0007275636B206973740070617573696572AB
:10380000742E2E2E0000576172746520617566203B
:1038100064656E0053746172742064657300466958
:103820006C616D656E747765636873656C732E2E5D
:103830002E0057617274652061756600486572617B
:1038400075736E61686D65006465732046696C61AF
:103850006D656E74732E2E2E0044C3BC7365206894
:1038600065697A7420617566006269747465207791
:10387000617274656E2E2E2E0000486F74656E6442
:1038800020746F6F20636F6C640A004D3630303ADD
:10389000207A75206B616C740050726573732062BE
:1038A0007574746F6E20746F2068656174206E6F1C
:1038B0007A7A6C650A004D32342053256C642054AA
:1038C000256C64004739322E392045257300473175
:1038D00020462564004739322E39205A2573004787
:1038E00031205A302046323030004731205825737D
:1038F00020592573204633303030004D343230208B
:10390000532569205A2573004D31303620502569E2
:1039100020532569004D31303920532569004D3140
:10392000393020532569004D323030204425730052
:1039300047323852305859004739322E39204530F5
:10394000205A300A47315A2573004D343230205303
:1039500030205A300020496E76616C6964206578A9
:1039600074727564657220000000000000000000A1
:10397000000000000000914300007A4300009B43D8
:1039800045696E7374656C6C2E206765737065692C
:103990002E0053657474696E67732053746F72657B
:1039A000642028004269747465206E6575737461C3
:1039B0007274656E00445255434B4552204745533F
:1039C000544F5050540025533A202553004142474C
:1039D0004542524F4348454E005072696E746572BD
:1039E0002068616C7465642E206B696C6C282920DA
:1039F00063616C6C6564210A006563686F3A004519
:103A000072726F723A000A4D656173757265642057
:103A1000706F696E74733A0A00337833206D657382
:103A2000682E205A206F66667365743A200047320C
:103A300036206162676562726F6368656E00426519
:103A400077656765205A0041425300504C41002081
:103A50002573206D6D0020302C312020206D6D00ED
:103A600020312C302020206D6D0031302C30202072
:103A7000206D6D0041636873656E206265776567D0
:103A8000656E00486F74656E64207A75206B616C9A
:103A90007400426577656765204578747275646562
:103AA00072004265776567652059004265776567F2
:103AB0006520580046696C616D656E74207765639A
:103AC0006873656C6E0046696C616D656E74206527
:103AD0006E746C6164656E0046696C616D656E74D0
:103AE000206C6164656E0062656E75747A657264DF
:103AF00065662E204865697A656E002420566F72CF
:103B000077C3A4726D656E005A7572C3BC636B0097
:103B100000002100240027002A002D00300033007F
:103B200001010000040107010A0100002200250034
:103B300028002B002E003100340002010000050196
:103B400008010B01000020002300260029002C00A2
:103B50002F003200000100000301060109010505E4
:103B60000505070508080808020202020A0A0808F3
:103B70000404040401010101010101010303030321
:103B800003030303040707070C0C0C0C0C0C0C0CB0
:103B90000202020206060606060606060B0B0B0BC1
:103BA0000B0B0B0B010210202008081020401020E6
:103BB00040800201020108040201010204081020F1
:103BC00040808040201008040201800402018040EF
:103BD0002010080402010804020101020408102058
:103BE0004080010204081020408000000A0B0209F6
:103BF0000C0D0E0807030401000000000000000087
:103C000000000000000000000000000000000000B4
:103C10000000000000001211100000000000000071
:103C20000000000000000000000000000000000094
:103C30004B3A473A41626272656368656E0042655D
:103C4000776567756E67004D383400426574742D72
:103C50004E6976656C6C696572756E670053746148
:103C600072746520447275636B00447275636B6592
:103C70006E0043616E6E6F7420656E7465722073A2
:103C800075626469723A2000022E2E004D6F746FC7
:103C900072656E206465616B746976696572656EC4
:103CA000004175746F20486F6D65004732380044DD
:103CB0007275636B20766F6D204D656469756D005C
:103CC000447275636B2070617573696572742E2E12
:103CD0002E00566F72686572202573257325732038
:103CE000686F6D656E00496E736572742066696CED
:103CF000616D656E7420616E6420707265737320EF
:103D0000627574746F6E0A00534F564F4C205356B1
:103D100030312062657265697400447275636B743A
:103D20002E2E2E00220A00556E6B6E6F776E20636A
:103D30006F6D6D616E643A2022006F70656E206653
:103D400061696C65642C2046696C653A20002045E9
:103D50003A00205A3A0020593A00452053746570C1
:103D6000732F6D6D005A2053746570732F6D6D0045
:103D7000592053746570732F6D6D0058205374650E
:103D800070732F6D6D0042657374C3A474696765A9
:103D90006E004D3432380046696C616D656E74009A
:103DA0004A756E6374696F6E204465760042657370
:103DB00063686C65756E6967756E670047657363E8
:103DC0006877696E6469676B656974005365747AB6
:103DD0006520486F6D657665727361747A004EC3B5
:103DE000A463687374652045636B650046657274EF
:103DF000696700576569746572002062797465733C
:103E00003B2063726320004E6F20454550524F4D5A
:103E10002E0A00454550524F4D206461746173690C
:103E20007A65206572726F722E0A002073746F7249
:103E300065642073657474696E677320726574724B
:103E40006965766564202800202863616C63756C61
:103E50006174656429210A0020213D2000454550F8
:103E6000524F4D20435243206D69736D61746368F6
:103E7000202D202873746F726564292000496E64B8
:103E800065783A2000204D61726C696E3D5638317C
:103E9000290A00454550524F4D2076657273696F6F
:103EA0006E206D69736D61746368202845455052BA
:103EB0004F4D3D0048617264636F646564204465E2
:103EC0006661756C742053657474696E6773204CF9
:103ED0006F616465640A003B20000000FA43000043
:103EE000FA430000A0400000C8410000A0420000CA
:103EF000A0420000C8430080CF43F4010000F40159
:103F0000000064000000E80300004361703A0043D1
:103F100048414D4245525F54454D504552415455DC
:103F2000524500424142595354455050494E470072
:103F300041524353004D4F54494F4E5F4D4F4445FE
:103F40005300544845524D414C5F50524F544543E5
:103F500054494F4E004C4F4E475F46494C454E41E9
:103F60004D45004155544F5245504F52545F5344B4
:103F70005F535441545553005344434152440050FD
:103F8000524F4D50545F535550504F525400454D71
:103F9000455247454E43595F5041525345520043A5
:103FA0004153455F4C494748545F42524947485442
:103FB0004E45535300544F47474C455F4C49474883
:103FC000545300534F4654574152455F504F574545
:103FD00052004255494C445F50455243454E5400AF
:103FE0004C4556454C494E475F44415441005A5F49
:103FF00050524F42450052554E4F55540041555472
:104000004F4C4556454C005052494E545F4A4F4222
:104010000050524F4752455353004155544F52455B
:10402000504F52545F54454D5000564F4C554D45DE
:104030005452494300454550524F4D0042494E416C
:1040400052595F46494C455F5452414E5346455282
:104050000053455249414C5F584F4E5F584F4646BA
:10406000004649524D574152455F4E414D453A4DEC
:1040700061726C696E20322E302E362E312028531C
:10408000657020323520323032302031333A3131D0
:104090003A35352920534F555243455F434F4445E8
:1040A0005F55524C3A68747470733A2F2F67697475
:1040B0006875622E636F6D2F4D61726C696E466913
:1040C000726D776172652F4D61726C696E2050520E
:1040D0004F544F434F4C5F56455253494F4E3A3120
:1040E0002E30204D414348494E455F545950453A82
:1040F000534F564F4C20535630312045585452554B
:104100004445525F434F554E543A3120555549442A
:104110003A63656465326132662D343161322D3423
:104120003734382D396231322D6335356336326696
:1041300033363766660A00656E7175657565696E3A
:10414000672022006F6B00526573656E643A200031
:104150004F46460A00466164652048656967687491
:1041600020004661696C656420746F20656E616231
:104170006C6520426564204C6576656C696E670AE3
:10418000004D65736820426564204C6576656C203F
:10419000646174613A0A00496E76616C6964206DED
:1041A0006573682E0A00206E6F7420656E746572E8
:1041B00065642E0A00206F6620004D424C20473275
:1041C0003920706F696E7420004A206F7574206FFB
:1041D000662072616E67652028302D0049206F755A
:1041E00074206F662072616E67652028302D004D47
:1041F0006573682070726F62696E6720646F6E65A8
:104200002E0A005374617274206D65736820707299
:104210006F62696E6720776974682022473239209F
:104220005331222066697273742E0A004732380AAD
:1042300047323920533200686173206E6F20646109
:1042400074612E0A004D65736820426564204C65D8
:1042500076656C696E67200053206F7574206F66F9
:104260002072616E67652028302D35292E0A004D99
:1042700034323120696E636F7272656374207061CD
:1042800072616D657465722075736167650A0020DF
:104290004D393220580020204D61783A20002020EE
:1042A0004D696E3A2000536F667420656E647374B6
:1042B0006F70733A200020436F756E7420583A0077
:1042C000453100626564002C2073797374656D203C
:1042D00073746F7070656421204865617465725FE6
:1042E00049443A20004845495A454E204552464FD8
:1042F0004C474C4F530048656174696E6720666196
:10430000696C656400202D20496E76616C696420BB
:104310006578747275646572206E756D6265722061
:10432000210A002008204E49434854204552524556
:104330004943485400546865726D616C2052756E33
:104340006177617900000A01140211241FBECFEFCA
:10435000D1E2DEBFCDBF00E00CBF12E0A0E0B2E0D2
:10436000E8EDF5E902E00BBF02C007900D92AC3E0C
:10437000B107D9F726E1ACEEB2E001C01D92A7313A
:10438000B207E1F711E2C4EAD1E200E006C02197EA
:104390000109802FFE010F942B47C33AD10780E01B
:1043A0000807A9F70F945F320D94DA4A0C940000C5
:1043B0002F923F924F925F926F927F928F929F9235
:1043C000AF92BF92CF92DF92EF92FF920F931F9323
:1043D000CF93DF93CDB7DEB7AD970FB6F894DEBFBE
:1043E0000FBECDBF8DA72091E80D2CA781E0809353
:1043F000E80D809127158D3409F4BEC2843511F47F
:104400000C945732873411F00C9469328091251541
:10441000909126158531910511F40C946B32B4F40A
:10442000843091053CF4823091050CF05CC097FF1C
:1044300031C09EC28A30910509F429C18B309105A3
:1044400009F42AC1049709F093C2E2C08D319105A5
:1044500009F451C16CF48B31910509F422C10CF0BF
:104460003AC14A9709F084C20E947B9D0C946B323A
:104470008A35910509F443C124F48A9709F4F9C1F6
:1044800077C28B35910509F43EC18C35910509F44D
:104490003FC16EC28091A106813011F00C946B3245
:1044A0000E9417DE80910D04882311F40C94A6322B
:1044B00085E40E948CF0882311F40C94A63288E5E0
:1044C0000E948CF081110C94A63289E50E948CF038
:1044D00081110C94A6328AE50E948CF081110C9413
:1044E000A6320C9474322091A106213011F00C9464
:1044F0006B3211E0029709F010E00E9417DE19827A
:104500001A821B821C821D821E821F82188682E5EF
:104510000E94D5F0882309F44BC00E9455F06B012E
:104520007C0120E030E0A9010F943040882309F499
:1045300055C08091511190915211A0915311B09199
:10454000541188A399A3AAA3BBA38091551190915C
:104550005611A0915711B09158118CA39DA3AEA3F1
:10456000BFA38090D60D9090D70DA090D80DB0909D
:10457000D90D4090DA0D5090DB0D6090DC0D7090FD
:10458000DD0DA501940168A179A18AA19BA10F94D9
:10459000304081110C94D132A30192016CA17DA114
:1045A0008EA19FA10F9430408823C1F00C94D1328A
:1045B00089E40E94D5F0882331F00E9455F0698388
:1045C0007A838B839C838AE40E94D5F0882331F020
:1045D0000E9455F06D837E838F83988720E030E0C2
:1045E000A90169817A818B819C810F94304081116E
:1045F0000C94853320E030E0A9016D817E818F81AC
:1046000098850F94304081110C9485330C94983325
:1046100080E50E94D5F0882329F00F94EB246B01EC
:104620007C0103C0C12CD12C760183E50E94D5F01A
:10463000882361F00E9455F020E030E04AE754E41E
:104640000F9496400F94B9486B017C010E94CAEC0C
:104650008091E20C811105C060E089E996E00E943A
:1046600068D60E9495FAC60ED71EE81EF91E0E9453
:1046700095FADC01CB018C199D09AE09BF09B7FD84
:1046800002C00C946B3280E00E946D39F0CF81E063
:104690000E94A4F10C946B3280E00E94A4F10C946F
:1046A0006B320F94930781110C946B328CE0E3E72B
:1046B000F2E0DE01119601900D928A95E1F760E03B
:1046C00070E080E50E94CCE5BE016F5F7F4F0E94E5
:1046D000BAD10C946B328091AE048770873011F0A0
:1046E0000C949F3360E08FE40E94F1F081110C94F0
:1046F0006B320C949F330F94DE250C946B32109226
:104700003C0E0C946B328FE080933C0E0C946B3219
:1047100080912415882349F1893009F0A6C00FE75C
:10472000A02E02E0B02E81E5E82E81E1F82ED12CFA
:1047300000E010E0D5018D915D010E94D5F0882345
:1047400069F00E9455F0F70160837183828393833F
:10475000133011F401E002C0DD24D3941F5FF4E0B4
:10476000EF0EF11C143031F775C0AFE72A2EA2E02E
:104770003A2EB2E5EB2EBEE0FB2E21E531E139A366
:1047800028A311E6C12E11E1D12E00E010E0D101E5
:104790008D911D010E94D5F0882309F44BC00E9421
:1047A00055F02B013C01133049F0F6012081318195
:1047B000428153810F9445472B013C01A8A1B9A127
:1047C0002D913D914D915C91C301B2010F944547EC
:1047D0004B015C012DEB37E346E855EB0F94A649FE
:1047E00087FD0AC02DEB37E346E855E3C501B40168
:1047F0000F9430401816F4F4133051F440925D11C8
:1048000050925E1160925F117092601101E012C0CF
:10481000A5019401F70160817181828193810F94D8
:104820004647D7016D937D938D939C931397812F6A
:104830000E9481851F5FB4E0EB0EF11CE8A1F9A195
:104840003496F9A3E8A3F4E0CF0ED11C143009F09C
:104850009ECF05C0DD2019F00E94A08A06C000236B
:1048600021F08DE591E10E94DBEC0E94A28A0C947C
:104870006B328091A106813011F00C946B3289E487
:104880000E94D5F0F82E882321F00E9451F0182FB5
:1048900001C010E08AE40E94D5F0082F882319F0A7
:1048A0000E9451F001C080E0FF2011F0133020F48D
:1048B000002341F0833030F083EA96E00E9446F412
:1048C0000C946B3290E1E1E5F1E1A6EDBDE00190E1
:1048D0000D929A95E1F7FF2091F024E01202F00189
:1048E0001124EB5DFD4E40815181628173814093C3
:1048F000D60D5093D70D6093D80D7093D90D00232A
:1049000091F034E08302F0011124E75EFD4E8081D6
:104910009181A281B3818093DA0D9093DB0DA093F6
:10492000DC0DB093DD0D40E050E0BA0186E40E945A
:1049300019566B017C0120E030E0A9010F94A649D3
:1049400018164CF420E030E040E752E4C701B6010D
:104950000F94404803C060E070E0CB0169837A8324
:104960008B839C83CE0101960E9412890C946B323A
:104970000F94D7050C946B328091251590912615D4
:104980008737910509F455C70CF0F3C08C349105B5
:1049900009F40EC40CF069C08931910509F4EAC22A
:1049A00054F58231910509F44FC65CF480319105CC
:1049B00009F43AC20CF04DC2029708F4FDC10C9400
:1049C00054328631910509F479C264F48431910539
:1049D00009F453C2459711F00C9454320E94F09799
:1049E0000C946B328731910509F472C2489709F42F
:1049F00086C20C9454328F31910509F48DC3BCF4F6
:104A00008C31910509F440C34CF48A31910509F4C5
:104A1000C5C24B9709F4D0C20C9454328D31910524
:104A200009F43AC34E9709F43EC30C9454328A32C7
:104A3000910509F491C364F48032910509F443C3EC
:104A4000819711F00C9454320E94005B0C946B32ED
:104A50008934910509F499C38B34910511F00C94B4
:104A600054320E9461EA0C946B328A36910509F443
:104A70009EC4ACF58335910509F4DFC5BCF48E34D2
:104A8000910509F49DC30CF497C38135910509F490
:104A9000C0C58235910511F00C94543280913C0EC2
:104AA0008F7D806180933C0E0C946B328C35910528
:104AB00009F4F0C554F48435910509F4C5C585356C
:104AC000910509F4C4C50C9454328836910509F453
:104AD00009C48936910509F456C40C9454328037C0
:104AE000910509F402C5F4F48D36910509F421C449
:104AF0007CF48B36910509F497C48C36910511F03E
:104B00000C9454321092E70D109223020C946B32E5
:104B10008E36910509F492C48F36910509F4A1C42B
:104B20000C9454328337910509F43EC68CF48137D6
:104B3000910509F4E7C48237910511F00C945432C1
:104B40000F94C60A89EA91E10F941B2E0C946B32E4
:104B50008537910509F42BC68637910511F00C9421
:104B600054320091B9031091BA0394E0F12C40E063
:104B700044C68E32A1E09A0711F40C94EF2F0CF08A
:104B800076C08D3C910509F49AC774F58B3991056F
:104B900009F419C584F48937910509F455C60CF454
:104BA0004BC68C38910509F4CFC48139910509F4BD
:104BB00052C60C945432893C910509F407C754F449
:104BC0008E3B910509F4DFC4883C910509F4B7C612
:104BD0000C9454328B3C910509F41EC78C3C910512
:104BE00009F439C70C9454328C3D910511F40C949E
:104BF0002C2EECF4803D910509F4D7C754F48E3C7B
:104C0000910509F46FC78F3C910509F48AC70C948C
:104C10005432813D910511F40C941F2E833D910572
:104C200011F00C9454320F9461230C946B32823245
:104C3000E1E09E0711F40C94F52E64F48D3D91058E
:104C400011F40C94532E823E910511F40C94A92E6C
:104C50000C9454328C3221E0920711F40C945B2FA7
:104C60008D32914011F40C94702F0C945432863F85
:104C7000A1E09A0711F40C94A9300CF048C08D39CA
:104C8000E1E09E0711F40C941932E4F4803921E03C
:104C9000920711F40C9433304CF48F32914011F0A0
:104CA0000C9454320E9430560C946B328A39B1E025
:104CB0009B0709F423C48C39914011F40C943630CD
:104CC0000C9454328C3AF1E09F0711F40C94493063
:104CD0007CF4843A31E0930711F40C944630853A21
:104CE000914011F00C9454320F94FB240C946B32CD
:104CF000843FB1E09B0711F40C94A630853F9140AE
:104D000011F00C9454320F946B1B0C946B328D3B4E
:104D1000F2E09F0711F40C944A310CF58C3032E02C
:104D2000930711F40C94C6306CF4873FB1E09B07F5
:104D300011F40C94AC30883F914011F40C94B530D0
:104D40000C9454328835F2E09F0711F40C94CE3065
:104D50008B35924011F40C94D1300C945432873E30
:104D600033E0930711F40C940B32CCF48E3BB2E099
:104D70009B0711F40C944D31803A934011F00C9440
:104D800054322091B9033091BA0390913C12926051
:104D900090933C12C9010E94FB990C946B32883E9F
:104DA000F3E09F0711F40C943032893E934011F4E4
:104DB0000C9433320C94543280E50E94D5F0882351
:104DC00029F00F94EB246B017C0103C0C12CD12C82
:104DD000760183E50E94D5F0882361F00E9455F0AA
:104DE00020E030E04AE754E40F9496400F94B9482D
:104DF0006B017C010E94CAEC8091B9039091BA03C7
:104E0000009721F061E00E94FCD605C060E08CEBC9
:104E100096E00E9468D640E0C701B6010E94503F6C
:104E20000F94E5050C946B326FE378E18091B90340
:104E30009091BA030F946E3F892B11F40C946B324E
:104E400040E060E070E081ED96E00E94BBF50C94DC
:104E50006B328091201584FF02C00C943F34809106
:104E6000221587FF02C00C943F3480912315837074
:104E700011F00C943F340C945B3486E097E00E9470
:104E800046F489E592E10E940DC58BE1E9E5F2E186
:104E9000DE01119601900D928A95E1F760E070E0D5
:104EA000CE0101960E942B9BCE0101960E9428F113
:104EB00087EF96E00E9446F40C946B320E94319783
:104EC00080913C12877F806280933C120C946B32FD
:104ED000E091B903F091BA038081882329F08032F0
:104EE00009F410823196F8CF60E08091B903909177
:104EF000BA030E94499A1092C1030C946B3283E565
:104F00000E94D5F0882321F00E941DF00E94D05B02
:104F100084E50E94D5F08823A9F00E941DF06B0162
:104F20007C010E948C8BC0927C0DD0927D0DE09212
:104F30007E0DF0927F0DCD28CE28CF2819F081E08C
:104F40008093380E0E948937882381F00E9442970F
:104F50000E9461EA81EB9EE00E94E796109228157C
:104F60001092291510922A1510922B150F94E50511
:104F70000C946B3280913C1282FF03C08B7F809334
:104F80003C1280912E04882319F081E00F94D804FC
:104F90000E94A78B0F94E5050C946B3280913C1214
:104FA00083FD02C00C946B3283E50E94D5F0811121
:104FB0000C9469340C946B3283E40E948CF0882347
:104FC000C1F181E297E00E9446F48091A01388230A
:104FD00039F1BE016F5F7F4F8DE993E10E9455C2A9
:104FE0008E010F5F1F4FD8018D918D01882319F01D
:104FF0000E944138F8CFCE0101960E94CD99809150
:10500000F60D882389F080E20E94413806EF1DE00A
:10501000F80181918F01882339F00E944138F8CF3F
:1050200087E197E00E9446F48AE00E9441380C94A0
:105030006B3280913C1282FF21C080E397E00E9496
:1050400046F4609138127091391280913A12909121
:105050003B124AE00E9448388FE20E94413860913A
:1050600034127091351280913612909137124AE0C5
:105070000E9448380E9446390C946B3282E497E0D3
:105080000E9446F40C946B328091B9039091BA035C
:105090000E94FB990C946B3280913C128E7F80931E
:1050A0003C120C946B3280913C1283FD02C00C9434
:1050B0006B320F94C0058091B9039091BA030E949E
:1050C00059990C946B3280913C1282FD0E94CAEC7B
:1050D00080913C1283FD02C00C946B3260E080E54D
:1050E0000E94F1F0182F682F8091B9039091BA03B4
:1050F0000E94499A83E50E94D5F0882321F00E94FE
:105100001DF00E94D05B0E94429711110C946B32EB
:105110000E9461EA0C946B320E94588B6C8F7D8FD9
:105120008E8F9F8FBE016F5F7F4FCE014C960E9486
:10513000215A60E0CE0101960E94FCD60E944EF5F5
:10514000BE016F5F7F4F83E597E00E9437F58AE0ED
:105150000E9441380C946B326DE070E080E50E9453
:10516000E2F08C0197FF02C00C946B32E82E60E0F5
:1051700089E40E94F1F081110C946E34802F0F9419
:105180009630811103C60C946E3480E50E948CF039
:10519000882311F40C946B320E942DF090E0853638
:1051A000910510F084E690E08093C1030C946B327B
:1051B0000E94A78B0C946B320E94BDEA0C946B3258
:1051C00060E070E083E50E94E2F08E34910531F4F6
:1051D0000E942EEB0F94E5050C946B3288EC97E05F
:1051E0000E9446F46091C7047091C8048FEB97E069
:1051F0000E940CF56091C9047091CA0482EB97E09B
:105200000E940CF56091C7047091C8048091C90494
:105210009091CA04681B790B8091380E815021E06F
:1052200030E0823010F020E030E0621B730B87EA40
:1052300097E00E940CF58AE00E94413888EC97E0E4
:105240000E9446F48091CB049091CC04A091CD04AF
:10525000B091CE048C8F9D8FAE8FBF8FBE016F5FDC
:105260007F4FCE014C960E94215ABE016F5F7F4F47
:105270008AE997E00E9437F58091CF049091D0049D
:10528000A091D104B091D2048C8F9D8FAE8FBF8F2F
:10529000BE016F5F7F4FCE014C960E94215ABE0126
:1052A0006F5F7F4F8AE897E00E9437F520E030E09B
:1052B0004AE754E46091D3047091D4048091D504FA
:1052C0009091D6040F944048AB01BC0182E797E06F
:1052D0000E9419F58DE60E9441388AE00E9441380B
:1052E0000C946B328091740C83FF02C00C946B326F
:1052F0000E9427DF87FF02C00C946B3289E40E9472
:10530000D5F0882311F40C94A5340E942DF090E080
:105310001816190614F481E090E026E0289FF001A9
:10532000299FF00D1124E15DFB4F808191810C9448
:10533000AF348091740C83FF02C00C946B320E94D6
:1053400027DFF82E87FF02C00C946B3289E40E949D
:10535000D5F0082F882311F40C94B8340E942DF056
:1053600090E01816190614F481E090E026E0289FDA
:10537000F001299FF00D1124E15DFB4F80819181A7
:1053800010E00C94C8340E9427DF182F87FD0AC054
:1053900084E491E40E9446F4812F0E9456C68AE07C
:1053A0000E9441382CA52093E80D0C948D3680E5A1
:1053B0000F94EA0781110C946B3281E40E948CF007
:1053C000882329F060917007062F10E002C00FEFCC
:1053D00010E089E40E94D5F0882399F00E942DF016
:1053E00090E01816190614F481E090E026E0289F5A
:1053F000F001299FF00D1124E15DFB4F048115811F
:1054000008C083E50E94D5F0882319F00E941DF0A2
:105410008B01B8010F3F110519F010F06FEF70E02C
:10542000609370070C946B3280E50F94EA0781114A
:105430000C946B32109270070C946B328EE40E94C5
:10544000D5F0882311F40C946B320E941DF0609308
:10545000B0157093B1158093B2159093B3150C9459
:105460006B3283E50E948CF0882329F083E50F944A
:10547000EA078093740C0E944EF589ED97E00E9434
:1054800046F48091740C882369F1F2E6EF2EF9E07E
:10549000FF2E00E010E020E08091740C90E0A0E08E
:1054A000B0E0002E04C0B695A795979587950A940D
:1054B000D2F780FF0EC0DD24D394D20E222319F040
:1054C0008CE20E944138F701859194910E9446F444
:1054D0002D2D0F5F1F4F32E0E30EF11C053011053B
:1054E000D9F6A2CD85ED97E09DCD41E060E070E07A
:1054F00080EE97E00E94BBF50C946B320E94D3368D
:105500000C946B3283E50E94D5F0882371F00E94E1
:105510002DF0282F30E02D3331051CF4809300024C
:10552000DAC78CE380930002D6C70E944EF5409103
:10553000000250E060E070E08EEE97E00E94FBF425
:105540008AE00E944138C7C78091740C83FDC3C7AD
:1055500089E40E94D5F0882311F40C9412350E943E
:105560002DF090E01816190614F481E090E026E082
:10557000289FF001299FF00D1124E15DFB4F8281EE
:1055800093810C941D358091740C83FDA4C789E42C
:105590000E94D5F0882311F40C9424350E942DF03C
:1055A00090E01816190614F481E090E026E0289F98
:1055B000F001299FF00D1124E15DFB4F8281938161
:1055C00010E00C94353583E50E94D5F0882309F46A
:1055D00082C70E942DF0182F90E0CD970CF01CE3AD
:1055E0001093F1020E9495FA6B017C01212F30E0AB
:1055F000A8EEB3E00F94DA46C60ED71EE81EF91ED9
:10560000C092ED02D092EE02E092EF02F092F00230
:1056100062C70E94BFCB0E94BDEA0E9444EE0E9476
:10562000AD3768EE73E080E090E00E9422F460E025
:1056300082E198E00E9468D64EC780913C0E8F7E32
:10564000806280933C0E47C70F94502444C783E583
:105650000E948CF0882309F43EC70E9495FA60935B
:10566000D80C7093D90C8093DA0C9093DB0C0E94C9
:1056700055F020E030E04AE754E40F9496400F9450
:10568000B9486093F2027093F3028093F40290930E
:10569000F50221C70E9427DF87FD1DC790912015C5
:1056A00094FD04C09091221597FF0AC07FE7C72E92
:1056B00072E0D72EE5E7EE2EECE0FE2E10E009C0FA
:1056C00090912315937091F7682F81E00F94B02487
:1056D00002C7D6018D916D010E94D5F0882309F48F
:1056E00059C0133009F04FC00E9455F04B015C01C6
:1056F00020E030E040EA51E40F94304087FF3AC0A8
:10570000A50194016091950C7091960C8091970C75
:105710009091980C0F9440482B013C019B01AC01E7
:105720006091A50C7091A60C8091A70C9091A80C8B
:105730000F9496406093A50C7093A60C8093A70CD1
:105740009093A80C6091640770916507809166073B
:10575000909167070F943540A30192010F949640F2
:105760000F94B94860936407709365078093660748
:10577000909367078092950C9092960CA092970C4C
:10578000B092980C07C00E9455F0F701648B758B9E
:10579000868B978B1F5FF4E0EF0EF11C143009F03D
:1057A00098CF0E94DFEB97C60F941A2294C680917F
:1057B000B9039091BA03009709F4D8CBDC012C917E
:1057C000222309F4D3CB60E00E94FCD684C6F80102
:1057D0008081282F2B7F213499F08035E9F4818155
:1057E00080538A30C8F498012E5F3F4F89012F5FA4
:1057F0003F4FF80180818032C9F3915041F70CC0CE
:105800002181213349F4813421F0853461F741E06D
:10581000EACFFF24F394E7CF41110E944EF5FF2019
:1058200021F082E298E00E9446F4C8010E944C39BF
:1058300052C60E94298B4FC681E08093D804809382
:10584000D7040E944D8B47C61092D8041092D704FB
:105850000E944D8B40C660E070E083E50E94E2F05C
:10586000823038F00E944AF586E298E00E9446F4C1
:1058700032C68C01112788E40E94D5F08823E1F01C
:105880000E9451F08A3A910544F00E9451F085300F
:10589000914034F40E9451F005C08AEA90E002C0C1
:1058A00084E091E026E0209FF001219FF00D11247B
:1058B000E15DFB4F9183808382E40E94D5F08823D1
:1058C000D9F00E9451F0059744F00E9451F08437BE
:1058D000910534F40E9451F005C085E090E002C0CB
:1058E00083E790E026E0209FF001219FF00D112436
:1058F000E15DFB4F9383828386E40E94D5F0882389
:1059000009F4E9C50E9451F097FD09C00E9451F0C9
:105910008F3F910509F034F40E9451F005C080E0FA
:1059200090E002C08FEF90E026E0209FF001219FE1
:10593000F00D1124E15DFB4F95838483CCC50E945B
:1059400027DF182F87FDC7C50091510E84E40E9400
:10595000D5F0882311F40C945E350E9455F06B014C
:105960007C0120E030E0A9010F943040882341F110
:1059700024E01202F0011124E35BF14FC082D182D6
:10598000E282F38220E030E0A90160914D0E709137
:105990004E0E80914F0E9091500E0F943040811119
:1059A0000CC080E090E0A0EEBFE380934D0E90939A
:1059B0004E0EA0934F0EB093500E01E00C945E3546
:1059C00080E08093510E0E94E38085C50E9427DF0E
:1059D00087FD81C55FE7E52E52E0F52E05E71CE067
:1059E00065E8C62E6CE0D62ED7018D917D010E9410
:1059F0008CF0882359F00E9455F00F94B948F801B3
:105A000060837183828393830E9498EB0C5F1F4FA6
:105A1000C016D10649F75FC50E9427DF87FD5BC529
:105A20004FE7E42E42E0F42E05E71CE0D7018D910C
:105A30007D010E948CF0882339F00E9455F0F80116
:105A400064A375A386A397A30C5F1F4FFCE00538E2
:105A50001F0761F740C58091211587FF02C00C9494
:105A60006435809122158E7011F00C94643540914C
:105A7000A90C5091AA0C6091AB0C7091AC0C88E40D
:105A800098E00E9419F54091AD0C5091AE0C6091D8
:105A9000AF0C7091B00C89EE9CE10E9419F5409119
:105AA000B10C5091B20C6091B30C7091B40C8DEEAE
:105AB0009EE10E9419F58AE00E9441380CC5809150
:105AC000201581FF02C00C94AA358091211581FF19
:105AD00002C00C94AA35809122158C7011F00C94A0
:105AE000AA35F9C43EE5E32E3EE0F32E10E088E54A
:105AF000810F0E948CF0882359F00E9455F0D70145
:105B00006D937D938D939C931397812F0E94818534
:105B10001F5FB4E0EB0EF11C133049F70E94A28A1C
:105B2000DAC483E50E948CF0882351F00E9455F07E
:105B300060930E0470930F048093100490931104EB
:105B400086E40E948CF0882381F00E9455F020E0CA
:105B500030E040E752E40F944048609312047093A1
:105B6000130480931404909315048AE50E948CF02A
:105B7000882351F00E9455F0609316047093170427
:105B8000809318049093190487E50E948CF0882371
:105B900009F4A1C40E9455F0609322047093230479
:105BA000809324049093250496C483E50E948CF08E
:105BB000882351F00E9455F060931A0470931B04DF
:105BC00080931C0490931D0486E40E948CF088232B
:105BD00081F00E9455F020E030E040E752E40F945D
:105BE000404860931E0470931F0480932004909398
:105BF000210482E50E948CF0882381F00E9455F0F8
:105C000020E030E040E752E40F94404860932A04DB
:105C100070932B0480932C0490932D0487E50E94AD
:105C20008CF0882309F457C40E9455F06093260431
:105C30007093270480932804909329044CC483E52F
:105C40000E948CF0882309F446C40E9441F080939E
:105C50000D040E9414DE3FC483E50E94D5F0882322
:105C600031F00E9451F090931102809310028091C4
:105C7000201590912115A0912215B0912315892B03
:105C80008A2B8B2B09F027C46091100270911102AE
:105C900087E798E00E942AF585E20E9441388AE071
:105CA0000E94413818C40E9427DFF82E87FD13C4D4
:105CB00083E50E94D5F00F2D0F2C000C110B8823CB
:105CC00069F10E9451F0F801EE0FFF1FEA5EFD4FEF
:105CD00091838083000F111F000F111FF801EC5DED
:105CE000FD4F7F01BC01990F880B990B0F94374032
:105CF0002AE037ED43E25CE30F949640F801E95463
:105D0000FB4F20813181428153810F949640D7010E
:105D10006D937D938D939C931397DDC30E944EF5F5
:105D200085E40E94413880E38F0D0E944138000FC6
:105D3000111FF801EA5EFD4F608171818BE798E0E9
:105D40000E942AF585E20E9441388AE00E9441388B
:105D5000C2C380E50E948CF0882309F4BCC360E0D4
:105D600070E080E50E94E2F0F82E6FEF7FEF83E5B0
:105D70000E94E2F08C010196039708F0ACC3F7FC97
:105D8000AAC38F2D0F949630882339F00E944AF5CC
:105D900083E898E00E9446F49EC30E94CAEC60E04B
:105DA0008F2D0E9456F90F3FBFEF1B0731F00130D6
:105DB000110571F000E010E00DC08F2D0F945D39DA
:105DC00031E020E0892B09F030E0032F122F02C0D0
:105DD00001E010E08F2D0F945D398017910709F4D1
:105DE0007AC380E00E946D39F5CF8AE50E94D5F034
:105DF000811106C083E50E94D5F0882309F440C0D4
:105E00000E9455F020E030E040E050EC0F9430402C
:105E100087FDFFC60E9455F020E030E040E050E4EE
:105E20000F94A64918160CF4EEC60E9455F06B01AB
:105E30007C0184E00E94A185811122C02091910CF7
:105E40003091920C4091930C5091940CC701B60183
:105E50000F9496400F94B2482091A5063091A60663
:105E6000260F371F3093A6062093A5062091D50C48
:105E70003091D60C620F731F7093D60C6093D50CC3
:105E80008091221587FDCBC680912315837009F080
:105E9000C6C60E944EF540913B0450913C0460916F
:105EA0003D0470913E0482E998E00E9419F58AE071
:105EB0000E94413810C364E071E083E50E94CCE5A4
:105EC0008C0168EE73E080E50E94CCE58938E3E15F
:105ED0009E0710F088E893E1B8010E9431D6FBC21A
:105EE00085E40F94EA07811173C080E50E948CF06D
:105EF000882351F00E9455F060933A0F70933B0F46
:105F000080933C0F90933D0F89E40E948CF088238E
:105F100081F00E9455F02CEA35EC47E25EE30F94E5
:105F2000964060933E0F70933F0F8093400F909385
:105F3000410F84E40E948CF0882381F00E9455F088
:105F40002CEA35EC47E25EE30F9440486093420F41
:105F50007093430F8093440F9093450F0E944EF52A
:105F600040913A0F50913B0F60913C0F70913D0F63
:105F700087EA98E00E9419F52CEA35EC47E25EE3E7
:105F800060913E0F70913F0F8091400F9091410FB3
:105F90000F944048AB01BC0183EA98E00E9419F5D8
:105FA0002CEA35EC47E25EE36091420F7091430FBB
:105FB0008091440F9091450F0F949640AB01BC0126
:105FC0008FE998E00E9419F58AE00E94413883C267
:105FD0000E944AF58DEE95E30E9446F47CC283E56B
:105FE0000E948CF0182F882371F00E9455F00F94B6
:105FF000B248709329026093280221E0672B09F0D0
:1060000020E02093810780E50E948CF0882359F0DE
:106010002091280230912902232B11F00E9441F097
:106020008093810758C2111156C20E944EF584EC2C
:1060300098E00E9446F480918107882319F08EED44
:1060400096E302C08BEA98E00E9446F46091280231
:106050007091290283EB98E00E942AF58FEA98E07C
:106060000E9446F438C20E94CAEC35C280912215C3
:10607000867009F0DAC50E944EF587ED98E00E941F
:1060800046F480910A020E94EFF425C20F94A627DD
:1060900022C20F94930781111EC208E619E321E57D
:1060A00031E139A328A3CE0101961C017AEBC72E5A
:1060B00078E2D72E7C01F8016591759185919491D4
:1060C000A8A1B9A18D909D90AD90BD90B9A3A8A3B2
:1060D000A50194010F9445472B013C01F701608312
:1060E00071838283938320E030E040EA51EC0F9487
:1060F000A64987FD0AC020E030E040EA51E4C30130
:10610000B2010F94304018162CF4F6018491181641
:106110000CF4A2C5D7018D909D90AD90BD907D01EE
:1061200020E030E040EA51ECC501B4010F94A649EB
:1061300087FD9DC520E030E040EA51E4C501B4018F
:106140000F94304018160CF0A6C591C50E9418E6B1
:10615000C2C10F94E414BFC161E083E50E94F1F075
:1061600091E089270E94877DB6C181E08093011567
:106170000F940B1610920115882309F4ACC10E94EC
:106180004EF586E299E00E9446F4A5C180913C124A
:1061900082FFA1C1806480933C129DC10E9498E25D
:1061A0009AC10E9427DF082F87FD95C185E50E94CF
:1061B0008CF08823B1F1E02E002E000CFF080E9425
:1061C00055F04B015C0120E030E0A9010F94A64995
:1061D00087FF04C0B7FAB094B7F8B094C70153E092
:1061E000880F991F5A95E1F79C012B5F3B4F79016E
:1061F000D9018D929D92AD92BC92139720E030E030
:1062000048E453E4C501B4010F94A64918164CF4B0
:1062100080E090E0A8E4B3E4F70180839183A28357
:10622000B3838CE40E948CF0882309F454C1002EBF
:10623000000C110B0E9455F06B017C0120E030E056
:10624000A9010F94A64987FF04C0F7FAF094F7F864
:10625000F09420E030E048E453E4C701B6010F9425
:10626000A649980143E0220F331F4A95E1F7F9014F
:10627000EB5FFB4F18162CF0C482D582E682F782C2
:106280002AC180E090E0A8E4B3E484839583A683E8
:10629000B78321C10E946AE11EC10E9427DF182F27
:1062A00087FD19C18AE50E94D5F0882349F040E0B6
:1062B00050E0BA018AE50E9419564B015C0106C004
:1062C000812C912C90EAA92E91E4B92E412F64E003
:1062D00083E00E94996320E030E0A901C501B40188
:1062E0000F94A64918167CF580E090E0A0EAB0E48F
:1062F00089839A83AB83BC832091591130915A11C1
:1063000040915B1150915C11C501B4010F94464757
:106310006B017C0120E030E04BE953E40F94304006
:1063200087FD06C0C12CD12C8BE9E82E83E4F82E22
:10633000CC8EDD8EEE8EFF8EBE016F5F7F4FCE0165
:106340004C960E94518A85E50E948CF0882329F0A2
:106350000E9455F06B017C010AC028E01202F00196
:106360001124EB5FFB4FC080D180E280F38020E0FE
:1063700030E0A901C701B6010F94A64987FF04C008
:10638000F7FAF094F7F8F094F7FAF094F7F8F0943D
:10639000C982DA82EB82FC8264E0CE0101960F941E
:1063A000080620E030E0A901C501B4010F94A64918
:1063B00018165CF580E090E0A0EAB0E489839A8347
:1063C000AB83BC83A50194016091591170915A115E
:1063D00080915B1190915C110F9445476B017C019A
:1063E00020E030E0A9010F94A64918161CF0C12C3A
:1063F000D12C7601CC8EDD8EEE8EFF8EBE016F5FCE
:106400007F4FCE014C960E94518A40E060E089E0C7
:106410000E94996360C081E08093A1061092370DBD
:1064200060E083E50E94F1F0811155C00F94DE1BFE
:1064300052C083E50E948CF0882339F00E9441F01D
:1064400080932E040E940EF146C00E944EF581E317
:1064500099E00E9446F480912E040E94EFF43BC024
:106460000E9450DF38C00E94588B6D337105810542
:10647000910520F08EE599E00F94CB228AE599E012
:106480000F94CB2284EE8093C1030E9406F10E94F8
:10649000C29986E499E00E9446F487E49CE39093D5
:1064A000DD048093DC0417C00F94D70514C010914D
:1064B00025150E9495FA6093D80C7093D90C80939F
:1064C000DA0C9093DB0C112331F0812F0E9431C63E
:1064D00002C00F94D7053DA5311102C00F94CE1B09
:1064E0008CA58093E80D19C48090E20D9090E30D87
:1064F000A090E40DB090E50D20915D1130915E11FA
:1065000040915F1150916011C501B4010F9445474E
:106510006B017C0120E030E0A9010F94A64987FFC0
:10652000EFC32DEC3CEC4CEC5DEBC701B6010F94D6
:10653000304018165CF0C701B601905820E030E0FA
:1065400040E251E40F94304018161CF40E94558626
:10655000C2CF11E020E030E0A901C701B6010F94DD
:10656000A64918160CF010E08091EC028113EECFD2
:1065700080925D1190925E11A0925F11B0926011B5
:106580008DE591E10E94DBEC20E030E0A901C7013C
:10659000B6010F943040881F8827881F0E94A4F1FD
:1065A0009ACF20E030E0A901C701B6010F94304036
:1065B000881F8827881F181709F4A2C080E090E080
:1065C000A0E8BFEB88A799A7AAA7BBA728A139A1D4
:1065D0004AA15BA1C501B4010F94454720E030E01A
:1065E00040E05FE30F94964068A379A38AA39BA33E
:1065F0002CA13DA14EA15FA1C301B2010F9445475B
:1066000020E030E040E05FE30F9496402B013C0136
:1066100028A139A14AA15BA1CA01B9010F949640F2
:106620004B015C01A3019201C301B2010F9496409A
:106630009B01AC01C501B4010F9446470F94F44986
:106640004B015C019B01AC01C701B6010F944547AA
:106650006CA37DA38EA39FA3A5019401C701B601DE
:106660000F9446479B01AC016CA17DA18EA19FA117
:106670000F9496406B017C0120E030E0A9010F945B
:10668000A64987FD07C0C701B6010F94F4496B0105
:106690007C0103C0C12CD12C7601C301B2019058FA
:1066A000A50194010F94404828A539A54AA55BA5EA
:1066B0000F949640A70196010F94964028A139A106
:1066C0004AA15BA10F94464769837A838B839C839D
:1066D000A501940168A179A18AA19BA10F944048CA
:1066E00028A539A54AA55BA50F949640A701960158
:1066F0000F949640A30192010F9446470C94EA220E
:1067000080E090E0A0E8BFE35DCF412FBE016F5F66
:106710007F4F86ED9DE00F94271E0E9495FA6093AF
:10672000D80C7093D90C8093DA0C9093DB0CD3CEF9
:106730000E944AF583E896E00E9446F4CCCE0E947F
:10674000CAECE090410E80E00E94F1F20E9495FABE
:106750006093D80C7093D90C8093DA0C9093DB0C77
:106760008091560290915702A0915802B09159021F
:106770008093F8029093F902A093FA02B093FB027F
:1067800080911002909111029093F7028093F6028B
:1067900084E690E0909311028093100281E0809350
:1067A000D8040E944D8B8AE50E948CF0F82E88E573
:1067B0000E948CF0182F89E50E948CF018135DC0A0
:1067C000F11611F0012F04C001E011E0FF24F39451
:1067D00082E50E94D5F0882319F00E9455F004C08C
:1067E00060E070E080EA90E469837A838B839C8325
:1067F00020E030E0A9010F943040882341F01111CE
:1068000002C0002371F0CE0101960F94F10711230D
:1068100019F080E00F948331002319F081E00F9488
:106820008331FF2019F082E00F9483310E94A08A07
:106830008091D7048093D8048E2D0E94F1F280912C
:10684000F8029091F902A091FA02B091FB028093B4
:10685000560290935702A0935802B0935902809128
:10686000F6029091F702909311028093100283E058
:1068700080936E020E94A28A2ECE082FA9CF88E5AF
:106880000E948CF081115F9889E50E948CF0811143
:106890008A988AE50E948CF0882329F0809108016B
:1068A00081708093060185E40E948CF0882309F4AE
:1068B00012CE129810CE60E082EE96E00E9468D66A
:1068C0005F988A98809108018170809306011298E0
:1068D00002CE0E941DF00E94D05BFDCD8DE40E948F
:1068E000D5F08823A9F00E942DF0813039F020F0F6
:1068F000823049F462E003C060E001C061E0802FB3
:106900000E9456F905C080E697E00E9446F4E3CD68
:1069100083E50E94D5F0882309F4DDCD0E942DF097
:10692000F82EF9E0EF1203C080937007D4CD61E038
:10693000802F0E9456F96F2D802F0E9427F96F2D0E
:1069400070E0802F0E9492F9C6CD83E50E94D5F0B9
:10695000882359F00E9455F00F94B248CB010E9451
:1069600046C661E080E00F94CE370F941238B3CD65
:1069700083E50E94D5F0182F811105C082E50E94A1
:10698000D5F0882341F10E9455F00F94B248CB0115
:106990000E9446C661E081E00F94CE376091370FC8
:1069A0007091380F072E000C880B990B0F9437400D
:1069B0004B015C014090330F5090340F6090350FC5
:1069C0007090360FA30192010F94A64918163CF15E
:1069D000112361F001E00F941238002309F47BCDFC
:1069E00040E0612F8F2D0E945BC875CDA3019201FD
:1069F000C501B4010F94A64918168CF08AEF97E0F0
:106A00009F938F9380ED97E09F938F931F920E94A7
:106A1000E1D60F900F900F900F900F90DBCF89E091
:106A200098E0EECF83E50E94D5F0882309F453CD9A
:106A30000E9455F00F94B248CB010E940FF061E024
:106A400080E00F94CE3747CD83E50E94D5F0182F14
:106A5000811106C082E50E94D5F0882309F43BCD60
:106A60000E9455F00F94B248CB010E940FF060E0F5
:106A700081E00F94CE3760914A0E70914B0E072E35
:106A8000000C880B990B0F9437402091460E3091E3
:106A9000470E4091480E5091490E0F94A649181682
:106AA00054F085EF97E060E00E9468D660E0812FA7
:106AB0000E94C8C610CD84E098E0F5CF602F83E532
:106AC0000E94F1F00C94E12C83E50E94D5F088231C
:106AD00091F00E9455F06093A90C7093AA0C8093DA
:106AE000AB0C9093AC0C6093B10C7093B20C809390
:106AF000B30C9093B40C80E50E94D5F0882351F03C
:106B00000E9455F06093A90C7093AA0C8093AB0C73
:106B10009093AC0C82E50E94D5F0882351F00E943E
:106B200055F06093AD0C7093AE0C8093AF0C9093C6
:106B3000B00C84E50E94D5F0882309F4CCCC0E94E7
:106B400055F06093B10C7093B20C8093B30C90939A
:106B5000B40CC1CC82E40E948CF0882351F00F94D5
:106B6000EB246093850C7093860C8093870C909334
:106B7000880C83E50E948CF0882351F00E9455F028
:106B80006093B50C7093B60C8093B70C9093B80CCF
:106B900084E50E948CF0882351F00E9455F06093A8
:106BA000B90C7093BA0C8093BB0C9093BC0C8AE424
:106BB0000E948CF0882309F48ECC0E9455F06B0162
:106BC0007C012AE037ED43E25CE30F94A64987FDA0
:106BD00013C02AE939E949E95EE3C701B6010F9418
:106BE000304018164CF0C0925407D0925507E092EE
:106BF0005607F09257076FCC0E944AF588E598E057
:106C00000E9446F468CCC12CD12CE12CF0E4FF2E7C
:106C100010C9C12CD12CE12CE0ECFE2E0AC982E572
:106C20000E948CF0811135C956CC82E50E948CF00F
:106C3000082F83E50E948CF0182F011103C0112347
:106C400009F449CC0E94B1EE112309F444CC0E940E
:106C500041F080930A023FCCB7FAB094B7F8B094F1
:106C6000D7018D929D92AD92BC92139753CA0E9408
:106C70004AF588E099E00E9446F461E08AEF98E0E6
:106C80000E9468D60E94584D68E270E088EC90E05F
:106C90000E9431D620CC0C5F1F4FBFEFCB1ADB0A0E
:106CA000E9E304371E0709F006CA6EE5E62E6EE03A
:106CB000F62E10E0F10181919191A191B1911F0106
:106CC000F70181939193A193B1937F01812F0E944A
:106CD00081851F5F133071F70E94A28A60E088EE01
:106CE00098E00E9468D663E972E084E690E00E9432
:106CF00031D66AEB72E084E690E00E9431D6EBCBAD
:106D00002DEC3CEC4CEC5DE3C701B6010F94A649B9
:106D100087FD1CCCC701B60111CCAD960FB6F89417
:106D2000DEBF0FBECDBFDF91CF911F910F91FF90BE
:106D3000EF90DF90CF90BF90AF909F908F907F901B
:106D40006F905F904F903F902F9008958091A7068D
:106D500081110AC08091380E813041F080913C123F
:106D600082FB882780F9089580E0089581E00895E6
:106D7000129A08955F9A8091DA048E7F8093DA04E4
:106D80008A9A8091DA048D7F8093DA0480910801D9
:106D900080958170809306018091DA048B7F8093C7
:106DA000DA040C94B8368F929F92AF92BF92CF9232
:106DB000DF92EF92FF920F931F93CF93DF93CDB7A4
:106DC000DEB760970FB6F894DEBF0FBECDBF0E944E
:106DD000F484182F809194118093931180939211D1
:106DE0008093911184E6809390110E948AEB80ED4C
:106DF00093E09093730C8093720C11110E940185A3
:106E000081E08093B9150E94CAEC81E00E941AEEDD
:106E10006B017C0180E00E941AEE4B015C016093E3
:106E2000FF02709300038093010390930203C092CA
:106E30000303D0920403E0920503F092060382E07C
:106E40000E941AEE6093070370930803809309036E
:106E500090930A038E010F5F1F4F20E1F8011192FA
:106E60002A95E9F789829A82AB82BC82CD82DE8242
:106E7000EF82F88669877A878B879C8783E00E94F8
:106E80001AEE6B017C0120913F0730914007409141
:106E900041075091420769857A858B859C850F94BF
:106EA000454769877A878B879C87A7019601609100
:106EB0003B0770913C0780913D0790913E070F94EE
:106EC00046476D877E878F87988B8091410E8823F8
:106ED00019F0C8010E945DEB80E1F801A1E5B1E184
:106EE00001900D928A95E1F70E94A08A60960FB6F4
:106EF000F894DEBF0FBECDBFDF91CF911F910F91F0
:106F0000FF90EF90DF90CF90BF90AF909F908F90C9
:106F1000089590913C1293FB882780F993FF06C057
:106F200081E09091A013911101C080E008958091BB
:106F3000A706811110C08091380E823061F00E9446
:106F40008937882349F080913C1282FB882780F999
:106F500091E08927089581E00895109270070895BF
:106F60008F929F92AF92BF92CF92DF92EF92FF9259
:106F70000F93CF93DF931F92CDB7DEB75C016B0108
:106F80007A014901F501808191810F9460468983DE
:106F9000002311F0F6018083BE016F5F7F4FC401B3
:106FA0000F94AE0AF50180819181019691838083CF
:106FB000FFEFCF1ADF0A81E0E81AF10819F780E045
:106FC0000F90DF91CF910F91FF90EF90DF90CF90D6
:106FD000BF90AF909F908F9008957F928F929F92D5
:106FE000AF92BF92CF92DF92EF92FF920F931F93D7
:106FF000CF93DF931F92CDB7DEB77C0159018B0190
:107000006B01C40ED51E0C151D0559F1F7018080CA
:107010009180F80171908F017982C4010F946046CC
:10702000781691F0672DC4010F946846C4010F943F
:1070300060469981891741F00E944EF58CE699E0EF
:107040000E9446F481E00EC0BE016F5F7F4FC50114
:107050000F94AE0AF701808191810196918380831C
:10706000D2CF80E00F90DF91CF911F910F91FF90D1
:10707000EF90DF90CF90BF90AF909F908F907F90D8
:1070800008959091C00095FFFCCF8093C6000895AD
:107090008F929F92AF92BF92EF92FF920F931F93A6
:1070A000CF93DF93CDB7DEB7A0970FB6F894DEBFCE
:1070B0000FBECDBF611571058105910591F100E00D
:1070C000842E912CA12CB12C102FEE24E394F12CC2
:1070D000EC0EFD1EE00EF11C07FDFA94A5019401D3
:1070E0000F948646F7016083B901CA010F5F6115ED
:1070F00071058105910541F71F3F31F1E1E0F0E0B5
:10710000EC0FFD1FE10FF11D17FDFA9580818A300C
:1071100010F097E301C090E3890F0E9441381150AD
:10712000EBCF80E3A0960FB6F894DEBF0FBECDBFC5
:10713000DF91CF911F910F91FF90EF90BF90AF9093
:107140009F908F900C944138A0960FB6F894DEBFB4
:107150000FBECDBFDF91CF911F910F91FF90EF90A8
:10716000BF90AF909F908F900895CF92DF92EF9253
:10717000FF926B017C0197FF0BC08DE20E944138AA
:10718000F094E094D094C094C11CD11CE11CF11C7B
:107190004AE0C701B601FF90EF90DF90CF900C94CA
:1071A00048388F929F92AF92BF92CF92DF92EF9228
:1071B000FF92CF936B017C01B42E20E030E0A90157
:1071C0000F94304087FF07C08DE20E944138F7FAE4
:1071D000F094F7F8F094C0E060E070E080E09FE3A6
:1071E000CB1541F02DEC3CEC4CEC5DE30F9496405C
:1071F000CF5FF6CF9B01AC01C701B6010F944647A4
:107200006B017C010F94B9484B015C014AE00E947C
:107210004838CC2389F1C501B4010F9435409B0156
:10722000AC01C701B6010F9445476B017C018EE2AA
:107230000E94413820E030E040E251E4C701B6014D
:107240000F9496404B015C010F94B2486B01770F8D
:10725000EE08FF08C701B6010E94B538C701B601A4
:107260000F9437409B01AC01C501B4010F94454711
:107270006B017C01C150F1F6CF91FF90EF90DF9050
:10728000CF90BF90AF909F908F9008958DE00E9417
:1072900041388AE00C944138CF93DF93EC01899117
:1072A000882319F00E944138FACFDF91CF910C94D6
:1072B000463980912C1590912D15981759F0E92F8A
:1072C000F0E0E45DFA4E82819F5F9F7790932D15E9
:1072D00090E008958FEF9FEF08952F923F924F9285
:1072E0005F926F927F928F929F92AF92BF92CF9256
:1072F000DF92EF92FF920F931F93CF93DF93CDB75F
:10730000DEB72A970FB6F894DEBF0FBECDBFF82EBA
:1073100080919F06843008F0E0C180919F06843000
:1073200008F001C180912C1590912D15891B8F7744
:1073300009F4F9C00E94593997FDEFCF8A3019F04E
:107340008D3009F0E7C010920B038091AE1590913B
:10735000AF15FC01E45FFC4F1082892B39F01092CD
:10736000AF151092AE150CE013E003C00F94B72ACE
:10737000D4CFF8018191803211F48F01FACF8E348D
:1073800009F06AC00115110509F466C063E97AE0E5
:10739000C8010F94AE3F6C01892B41F06EE470E0A0
:1073A000C80104960F94A04A009709F4C8014AE066
:1073B00050E060E070E001960F94163D4B015C01D7
:1073C0008091B0159091B115A091B215B091B315FF
:1073D0000196A11DB11D88169906AA06BB0631F0BB
:1073E000CD2821F460E080E69AE049C06AE270E0CE
:1073F000C8010F94CF4A9C01009709F1982F901B68
:10740000E12C992339F09150F801E90FF11D8081A9
:10741000E826F7CF4AE050E060E070E0C90101964D
:107420000F94163D4E2C512C612C712C6415750552
:107430008605970541F060E081E49AE020C060E0B5
:1074400087E19AE01CC08092B0159092B115A0928D
:10745000B215B092B31516C080913C1280FF12C0D5
:1074600063E071E3C8010F94AE3F009729F0FC017F
:10747000838180538A3030F460E087E19AE00F9492
:10748000FA1B51C08091A1068130E1F067E470E001
:10749000C8010F94A04A0097A9F04AE050E060E0CC
:1074A00070E001960F94163D6430710581059105D9
:1074B00048F480EA99E00E9446F460E085E999E0AA
:1074C0000E9468D660E979E0C8010F946E3F892B6D
:1074D00021F4109223021092E70D6BE879E0C801C5
:1074E0000F946E3F892B39F441E060E070E080EE4C
:1074F00097E00E94BBF566E879E0C8010F946E3F03
:10750000892B11F40E94D33661E08CE093E00F9454
:10751000521C03CF2EEA35E14CE053E06BE073E000
:107520000F94931BFACE80913C1282FFD6C01A8230
:10753000198211E0409138125091391260913A123B
:1075400070913B128091341290913512A0913612B5
:10755000B0913712481759076A077B0708F410E003
:1075600000E680E1E82E99E6D92E80919F068430CE
:1075700008F0B3C01111B1C08091A5139091A6136A
:10758000A091A713B091A813809338129093391249
:10759000A0933A12B0933B1241E050E0BE016D5F00
:1075A0007F4F8DE993E10E9478BE019719F48B819A
:1075B00090E002C08FEF9FEF409038125090391248
:1075C00060903A1270903B12809034129090351275
:1075D000A0903612B090371211E0481459046A0492
:1075E0007B0408F410E08F3FFFEF9F0761F448141D
:1075F00059046A047B0438F40E944AF588E99AE049
:107600000E9446F4B2CF4091DB048A3079F08D308D
:1076100069F0481459046A047B0408F4A7C38981FB
:107620009A81009719F001969A83898310926C03CE
:1076300089819A81FC01049FE00DF11D1124E25E15
:10764000FA4F1082892BB1F01A82198280E00F94D0
:10765000291C8091381290913912A0913A12B09160
:107660003B128093281590932915A0932A15B09367
:107670002B1502C00F94B72A481459046A047B04DE
:1076800008F473CF0E94CAEC8DE993E10E9489C28D
:10769000809133128823E1F0815080933312D89E79
:1076A000C001112462E08455994F0E94499AE091EB
:1076B000331224E0E29FF0011124E855F94F608174
:1076C0007181828193810E94D05B0E9442974DCF4D
:1076D0000E943197E092A10648CF0E9495FA4B0193
:1076E0005C01F11050C38091A70681114CC310E0DA
:1076F0004091F2025091F3026091F4027091F50210
:107700004115510561057105A1F08091D80C90914A
:10771000D90CA091DA0CB091DB0C840F951FA61F39
:10772000B71FA5019401281B390B4A0B5B0B57FFB0
:1077300034C380916A0290916B02A0916C02B09167
:107740006D02892B8A2B8B2B09F44FC090919311DA
:1077500080919411981749F08092D80C9092D90C8E
:10776000A092DA0CB092DB0C40C011112BC30E9426
:1077700095FAC090D80CD090D90CE090DA0CF0902B
:10778000DB0C00916A0210916B0220916C02309127
:107790006D020C0D1D1D2E1D3F1DDC01CB01801B3C
:1077A000910BA20BB30BB7FD0DC380917703811131
:1077B0001CC081E0809377035F9A8091DA048E7F0A
:1077C0008093DA048A9A8091DA048D7F8093DA04B8
:1077D0008091080180958170809306018091DA0480
:1077E0008B7F8093DA040E94B83680917503909164
:1077F0007603909902C0019604C0181619062CF45D
:10780000019790937603809375038091750390910F
:1078100076038E3E92406CF00E944AF587EA9AE029
:107820000E9446F440E060E070E080E090E00E945A
:10783000BBF58091710390917203A0917303B09195
:10784000740395018401081B190B2A0B3B0B37FDB0
:1078500023C19091931180919411981751F0E09168
:1078600094111FE4E19FF0011124E853F84F608167
:1078700002C060917007662311F070E002C060E002
:1078800070E089E00E9492F98091D70C882309F476
:10789000F6C0E0903502F090360200913702109168
:1078A00038026091370F7091380F6E5F7F4F072E4F
:1078B000000C880B990B0F9437409701A8010F9487
:1078C000304087FDDCC030909411212C1C821D8239
:1078D0001E8280919311831509F467C0832D90E077
:1078E0002FE4289FF001299FF00D1124EE57F84F47
:1078F000458956896789708D452B462B472B89F41E
:10790000418D528D638D748D452B462B472B49F449
:10791000458D568D678D70A1452B462B472B09F45D
:107920003FC04FE4489F9001499F300D1124C90189
:107930008E57984F6C01FC01618172818381948123
:107940000F94F4492B013C01F60161A172A183A1BE
:1079500094A10F9435406F83788789879A87F601C1
:1079600065A176A187A190A50F9435409B01AC013C
:107970006F81788589859A850F944048A30192018B
:107980000F9496403B016C01222D3C814D815E811C
:107990000F94A649181624F4262C7C82CD82DE8210
:1079A00081E0830D8F70382E94CF20912D0230917D
:1079B0002E0240912F0250913002622D7C818D81E8
:1079C0009E810F9496409701A8010F9446473B0172
:1079D0006C0120903102309032024090330250907E
:1079E00034029B01AC01B701C8010F94A6491816D7
:1079F0006CF09101A201B301C6010F94A6491816BB
:107A00001CF47101820102C07301860140906D0374
:107A100050906E0360906F03709070039701A801FF
:107A2000C301B2010F94A6491816C4F420E037ED43
:107A300043EA5CE3B701C8010F9496406B017C01F7
:107A400028E431EE4AE75FE3C301B2010F949640A8
:107A5000A70196010F9446477B018C01C701D8010D
:107A600080936D0390936E03A0936F03B0937003A4
:107A7000B701C8010F94B248CB010E9446C6F4E694
:107A80008F0E911CA11CB11C809271039092720305
:107A9000A0927303B09274030F94B72A8091A10649
:107AA000882309F4E4C180910A028823C9F08091F7
:107AB000650D811115C00E94A636811104C0809108
:107AC000A706882369F08091940D87FD03C081503B
:107AD0008093940D959989C18091940D87FD75C10E
:107AE00080910901817011E01827009101020117AE
:107AF00009F44AC090913C12906290933C1210930A
:107B0000010281110DC064EF71E080E090E00E94FD
:107B100022F40E94F09780913C1283FD09C069C154
:107B20000E94319780913C12877F806280933C1243
:107B3000112309F461C1023028F460E088E59BE07C
:107B40000E9468D681E08093C00385ED9BE190930D
:107B5000260F8093250F1092280F1092270F83E095
:107B600080936E020E9495FADC01CB018C599F4FE5
:107B7000AF4FBF4F8093C4039093C503A093C60338
:107B8000B093C703111147C10E9495FA6B017C01A4
:107B900080910002882359F18091E80D882339F102
:107BA000409180035091810360918203709183031F
:107BB00097018601041B150B260B370B37FD2AC0D6
:107BC000833079F03CF4813094F00E944EF586E3E6
:107BD0009BE00BC0843059F40E944EF587E09BE097
:107BE00004C00E944EF58FE19BE00E9446F4209174
:107BF000000230E0A8EEB3E00F94DA46C60ED71EBE
:107C0000E81EF91EC0928003D0928103E0928203A5
:107C1000F09283038091380E813009F06EC00E948B
:107C200095FA6B017C0180917C0390917D03A0917A
:107C30007E03B0917F03A7019601281B390B4A0BE5
:107C40005B0B57FD3AC08090840D9090850DA090FD
:107C5000860DB090870D0E94588B6093840D7093B1
:107C6000850D8093860D9093870D0091CB04109124
:107C7000CC042091CD043091CE04081919092A09A9
:107C80003B09DC01CB01800F911FA21FB31F809322
:107C9000CB049093CC04A093CD04B093CE04D70131
:107CA000C601805F984DAF4FBF4F80937C03909388
:107CB0007D03A0937E03B0937F038091780390911E
:107CC0007903A0917A03B0917B0397018601081B89
:107CD000190B2A0B3B0B37FD10C010E8C10E1EEE2E
:107CE000D11EE11CF11CC0927803D0927903E0927E
:107CF0007A03F0927B030E949BEA0E9475D20E9455
:107D0000686C8091F102882309F4B1C00E9495FA51
:107D10000091ED021091EE022091EF023091F002FD
:107D2000DC01CB01801B910BA20BB30BB7FD9FC0F5
:107D30000E9495FA6B017C012091F10230E0A8EEDF
:107D4000B3E00F94DA46C60ED71EE81EF91EC092A5
:107D5000ED02D092EE02E092EF02F092F00280E0AB
:107D60000E9456C68AE00E94413881C0049FA0014B
:107D70001124425E5A4F9E012F5F3F4F6CE673E025
:107D80000F94931BF2CB8092D80C9092D90CA092B6
:107D9000DA0CB092DB0C11E0ABCC0E944AF560919A
:107DA0003A0E70913B0E8AEC9AE00E9437F58AE019
:107DB0000E94413840E060E070E080E090E00E9486
:107DC000BBF5B7CC1092770310CD81E08093650DA1
:107DD0008091A706811106C08FE69BE09093DD0499
:107DE0008093DC040E94CAEC7BCE85E08093940DE6
:107DF00073CE002309F4C8CE023058F460E088E462
:107E00009BE00E9468D680913A0D811102C00E94C9
:107E1000584D10E097CE023009F0B6CE80913C125A
:107E200083FFB2CE0E94D396882379F081E00E942E
:107E3000A19649EB50E06AE67EE08EE392E10E9473
:107E400078BE8EE392E10E9489C20E941EF18111E8
:107E500007C00E9406F10E94C2991092311294CE7E
:107E600087E69BE09093DD048093DC048DCE2A9618
:107E70000FB6F894DEBF0FBECDBFDF91CF911F913B
:107E80000F91FF90EF90DF90CF90BF90AF909F90B9
:107E90008F907F906F905F904F903F902F900895BC
:107EA000CF92DF92EF92FF92CF93DF936B017C0131
:107EB000D42FC091E80D83E08093E80D81E080939A
:107EC000E70DC114D104E104F10431F00E9495FAE8
:107ED000C60ED71EE81EF91E8091E70D882399F083
:107EE000C114D104E104F10421F48D2F0E946D39F5
:107EF000F3CF0E9495FADC01CB018C199D09AE09E4
:107F0000BF09B7FDF2CF1092E70DC093E80DDF91E6
:107F1000CF91FF90EF90DF90CF9008951F920F9236
:107F20000FB60F9211240F900FBE0F901F9018954F
:107F30001F920F920FB60F9211240BB60F922F9330
:107F40008F939F93EF93FF939091C60020912D15EF
:107F5000E0912C1581E08E0F8F77281729F0F0E043
:107F6000E45DFA4E9283E82FE0932C15FF91EF9198
:107F70009F918F912F910F900BBE0F900FBE0F907E
:107F80001F9018958EBD0DB407FEFDCF08958FEF9D
:107F90008EBD0DB407FEFDCF8EB50895909164009F
:107FA0009B7F90936400982F906A96959CBD80FD6E
:107FB00003C091E0863009F490E09DBD08950C94D3
:107FC00098EB0C9498EB0C9498EB0C9498EBCF9264
:107FD000DF92EF92FF920F931F93CF93DF9361E0B5
:107FE00081E00E943F4CD091AE0DC0E0D1110BC09A
:107FF0008091AD0D81112AC08091A80D1092A80D1D
:1080000081111EC023C0D13061F48091AD0D81304B
:1080100009F045C08091A80D1092A80D811128C0CB
:108020003EC0D23009F060C08091AD0D823009F0C1
:108030008FC08091A80D1092A80D811172C088C0C8
:108040000E94604D8091CF0D81117CC180916E02A4
:10805000882309F440C081E09091AD0D911180E03A
:1080600004E024E043EF56E36C2F0E94555333C0E5
:108070000E9462F7C12CD12CE12C10ECF12E09E703
:1080800014E420E030E040E85FE369E97CE086E169
:108090009CE00E94C0F68091CF0D811153C1809168
:1080A0006E028823C1F011E08091AD0D813009F09E
:1080B00010E06091990C70919A0C80919B0C9091BA
:1080C0009C0C0E94E04B00E09C0146E15CE06C2FC0
:1080D000812F0E945855CF5FDF5FC53009F086CFF2
:1080E00087E08093A90D2EC1D33061F48091AD0D4E
:1080F000833009F06DC08091A80D1092A80D8111F8
:1081000050C066C0D43009F03DC08091AD0D8430C0
:1081100009F09EC08091A80D1092A80D811181C018
:1081200097C00E9462F7C12CD12CE12C10ECF12EEB
:1081300009E714E420E030E040E85FE36DE97CE02B
:108140008EE09CE00E94C0F68091CF0D8111FAC0B4
:1081500080916E02882309F4BECF11E08091AD0DAD
:10816000823009F010E060919D0C70919E0C80911E
:108170009F0C9091A00C0E94E04B00E09C014EE00F
:108180005CE0A5CFD53009F03DC08091AD0D8530C4
:1081900009F08EC08091A80D1092A80D811172C0B7
:1081A00087C00E9462F7C12CD12CE12C10ECF12E7B
:1081B00009E714E420E030E040E85FE361EA7CE0B6
:1081C00086E09CE00E94C0F68091CF0D8111BAC07C
:1081D00080916E02882309F47ECF11E08091AD0D6D
:1081E000833009F010E06091A10C7091A20C809195
:1081F000A30C9091A40C0E94E04B00E09C0146E08F
:108200005CE065CFD63009F066CF8091AD0D863049
:1082100009F07EC08091A80D1092A80D811162C056
:1082200077C00E9462F7C12CD12CE12C10ECF12E0A
:1082300009E714E420E030E040E85FE365EA7CE031
:108240008EEF9BE00E94C0F68091CF0D81117AC025
:1082500080916E02882309F43ECF11E08091AD0D2C
:10826000843009F010E06091A50C7091A60C80910B
:10827000A70C9091A80C0E94E04B00E09C014EEFEF
:108280005BE025CF0E9462F7C12CD12CE12C10ECD1
:10829000F12E09E714E420E030E0A90165EB7CE071
:1082A00087EF9BE00E94C0F68091CF0D81114AC0FC
:1082B00080916E02882309F40ECF11E08091AD0DFC
:1082C000853009F010E06091B50C7091B60C80918A
:1082D000B70C9091B80C0E94E04B00E09C0147EF76
:1082E0005BE0F5CE0E9462F7C12CD12CE12C10ECA2
:1082F000F12E09E714E420E030E0A90169EB7CE00D
:1083000087EE9BE00E94C0F68091CF0D81111AC0CC
:1083100080916E02882309F4DECE11E08091AD0DCC
:10832000863009F010E06091B90C7091BA0C809120
:10833000BB0C9091BC0C0E94E04B00E09C0147EE0E
:108340005BE0C5CEDF91CF911F910F91FF90EF9031
:10835000DF90CF9008955F926F927F928F929F925D
:10836000AF92BF92CF92DF92EF92FF920F931F9343
:10837000CF93DF9300D01F92CDB7DEB761E081E0ED
:108380000E943F4C6090AE0D712C43E0542E611062
:108390000BC08091AD0D81112AC08091A80D109263
:1083A000A80D81111EC023C081E068120BC09091FE
:1083B000AD0D9130C1F58091A80D1092A80D8111DD
:1083C00027C031C082E068124AC08091AD0D823072
:1083D00009F079C08091A80D1092A80D811160C09C
:1083E00072C00E94604D8091CF0D81111AC18091A1
:1083F0006E02882361F181E09091AD0D911180E0D2
:1084000004E024E043EF56E3672D0E9455531FC05C
:108410008091D70C86258093D70C50926E02809164
:10842000CF0D8111FEC080916E02882381F081E022
:10843000913009F080E09091D70C91111FC026E097
:1084400037E301E047ED5BE0672D0E9458557394D8
:10845000639485E078129BCF7092A90DE2C083E00F
:1084600068120FC08091AD0D833009F059C0809122
:10847000A80D1092A80D811140C052C02AE037E328
:10848000E0CF84E06812E3CF8091AD0D843009F035
:1084900092C08091A80D1092A80D81115DC08BC073
:1084A000C12CD12CE12CF12C02E813E420E030E0C7
:1084B000A90165E372E080ED9BE00E94C0F6809127
:1084C000CF0D8111AEC080916E02882309F4BFCF19
:1084D00011E08091AD0D823009F010E0609135021D
:1084E0007091360280913702909138020E94E04BE1
:1084F00000E09C0140ED5BE02CC0C12CD12CE12CB4
:10850000F12C02E813E420E030E0A90161E372E01D
:1085100089EC9BE00E94C0F68091CF0D811181C053
:1085200080916E02882309F492CF11E08091AD0D05
:10853000833009F010E06091310270913202809135
:108540003302909134020E94E04B00E09C0149EC20
:108550005BE0672D812F79CF20E030E048EC52E4DA
:1085600060912D0270912E0280912F029091300225
:108570000F94964020E030E0A9010F9446470F94F5
:10858000B948812C912C80E5A82E81E0B82E6B0192
:1085900018EEE12E13E0F12E00E010E020E030E0D4
:1085A000A9016DE272E08FEB9BE00F943E0A80918F
:1085B000CF0D811136C080916E02882309F447CF18
:1085C00011E08091AD0D843009F010E0C0902D02D3
:1085D000D0902E02E0902F02F090300220E030E0A8
:1085E000A901C701B6010F94304087FD05C02DEBEE
:1085F00037E346E055E304C02DEB37E346E055EBA7
:10860000C701B6010F94464769837A838B839C83A5
:10861000CE0101960E94DDCF00E09C014FEB5BE0B4
:1086200098CF0F900F900F900F90DF91CF911F91E7
:108630000F91FF90EF90DF90CF90BF90AF909F9001
:108640008F907F906F905F900895CF93DF9300D0CD
:108650001F92CDB7DEB70F94B9480F9435406983A8
:108660007A838B839C83CE0101960E940FCD0F905D
:108670000F900F900F90DF91CF9108958F929F925E
:10868000AF92BF92CF92DF92EF92FF92CF936B01A6
:108690007C0120E030E0A9010F94304087FD05C047
:1086A0006DEB77E386E095E304C06DEB77E386E05E
:1086B00095EBA70196010F9446476B017C0120E0E2
:1086C00030E0A9010F94304087FF1BC0C701B601FD
:1086D000905820E030E040E251E40F94964020E0D2
:1086E00030E040E251E40F9496404B015C0120E001
:1086F00030E0A901C701B6010F94A6491816FCF095
:1087000019C020E030E040E251E4C701B6010F9407
:10871000964020E030E040E251E40F9496404B0157
:108720005C0120E030E0A901C701B6010F943040A0
:1087300087FD05C060E070E080EA90E404C060E07E
:1087400070E080EA90ECA50194010F94464720E088
:1087500030E040E251E40F9440480F94B2486B017E
:108760007C0180E280933B0D80E1C81687E2D80649
:10877000E104F10494F0C701B60120E137E240E0E2
:1087800050E00F94A846CA01B9012AE030E040E069
:1087900050E00F94A846605D01C060E260933C0D1C
:1087A00088EEC81683E0D806E104F10494F0C7010E
:1087B000B60128EE33E040E050E00F94A846CA012D
:1087C000B9012AE030E040E050E00F94A846605D37
:1087D00001C060E260933D0D84E6C816D104E10457
:1087E000F10494F0C701B60124E630E040E050E027
:1087F0000F94A846CA01B9012AE030E040E050E0F9
:108800000F94A846605D01C060E260933E0D8AE06F
:10881000882E912CA12CB12CC701B601A501940181
:108820000F94A846C62FCA01B901A50194010F945F
:10883000A846605D60933F0D8EE28093400DC05D61
:10884000C093410D8BE39DE0CF91FF90EF90DF90BF
:10885000CF90BF90AF909F908F900895CF92DF926E
:10886000EF92FF92CF93DF9300D01F92CDB7DEB788
:108870006B017C0120E030E0A9010F94304087FDBE
:1088800005C06DEB77E386E095E304C06DEB77E31D
:1088900086E095EBA70196010F94464769837A839A
:1088A0008B839C83CE0101960E940FCD0F900F9079
:1088B0000F900F90DF91CF91FF90EF90DF90CF90CE
:1088C00008954F925F926F927F928F929F92AF9294
:1088D000BF92CF92DF92EF92FF920F931F93CF93AD
:1088E000DF9300D000D0CDB7DEB7C090790CD09028
:1088F0007A0CE0907B0CF0907C0C80917D0C909138
:108900007E0CA0917F0CB091800C8C159D05AE055E
:10891000BF0510F4D701C601C090750CD090760C3D
:10892000E090770CF090780CBC01CD016C157D05C2
:108930008E059F0510F4C701B6010F9435402B0139
:108940003C0161E081E00E943F4C2091AE0D2E83FE
:108950001D828E8181110BC08091AD0D81112CC0C3
:108960008091A80D1092A80D811120C025C02E81E4
:10897000213061F48091AD0D813009F08DC080917E
:10898000A80D1092A80D811129C086C08E81823059
:1089900009F0ABC08091AD0D823009F01FC180910C
:1089A000A80D1092A80D8111BFC018C10E94604D82
:1089B0008091CF0D81118BC280916E02882309F4C2
:1089C00087C081E09091AD0D911180E004E024E03A
:1089D00043EF56E36D810E9455537AC00E9462F7BF
:1089E0002AE037ED43E25DE3C301B2010F94964004
:1089F00020E030E0A9010F9446474B015C0120E0E4
:108A000030E040E05FE40F94304087FD05C0812CEA
:108A1000912CA12C5FE4B52E2AE037ED43E25DE313
:108A20006091A90C7091AA0C8091AB0C9091AC0C48
:108A30000F94964020E030E0A9010F94464720E0D3
:108A400030E040E85FE30F9445470F94B9486983ED
:108A50007A838B839C83C501B4010F94B2487B0158
:108A60008C0121E0E21AF10801091109812C912CF5
:108A700040EFA42E41E0B42EC980DA8021E030E03E
:108A800040E050E069EA7CE08DEA9DE30F943E0A05
:108A90008091CF0D81111BC280916E028823C1F09D
:108AA00011E08091AD0D813009F010E06091A90CCA
:108AB0007091AA0C8091AB0C9091AC0C0E942E444A
:108AC00000E09C014DEA5DE36D81812F0E945855C5
:108AD0008D818F5F8D832E812F5F2E83853009F0EE
:108AE00038CF88E08093A90DF2C18E81833061F484
:108AF0008091AD0D833009F0F9C08091A80D1092DE
:108B0000A80D811195C0F2C02E81243009F080C0DB
:108B10008091AD0D843009F024C18091A80D109290
:108B2000A80D81110CC11DC10E9462F76091810CDA
:108B30007091820C8091830C9091840C0F9435403D
:108B400020E030E0A9010F9446474B015C0120E092
:108B500030E040E05FE40F94304087FD05C0812C99
:108B6000912CA12C3FE4B32E20E030E0A9016091CC
:108B7000AD0C7091AE0C8091AF0C9091B00C0F9435
:108B8000464720E030E048EC52E40F9445470F940C
:108B9000B94869837A838B839C83C501B4010F94A0
:108BA000B2487B018C0124E6E21AF108010911099F
:108BB000812C912C26EDA22E21E0B22EC980DA80E4
:108BC00024E630E040E050E06DEA7CE08AE49CE09E
:108BD0000F943E0A8091CF0D811179C180916E0270
:108BE000882309F475CF11E08091AD0D823009F032
:108BF00010E06091AD0C7091AE0C8091AF0C909133
:108C0000B00C0E942E4400E09C014AE45CE05CCF82
:108C10008E81853009F084C08091AD0D853009F0DA
:108C2000DEC08091A80D1092A80D8111C6C0D7C0DA
:108C30000E9462F72AE037ED43E25DE3C301B2012F
:108C40000F94964020E030E0A9010F9446474B0175
:108C50005C0120E030E040E05FE40F94304087FDAD
:108C600005C0812C912CA12C9FE4B92E2AE037ED70
:108C700043E25DE36091B10C7091B20C8091B30C52
:108C80009091B40C0F94964020E030E0A9010F942D
:108C9000464720E030E040E85FE30F9445470F94FB
:108CA000B94869837A838B839C83C501B4010F948F
:108CB000B2487B018C0121E0E21AF1080109110997
:108CC000812C912C80EFA82E81E0B82EC980DA800B
:108CD00021E030E040E050E061EB7CE08EE39CE09E
:108CE0000F943E0A8091CF0D8111F1C080916E02E8
:108CF000882309F4EDCE11E08091AD0D833009F0A9
:108D000010E06091B10C7091B20C8091B30C909115
:108D1000B40C0E942E4400E09C014EE35CE0D4CEF3
:108D20002E812630D1F58091AD0D863009F085C0B9
:108D30008091A80D1092A80D81116DC07EC00E9477
:108D400062F70FED1FE324E630E040E050E065E716
:108D50007CE086E39CE00F9451388091CF0D811127
:108D6000B6C080916E02882309F4B2CE11E08091E2
:108D7000AD0D843009F010E06091750C7091760CA7
:108D80008091770C9091780C0F9435400E94254388
:108D900000E09C0146E35CE097CE8E81873009F0CD
:108DA00097CE8091AD0D873009F075C08091A80DE8
:108DB0001092A80D81115DC06EC00E9462F705EE91
:108DC0001FE324E630E040E050E069E77CE08EE21B
:108DD0009CE00F9451388091CF0D811178C0809123
:108DE0006E02882309F474CE11E08091AD0D8530B8
:108DF00009F010E06091790C70917A0C80917B0CF5
:108E000090917C0C0F9435400E94254300E09C011A
:108E10004EE25CE059CE0E9462F703EE1FE32AE0C7
:108E200030E040E050E06DE77CE086E29CE00F94AB
:108E300051388091CF0D81114AC080916E028823F4
:108E400009F446CE11E08091AD0D863009F010E0B6
:108E500060917D0C70917E0C80917F0C9091800CC4
:108E60000F9435400E94254300E09C0146E25CE0FF
:108E70002BCE0E9462F701EE1FE324E630E040E0D3
:108E800050E061E87CE08EE19CE00F9451388091E5
:108E9000CF0D81111CC080916E02882309F418CE79
:108EA00011E08091AD0D873009F010E06091810CE8
:108EB0007091820C8091830C9091840C0F943540BA
:108EC0000E94254300E09C014EE15CE0FDCD26962A
:108ED0000FB6F894DEBF0FBECDBFDF91CF911F91CB
:108EE0000F91FF90EF90DF90CF90BF90AF909F9049
:108EF0008F907F906F905F904F900895CF92DF9208
:108F0000EF92FF92CF93DF9300D01F92CDB7DEB7E1
:108F10006B017C0120E030E0A9010F94304087FD17
:108F200005C06DEB77E386E095E304C06DEB77E376
:108F300086E095EBA70196010F94464769837A83F3
:108F40008B839C8360E2CE0101960E94BBCD0F9083
:108F50000F900F900F90DF91CF91FF90EF90DF90E7
:108F6000CF9008956F927F928F929F92AF92BF920F
:108F7000CF92DF92EF92FF920F931F93CF93DF93E5
:108F800061E081E00E943F4CC091AE0D712C53E036
:108F9000652EC1110BC08091AD0D81111BC0809158
:108FA000A80D1092A80D81110FC014C0C13011F589
:108FB0008091AD0D813009F0C2C08091A80D109252
:108FC000A80D8111AFC0BBC00E94604D8091CF0D34
:108FD000811128C180916E02882361F081E0909117
:108FE000AD0D911180E004E024E043EF56E3672DDE
:108FF0000E9455538091510E882371F0C23071F454
:109000008091AD0D823009F0EFC08091A80D1092D3
:10901000A80D8111AFC0E8C0D2E001C0D3E0DC13DD
:109020003AC08091AD0D8D131BC08091A80D109298
:10903000A80D8823A9F00E9462F7C12CD12CE12C45
:10904000F12C08E413E420E030E0A90165E074E0CD
:1090500085E99BE00E94C0F68091CF0D8111E2C0AE
:1090600080916E028823B9F011E08091AD0D8C13D0
:1090700010E06091050470910604809107049091BE
:1090800008040E94E04B00E09C0145E95BE0672D8D
:10909000812F0E94585581E08D0F8C133AC080912A
:1090A000AD0D8C131BC08091A80D1092A80D8823C4
:1090B000A9F00E9462F7C12CD12CE12CF12C08E41C
:1090C00013E420E030E0A90169E074E08CE89BE063
:1090D0000E94C0F68091CF0D8111A4C080916E02D4
:1090E0008823B9F011E08091AD0D8C1310E06091F0
:1090F000090470910A0480910B0490910C040E9461
:10910000E04B00E09C014CE85BE0672D812F0E9462
:1091100058557394CF5F85E078123BCFDE5FD093D4
:10912000A90D80C08091510E8C278093510E6092C2
:109130006E020E94E3808091CF0D811173C08091F7
:109140006E02882309F456CF81E09091AD0D9130E5
:1091500009F080E09091510E911103C026E037E3B1
:1091600002C02AE037E301E045EB5BE0672D0E9497
:10917000585540CF0E9462F720E030E04AE754E4BF
:1091800060914D0E70914E0E80914F0E9091500E49
:109190000F94964020E030E0A9010F94464720E06C
:1091A00030E84BEB54E40F9445470F94B94823EE55
:1091B000822E20E8922E32E1A32E31E0B32E6B01F5
:1091C00016EDE12E16E0F12E00E010E02CED35E07A
:1091D00040E050E06DE47EE081EA9BE00F943E0ABF
:1091E0008091CF0D81111EC080916E028823C1F045
:1091F000D1E08091AD0D823009F0D0E060914D0E4C
:1092000070914E0E80914F0E9091500E0E947E47AD
:1092100000E09C0141EA5BE0672D8D2F0E945855CC
:10922000D3E039CFDF91CF911F910F91FF90EF9055
:10923000DF90CF90BF90AF909F908F907F906F9076
:109240000895FC0184910895FC0180810895909116
:10925000410E81E089270C94F1F280916E028823FF
:1092600051F06091380D7091390D20E030E041E00F
:1092700081E00C9455540895BF92CF92DF92EF9203
:10928000FF920F931F93CF93DF936B0189014A30B5
:1092900009F49DC0453109F06EC0DB011296ED91D5
:1092A000FC911397F280C681D7818091020180954D
:1092B00082708093000188E28A950000E9F720E13E
:1092C000B22EBF0C38E2E32E88EF0E942B528E2D77
:1092D0008A950000E9F7BFE1BF1508F45EC08F2D45
:1092E000807780680E942B528F2D8295807F0E940C
:1092F0002B528E2D8A950000E9F780E80E942B52B0
:1093000080E00E942B528E2D8A950000E9F78AEFAB
:109310000E942B528E2D8A950000E9F78E01005F86
:109320001F4F8881807F0E942B5289918295807F78
:109330000E942B52C017D107A1F78E2D8A950000ED
:10934000E9F7F394BF10C0CF80910201827080933F
:109350000001F601C281D381CE010E94D28C81111D
:10936000D3C1DF91CF911F910F91FF90EF90DF90CC
:10937000CF90BF900895DB011296CD91DC911397A9
:10938000842F90E0FC017497E433F105F0F4882712
:10939000EE58FF4F8F4F0D942B4710EE1F0D1068A6
:1093A000812F807F0E942B52812F8295807F0E9487
:1093B0002B528E2D8A950000E9F780E80E942B52EF
:1093C00080E89FCF8981F901808381E0CACF8091B5
:1093D000010182608093010180910201827080937B
:1093E000000180910101816080930101809102015F
:1093F000817080930001099A119A809102018095F1
:1094000082708093000188E28A950000E9F788E77E
:1094100090E02EE93FE0CEE9DFE0F9013197F1F786
:109420000197C9F788EF0E942B5218E2812F8A9585
:109430000000E9F780E20E942B5280E00E942B524C
:10944000812F8A950000E9F780E00E942B5280E886
:109450000E942B52812F8A950000E9F780E00E943C
:109460002B5280E10E942B52812F8A950000E9F750
:10947000CE010197F1F7CE010197F1F7CE010197E7
:10948000F1F7CE010197F1F7CE010197F1F7CE0187
:109490000197F1F7CE010197F1F7CE010197F1F7AE
:1094A000CE010197F1F7CE010197F1F7CE010197B7
:1094B000F1F7CE010197F1F7CE010197F1F7CE0157
:1094C0000197F1F72197F1F780E20E942B5280E497
:1094D0000E942B52812F8A950000E9F780E20E94BA
:1094E0002B5280E60E942B521A950000E9F7D0E03B
:1094F000C8E218E28D2F807780680E942B528D2F52
:109500008295807F0E942B528C2F8A950000E9F76C
:1095100080E80E942B5280E00E942B528C2F8A956B
:109520000000E9F78AEF0E942B528C2F8A950000E9
:10953000E9F790E211988091020181708093000117
:10954000119A0000119880910201817080930001AE
:10955000119A00001198809102018170809300019E
:10956000119A00001198809102018170809300018E
:10957000119A00001198809102018170809300017E
:10958000119A00001198809102018170809300016E
:10959000119A00001198809102018170809300015E
:1095A000119A00001198809102018170809300014E
:1095B000119A00001198809102018170809300013E
:1095C000119A00001198809102018170809300012E
:1095D000119A00001198809102018170809300011E
:1095E000119A00001198809102018170809300010E
:1095F000119A0000119880910201817080930001FE
:10960000119A0000119880910201817080930001ED
:10961000119A0000119880910201817080930001DD
:10962000119A0000119880910201817080930001CD
:10963000119A00008C2F8A950000E9F7915009F0EB
:1096400079CF88EF0E942B52812F8A950000E9F78D
:10965000DF5FD03209F04ECF80E00E942B5280ECC9
:109660000E942B5288E28A950000E9F7809102015E
:1096700082708093000181E074CE4D8150E0440FF0
:10968000551F60E070E08E819F810F947B4ACE0170
:109690000E94E88C81E065CEF9018181938191304F
:1096A00009F46EC0933009F040C048EF480F91E0D4
:1096B0002B81241708F490E021E03A81831708F405
:1096C00020E031E0841708F030E0492F432B2423B9
:1096D00019F4932309F479CED8011296FC90EE2464
:1096E000EA94D12C44C0B901CE010E94EF8C81E0F4
:1096F00038CEF90110828A8181838D8181508283E5
:109700008B81838381E02DCE4D8150E0440F551F26
:1097100060E070E08E819F810F947B4A81E021CED2
:109720008D81D9018C9381E01CCE2B81281708F400
:109730004CCE2A81821708F448CEF2809130C9F1CC
:10974000D8F19230B9F4E12CDD24DA9410C0B801DC
:10975000CE010E94EF8CF8018181D8019C919D0D72
:109760009C938E0D11968C93FF0C09F42ECEF7FE70
:10977000F4CFEDCF933009F4B2CFE12CD12CF7CF59
:1097800048E0480F91E02B81281708F490E021E091
:109790003A81431708F420E031E0481708F030E040
:1097A000492F432B242319F4932309F40ECEF801F7
:1097B000F280EE24E39495CFE12CDD24D394D7CF2F
:1097C000CF92DF92EF92FF926B017C0120E030E0BC
:1097D000A9010F94304087FD05C06DEB77E386E06B
:1097E00095E304C06DEB77E386E095EBA701960166
:1097F0000F9446476B017C0120E030E0A9010F94F3
:10980000304087FD05C020E030E040E05FE304C069
:1098100020E030E040E05FEBC701B6010F9446471F
:109820000F94B248CB01FF90EF90DF90CF900C9453
:1098300028D10F93CF93DF93CDB7DEB700E22EE3AD
:1098400049855A8568858F810E945553DF91CF9154
:109850000F91089563E972E084E690E00E9431D6AA
:109860006AEB72E084E690E00C9431D681110C949E
:109870002A4C68EB71E084E190E00C9431D6282FFB
:109880001092B90D8091BF0D9091C00DA091C10DA6
:10989000B091C20DB7FF08C01092BF0D1092C00D5D
:1098A0001092C10D1092C20D8091C203882331F035
:1098B0008091BF0D8093AD0D1092CF0D8091A90DB9
:1098C0001816FCF4082E000C990B821B91092091AC
:1098D000AD0D022E000C330B2817390794F097FFBB
:1098E00002C080E090E08093AD0D092E000CAA0B21
:1098F000BB0B8093BF0D9093C00DA093C10DB0938F
:10990000C20D8091AD0D6623A9F09091AE0D89171F
:1099100014F48093AE0D2091AE0D022E000C330B8B
:109920002C5F3F4F482F082E000C550B241735078E
:109930001CF484508093AE0D089580919311909102
:109940009411891B8F7011F40C94A63681E0089550
:109950008F929F92AF92BF92CF92DF92EF92FF923F
:109960000F931F93CF93DF93EC01042F122F80915D
:10997000D5119091D6118C179D0709F48CC02091B8
:10998000C10327FD1092C1036B01E12CF12C20E6ED
:10999000C636D207A1F486589F46B9F50E9495FABB
:1099A000DC01CB018E519B4FAF4FBF4F8093B5036E
:1099B0009093B603A093B703B093B80326C02FE6E5
:1099C000C638D20709F043C08656904609F050C009
:1099D0000E9495FA8090B5039090B603A090B703CB
:1099E000B090B803DC01CB0188199909AA09BB0919
:1099F000B7FF3EC08091DA048770873031F40E944F
:109A00009D4C882311F0C0E5DDE8D093D611C093BA
:109A1000D511C092BF0DD092C00DE092C10DF09251
:109A2000C20D0093AE0D1093A90DC658DF4621F468
:109A300010923A0D1092B40382E080936E0281E09E
:109A40008093CF0D1092C3031092FE1424C0D093C4
:109A5000D611C093D511C092BF0DD092C00DE09227
:109A6000C10DF092C20D0093AE0D1093A90DE4CF7D
:109A700086E89FE69093D6118093D511C092BF0DD2
:109A8000D092C00DE092C10DF092C20D0093AE0DC8
:109A90001093A90DCDCFDF91CF911F910F91FF9022
:109AA000EF90DF90CF90BF90AF909F908F900895F0
:109AB00020E040E060E070E086E89FE60C94A84C6F
:109AC000E091B403EE2389F0E150E093B40388E021
:109AD000E89FF0011124EC57FC4F628173812781CC
:109AE0004681808191810C94A84C0C94584D0F9321
:109AF0001F93CF93DF93FC01EB018091BF0D9091F9
:109B0000C00DA091C10DB091C20DB7FF08C0109259
:109B1000BF0D1092C00D1092C10D1092C20D809118
:109B2000C30D9091C40DA091C50DB091C60D40918B
:109B3000BF0D5091C00D6091C10D7091C20D841781
:109B40009507A607B70744F48093BF0D9093C00D07
:109B5000A093C10DB093C20D80916E02882301F1D4
:109B60004091BF0D5091C00D6091C10D7091C20D1B
:109B70008091C70D9091C80DA091C90DB091CA0DEB
:109B80008A019B01080F191F2A1F3B1FC901B80139
:109B90001995BC018091CD0D9091CE0D0E94D354AA
:109BA0008091A80D811108C08091BC0D8823D1F14E
:109BB00080916E028823B1F18091CB0D9091CC0DF4
:109BC0000097B1F00091BF0D1091C00D2091C10D13
:109BD0003091C20D4091C70D5091C80D6091C90DD3
:109BE0007091CA0D400F511F621F731FFE0119951E
:109BF000E091BD0DF091BE0D309741F08091BC0D0C
:109C0000811103C08091A80D811119958091A80D33
:109C10001092A80D882331F0DF91CF911F910F9101
:109C20000C94604DDF91CF911F910F910895E091B9
:109C3000B403E63010F581E08E0F8093B4034091B9
:109C4000BF0D5091C00D6091C10D7091C20D9091EA
:109C5000AE0D8091A90D28E0E29FF0011124EC5790
:109C6000FC4F2091D5113091D6113183208342834E
:109C700053836483758396838783089510923A0D86
:109C80000C94604DAF92BF92CF92DF92EF92FF9211
:109C90000F931F93CF93DF93EC015B018A01FB01CC
:109CA000199587FD05C090E0A0E0B0E0219628C19D
:109CB000982F907E903CC9F48F7190E0A0E0B0E0C6
:109CC0006C017D0126E0CC0CDD1CEE1CFF1C2A95EE
:109CD000D1F7CE010196F50119958F73A701960171
:109CE000282BDA01C90122960BC1982F907F903E54
:109CF00029F58F70C82ED12CE12CF12C86E0CC0CEC
:109D0000DD1CEE1CFF1C8A95D1F7CE010196F501F2
:109D100019958F73C82A96E0CC0CDD1CEE1CFF1C35
:109D20009A95D1F7CE010296F50119958F73A70187
:109D30009601282BDA01C9012396E2C0982F987F5B
:109D4000903F91F58770C82ED12CE12CF12CF6E0D4
:109D5000CC0CDD1CEE1CFF1CFA95D1F7CE01019650
:109D6000F50119958F73C82AA6E0CC0CDD1CEE1CFA
:109D7000FF1CAA95D1F7CE010296F50119958F73B4
:109D8000C82AB6E0CC0CDD1CEE1CFF1CBA95D1F73E
:109D9000CE010396F50119958F73A7019601282B23
:109DA000DA01C9012496ACC0982F9C7F983F09F036
:109DB0003FC08370C82ED12CE12CF12C56E0CC0C86
:109DC000DD1CEE1CFF1C5A95D1F7CE010196F50162
:109DD00019958F73C82A66E0CC0CDD1CEE1CFF1CA5
:109DE0006A95D1F7CE010296F50119958F73C82AAD
:109DF00076E0CC0CDD1CEE1CFF1C7A95D1F7CE0171
:109E00000396F50119958F73C82AE6E0CC0CDD1C8A
:109E1000EE1CFF1CEA95D1F7CE010496F5011995C9
:109E20008F73A7019601282BDA01C901259668C016
:109E3000982F9E7F9C3F09F04CC08170C82ED12C7A
:109E4000E12CF12C86E0CC0CDD1CEE1CFF1C8A956D
:109E5000D1F7CE010196F50119958F73C82A96E0C6
:109E6000CC0CDD1CEE1CFF1C9A95D1F7CE0102969E
:109E7000F50119958F73C82A26E0CC0CDD1CEE1C69
:109E8000FF1C2A95D1F7CE010396F50119958F7322
:109E9000C82A36E0CC0CDD1CEE1CFF1C3A95D1F72D
:109EA000CE010496F50119958F73C82A46E0CC0CB3
:109EB000DD1CEE1CFF1C4A95D1F7CE010596F5017D
:109EC00019958F73A7019601282BDA01C9012696EF
:109ED00017C0982F907C903841F4807C803869F4CA
:109EE0002196CE01F5011995F8CF8E7F8D3F28F090
:109EF0002196CE01F5011995F8CF80E090E0DC01C4
:109F00000115110529F0F80180839183A283B383A1
:109F1000CE01DF91CF911F910F91FF90EF90DF90D5
:109F2000CF90BF90AF9008956F927F928F929F9243
:109F3000AF92BF92CF92DF92EF92FF920F931F9357
:109F4000CF93DF9300D01F92CDB7DEB7862E6A0184
:109F5000122F2EEF621305C033E5A32E3CE0B32E83
:109F600004C02BEFA22E22E3B22E082F992E86E0FA
:109F7000E82EF12C9AE0792E11160CF08DC0AE016E
:109F80004F5F5F4F61E279E4802F992D0E94424E2E
:109F9000082F992E69817A818B819C8161157105C9
:109FA0008105910509F478C06D337105810591052E
:109FB00009F45BC06E3771058105910509F455C040
:109FC0006A32710581059105C1F064327105810520
:109FD000910579F4C114D10461F086E01802B00152
:109FE0001124C6010E949553B7010F941747161B01
:109FF000C3CF0E94E4521150BFCF87FC38C065E444
:10A0000070E080E090E00E94E452115009F443C0F7
:10A0100061E089819A81AB81BC81CD97A105B105B1
:10A0200009F460E0862F880D8A3094F0672D0F9434
:10A03000F546692E682F880F770B605D7F4F072EDE
:10A04000000C880B990B0E94E452115021F1862DCF
:10A05000682F880F770B605D7F4F072E000C880BF1
:10A06000990B0E94E45211500DC087FED1CF86E0BB
:10A070001802B0011124C5010E949553B7010F9435
:10A080001747161B112339F026E01202B0011124E4
:10A09000802F992DA7CF10E0812F0F900F900F9058
:10A0A0000F90DF91CF911F910F91FF90EF90DF9074
:10A0B000CF90BF90AF909F908F907F906F900895BA
:10A0C0001F93CF93DF9300D01F92CDB7DEB710E080
:10A0D000AE014F5F5F4F64E279E40E94424E4981D6
:10A0E0005A816B817C81452B462B472B11F01F5FDA
:10A0F000EFCF812F0F900F900F900F90DF91CF91A6
:10A100001F9108951F93CF93DF9300D01F92CDB777
:10A11000DEB710E0AE014F5F5F4F61E279E40E946D
:10A12000424E49815A816B817C81452B462B472BBE
:10A1300011F01F5FEFCF812F0F900F900F900F90B6
:10A14000DF91CF911F9108952F923F924F925F928E
:10A150006F927F928F929F92AF92BF92CF92DF9237
:10A16000EF92FF920F931F93CF93DF9300D0CDB761
:10A17000DEB74C013B015A012B83232E280140916D
:10A18000BF0D5091C00D6091C10D7091C20D411570
:10A1900051056105710579F081E0141615060CF082
:10A1A00080E08093FE141092BF0D1092C00D1092AB
:10A1B000C10D1092C20D1091FE143090A80D109296
:10A1C000A80D311005C080916E02882309F478C073
:10A1D000C2010E948250082FC114D10409F46EC03C
:10A1E000C6010E9482501A821982E114F104B1F46E
:10A1F000402F50E0282F30E0CA01820F931F46976E
:10A200006CF485E190E0841B950B821B930B97FD0A
:10A210000196959587958A8381E0898301E021E203
:10A2200039E4A201BE016F5F7F4FCE0102960E940A
:10A23000D48FE114F10491F08A81882321F01A82ED
:10A2400089818F5F898300E024E239E4A701BE01A0
:10A250006F5F7F4FCE0102960E94D48FC114D1044C
:10A2600059F000E021E239E4A601BE016F5F7F4FA3
:10A27000CE0102960E94D48F41E04127B30181E0D4
:10A280000F94A509C4010E948250412FB40194E1AA
:10A29000981B892F0F94A509332061F0111102C07A
:10A2A000AB80B22CA114B10419F0F501199502C0CC
:10A2B0000E94604D81E080933A0D02C080E093CF10
:10A2C0000F900F900F90DF91CF911F910F91FF9002
:10A2D000EF90DF90CF90BF90AF909F908F907F9046
:10A2E0006F905F904F903F902F900895089580E079
:10A2F00090E00895DF92EF92FF920F931F93CF9318
:10A30000DF93EC01D62E1CAD0BAD7C0184E0E80E92
:10A31000F11CE98DFA8DC7011995412F480F2D2D9C
:10A32000602FC7010E9432969BAD890F8BAF81E0F1
:10A3300090E0DF91CF911F910F91FF90EF90DF9010
:10A3400008959F92AF92BF92CF92DF92EF92FF92C9
:10A350000F931F93CF93DF93EC018B01942EC52EA7
:10A360008A859B858617970731F0888199810E949D
:10A37000E2941B870A8788859985019691F00E8162
:10A380001F81692D7C2D888199810F945809080FB0
:10A39000111D888599858017910718F481E090E058
:10A3A00026C0DC801A819E81190FA880B980D50152
:10A3B0005596ED91FC915697C5011995D80EE92C4B
:10A3C000FC2C00E0D7012D917D01222341F04D2D81
:10A3D000612FC5010E943296180F080FF3CF8E81AE
:10A3E0009F81800F911D9F838E8380E090E0DF919D
:10A3F000CF911F910F91FF90EF90DF90CF90BF9082
:10A40000AF909F900895EF92FF920F931F93CF9379
:10A41000DF93EC018B017A018A859B85861797076C
:10A4200031F0888199810E94E2941B870A87B701E5
:10A43000888199810F9458092E813F81280F311D01
:10A440003F832E8380E090E0DF91CF911F910F91A9
:10A45000FF90EF90089511989091020187FD64C0DC
:10A46000917090930001119A00001198909102014F
:10A47000382F330F86FD56C0917090930001119ACA
:10A480000000119880910201232F220F36FD48C051
:10A49000817080930001119A00001198809102014F
:10A4A000922F990F26FD3AC0817080930001119A76
:10A4B0000000119880910201292F220F96FD2CC0D7
:10A4C000817080930001119A00001198809102011F
:10A4D000922F990F26FD1EC0817080930001119A62
:10A4E0000000119880910201292F220F96FD10C0C3
:10A4F000817080930001119A0000119880910201EF
:10A5000026FD8095817080930001119A00000895C6
:10A510008095EECF8095E0CF8095D2CF8095C4CF47
:10A520008095B6CF9095A8CF90959ACF9CE0899FC3
:10A53000802D112491E0980F9093670D2CE0280F47
:10A540002093660D30E02E5F3F4F40910F1250E098
:10A550002417350714F480E00895292F30E0409146
:10A56000111250E024173507B4F7662341F08E5FCF
:10A570000F948C098091660D8E5F0F948C098091E9
:10A58000660D90910F12891730F32091111290915E
:10A59000670D291700F3109212128093131281E0B5
:10A5A0000895482F50E02091BB03022E000C330B7E
:10A5B0004217530741F08093BB0367EE7DE08BEDBC
:10A5C00091E10C94E2940895CF92DF92EF92FF9282
:10A5D0000F931F93CF93DF93CDB7DEB72C970FB6B2
:10A5E000F894DEBF0FBECDBF6F3F710581059105A9
:10A5F00009F060F487ED91E10E947A51E091DF115A
:10A60000F091E0113196849190E040C0F0901212E8
:10A61000E09013122091C003211109C047EC5DE0C6
:10A620006E2D8F2D0F94C82E80E090E029C0C09031
:10A63000DF11D090E0112BED31E13A8329832F2DEA
:10A6400030E03C832B832E2D30E03E832D83188613
:10A650001F822FEF3FEF3A8729871C861B8601EA6E
:10A6600011E59E012F5F3F4FAB01BC01C6010F9466
:10A67000B50EB6018BED91E10E94E2948F81988531
:10A68000F80EF0921212E092131299272C960FB640
:10A69000F894DEBF0FBECDBFDF91CF911F910F9118
:10A6A000FF90EF90DF90CF9008950F93CF93DF93BB
:10A6B000982F862FEA01692F0E949652882389F1EC
:10A6C0004091AA0D5091AB0D24E16091AC0DCE01EB
:10A6D0000E94944F96E0899FE0011124C730D10574
:10A6E00048F060E270E080E090E00E94E452C81B15
:10A6F000D90BF4CF8091660D9AE790931212809354
:10A700001312602F000F770B880B990B0E94E452F5
:10A7100060E270E080E090E0DF91CF910F910C94C7
:10A72000E452DF91CF910F910895CF92DF92EF9293
:10A73000FF920F931F93CF93DF93CDB7DEB72C9784
:10A740000FB6F894DEBF0FBECDBFF0901212E090AE
:10A7500013122091C003211109C047EC5DE06E2D5A
:10A760008F2D0F94C82E80E090E028C0C090DF119C
:10A77000D090E0112BED31E13A8329832F2D30E089
:10A780003C832B832E2D30E03E832D8318861F8241
:10A790007A8769871C861B8601EA11E59E012F5F77
:10A7A0003F4F41E259E4BC01C6010F94832EB6012C
:10A7B0008BED91E10E94E2948F819885F80EF092E2
:10A7C0001212E092131299272C960FB6F894DEBF5E
:10A7D0000FBECDBFDF91CF911F910F91FF90EF90F2
:10A7E000DF90CF9008956FEF7FEF0C949553CF9249
:10A7F000DF92EF92FF920F931F93CF93DF93CDB72A
:10A80000DEB72C970FB6F894DEBF0FBECDBFF09029
:10A810001212E09013122091C003211109C047ECDD
:10A820005DE06E2D8F2D0F94C82E80E090E028C043
:10A83000C090DF11D090E0112BED31E13A832983F4
:10A840002F2D30E03C832B832E2D30E03E832D8353
:10A8500018861F827A8769871C861B8601EA11E5A4
:10A860009E012F5F3F4F44E259E4BC01C6010F94A3
:10A87000832EB6018BED91E10E94E2948F81988541
:10A88000F80EF0921212E092131299272C960FB63E
:10A89000F894DEBF0FBECDBFDF91CF911F910F9116
:10A8A000FF90EF90DF90CF900895BF92CF92DF920C
:10A8B000EF92FF920F931F93CF93DF938B01F42EB0
:10A8C000E90141FB662760F90E949652882309F44A
:10A8D0005CC00115110529F0C8010E948250B82EF4
:10A8E00001C0B12C209729F0CE010E946050E82EC3
:10A8F00001C0E12CF0FE1EC085E190E08B199109AA
:10A90000B7FC93958E199109E7FC939597FD0196F5
:10A9100095958795F82E30E8C32ED12CFA94F7FC44
:10A920000CC060E270E080E090E00E94E452C81A3F
:10A93000D90AF4CF80E8C82ED12CBB2099F0C601EB
:10A9400066E070E00F940347262F4091AA0D5091C6
:10A95000AB0D6091AC0DC8010E94944F96E0899FA9
:10A9600060011124EE2031F0B601CE010E94F753B0
:10A97000C81AD90A87E0C816D10438F060E270E03E
:10A9800080E090E00E94E452F3CFDF91CF911F91DD
:10A990000F91FF90EF90DF90CF90BF9008956FEFF1
:10A9A0007FEF0C94F753AF92BF92CF92DF92EF926A
:10A9B000FF920F931F93CF93DF935C016B010E9473
:10A9C0008250E82EC6010E946050F12C03E110E095
:10A9D000081B11090E151F0514F0C5E201C0CFE1D7
:10A9E0008C2F90E0AC014E5F5F4F20910F1230E052
:10A9F000421753073CF009972091111230E02817B5
:10AA00003907DCF5D0E0C114D10409F446C06AE38B
:10AA100070E080E090E00E94E4520E151F0584F47F
:10AA2000C45F80910F12C817C0F12C2F30E029505D
:10AA300031098091111290E0821793071CF42DC008
:10AA4000DD2359F1802F880F080F000F0093121299
:10AA5000C093131260E270E080E090E00E94E45244
:10AA6000C601DF91CF911F910F91FF90EF90DF9082
:10AA7000CF90BF90AF900C94CF544091AA0D5091BD
:10AA8000AB0D6091AC0D10921212C093131225E120
:10AA9000C5010E94944FD1E0B6CFDF91CF911F91B5
:10AAA0000F91FF90EF90DF90CF90BF90AF900895FF
:10AAB0008F929F92AF92BF92CF92DF92EF92FF92CE
:10AAC0000F931F93CF93DF93CDB7DEB72C970FB6BD
:10AAD000F894DEBF0FBECDBF982F862F5A017901A3
:10AAE000D02E692F0E949652882309F488C0C7018E
:10AAF000002361F00E948250C82E8090DF11909058
:10AB0000E0118091C00381110EC00BC00E94605003
:10AB1000C82E8090DF119090E0118091C0038111C8
:10AB200013C02FEF2BC09E012F5F3F4F8CE0F90128
:10AB300011928A95E9F78BED91E19A83898303E07D
:10AB400012E541E259E410C09E012F5F3F4F8CE0B7
:10AB5000F90111928A95E9F78BED91E19A83898346
:10AB600003E012E544E259E4B701C4010F94832ED7
:10AB7000B4018BED91E10E94E2942F81122F23E129
:10AB80002C194091AA0D5091AB0D6091AC0DC501EF
:10AB90000E94944FCC2099F1F6E08F9F5001112430
:10ABA0006AE370E080E090E00E94E45257E0A5166E
:10ABB000B10448F060E270E080E090E00E94E4526E
:10ABC000A81AB90AF3CF4091660D212F30E0E6E0D4
:10ABD000CE9EC00111242E5F3F4F281739070CF479
:10ABE0009C0180E8821B8093121240931312C701CC
:10ABF000DD2019F00E94F35302C00E94CF542C961E
:10AC00000FB6F894DEBF0FBECDBFDF91CF911F917D
:10AC10000F91FF90EF90DF90CF90BF90AF909F90FB
:10AC20008F900895E7EDF1E183AF64AFCA010C9412
:10AC3000CF54CF92DF92EF92FF926A017B010E9484
:10AC4000D5F0882331F0FF90EF90DF90CF900C94F7
:10AC500055F0C701B601FF90EF90DF90CF900895B7
:10AC60002F923F924F925F926F927F928F929F921C
:10AC7000AF92BF92CF92DF92EF92FF920F931F930A
:10AC8000CF93DF93CDB7DEB7E7970FB6F894DEBF6B
:10AC90000FBECDBF60E070E085E40E94E2F0882343
:10ACA000E1F08DE99DE0E7960FB6F894DEBF0FBEA8
:10ACB000CDBFDF91CF911F910F91FF90EF90DF906B
:10ACC000CF90BF90AF909F908F907F906F905F904C
:10ACD0004F903F902F900C9446F465E070E083E431
:10ACE0000E94E2F08EA360E085E50E94F1F08DAB5A
:10ACF00040E050E06EE373E483E50E9419566B0177
:10AD00007C0160E080E99DE00E94FCD6C701B601AD
:10AD10000F94B248072E000C880B990B0F94374004
:10AD2000162F7D838E83292E0E9495FA2B013C01DC
:10AD300060912102709122026F507109072E000C60
:10AD4000880B990B0F9437409B01AC01612F7D81DB
:10AD50008E81922D0F94A64918162CF485E69DE05D
:10AD60000E9446F427C2A3019201205C33464F4F54
:10AD70005F4F29AB3AAB4BAB5CAB81E59DE00E94EA
:10AD800046F40E94BFCB8FE78093390F81E0809318
:10AD900023024D8A5E8A6F8A788E48A659A66AA6D3
:10ADA0007BA68FE790E0A0E0B0E08F839887A9872B
:10ADB000BA871D8E1E8E1F8E18A2198E1A8E1B8E9C
:10ADC0001C8E812C912C54011D8690E49E87ACE151
:10ADD000AF87B6E4B88B198A1A8A1B8A1C8A1CA60C
:10ADE0008DA69EA6AFA6B8AAFFE7CF2ED12CE12C48
:10ADF000F12C1AA21BA21CA21DA221E029A31C86D1
:10AE00001B86312C00E01EAA1FAA4EA1042E000CA6
:10AE1000550B5FA34EA380912302882309F4C8C178
:10AE20000E9495FA69837A838B839C838091D40CEA
:10AE3000882309F490C00E9472CC3090330F0091A7
:10AE4000340F5091350F5EAB8091360F8FAB29894F
:10AE50003A894B895C89632D702F8EA99FA90F9425
:10AE6000A649181634F4398A0A8B9EA99B8BAFA980
:10AE7000AC8B2D853E854F855889632D702F8EA90B
:10AE80009FA90F94304087FF06C03D860E87BEA95C
:10AE9000BF872FA9288B39A1232D3323E9F1302F28
:10AEA0004EA95FA9612F7D818E81922D0F94304034
:10AEB00087FF51C049815A816B817C8144195509B2
:10AEC00066097709DB01CA0188589341A109B109D4
:10AED000B7FD41C08F819885A985BA858C199D09D8
:10AEE000AE09BF09B595A795979587958093390FBA
:10AEF0004AA35BA36CA37DA3198B4D814A8B5E8112
:10AF00005B8B2C8A89819A81AB81BC818D8B9E8BD6
:10AF1000AF8BB88F19A21FC0302F4EA95FA9612F28
:10AF20007D818E81922D0F94A6491816A4F48981F3
:10AF30009A81AB81BC812D893E894F89588D821BB6
:10AF4000930BA40BB50BAC01BD01485853416109EB
:10AF5000710977FF49C120E030E040EF51E4612FF3
:10AF60007D818E81922D0F944647232D302F4EA93F
:10AF70005FA90F94304087FF03C085E69DE0A8C01D
:10AF800089819A81AB81BC8128A539A54AA55BA599
:10AF9000821B930BA40BB50BB7FD7EC080E00E9413
:10AFA00056C68AE00E94413889819A81AB81BC8172
:10AFB0008053984FAF4FBF4F88A799A7AAA7BBA7A9
:10AFC0009CA591114EC02DA53EA54FA558A9632D56
:10AFD000702F8EA99FA90F94A64918167CF520E022
:10AFE00030E040E050E4632D702F8EA99FA90F94AC
:10AFF00046476DA77EA78FA798AB29813A814B81E1
:10B000005C81205C33464F4F5F4F29AB3AAB4BAB73
:10B010005CAB20E030E040EE50E4612F7D818E811A
:10B02000922D0F944547232D302F4EA95FA90F94E1
:10B030003040881F8827881F8CA72EC089819A815D
:10B04000AB81BC8129A93AA94BA95CA9821B930BAE
:10B05000A40BB50BB7FD20C045EE52E466EF72E4D9
:10B0600018C020E030E040EF51E4612F7D818E81F7
:10B07000922D0F9445479B01AC01632D702F8EA933
:10B080009FA90F94304087FF07C043E253E465E374
:10B0900073E480E00F94592A8D899E89AF89B88D19
:10B0A000481659066A067B0610F4D301C2012981AD
:10B0B0003A814B815C81281B390B4A0B5B0BDA010F
:10B0C000C90181389F44A241B10528F08AEE9CE075
:10B0D0000E9446F46DC04EA15FA18B859C854817E8
:10B0E00059070CF062C003970CF45FC08DE89CE038
:10B0F0000E9446F480E79CE00E9446F4B501A4015A
:10B1000089E89CE00E9419F58AE00E94413880E7B6
:10B110009CE00E9446F4498D5A8D6B8D7C8D85E8AC
:10B120009CE00E9419F58AE00E94413880E79CE08B
:10B130000E9446F44D8D5E8D6F8D78A181E89CE074
:10B140000E9419F58AE00E9441389DA9992391F146
:10B1500080923A0F90923B0FA0923C0FB0923D0F1D
:10B160002CEA35EC47E25EE3698D7A8D8B8D9C8D00
:10B170000F94964060933E0F70933F0F8093400F63
:10B180009093410F2CEA35EC47E25EE36D8D7E8DA6
:10B190008F8D98A10F9440486093420F7093430F96
:10B1A0008093440F9093450F05C00E94686C33CE86
:10B1B0000E94BFCBE7960FB6F894DEBF0FBECDBF9F
:10B1C000DF91CF911F910F91FF90EF90DF90CF9083
:10B1D000BF90AF909F908F907F906F905F904F90B7
:10B1E0003F902F900D94E5054B855C85452B09F428
:10B1F00007C14AA05BA06CA07DA0480E591E6A1E24
:10B200007B1E2AA13BA14CA15DA1281B390B4A0B37
:10B210005B0BC701B6010F947646A30192010F9410
:10B22000A846CF80D884E984FA84C20ED31EE41ED7
:10B23000F51E54E1C516D104E104F1040CF18CEEC5
:10B24000C816D104E104F1043CF490E8C916D10415
:10B25000E104F10434F422C04BEEC42ED12CE12CD5
:10B26000F12CCF82D886E986FA862EEF30E040E0D6
:10B2700050E02C193D094E095F0969017A0112C09D
:10B2800084E190E0A0E0B0E08F839887A987BA8737
:10B2900034E1C32ED12CE12CF12C04C0CF82D8860E
:10B2A000E986FA8689E49DE00E9446F46F817885FC
:10B2B00089859A850E94B53884E49DE00E9446F411
:10B2C000C701B6010E94B5384D855E856F857889C6
:10B2D0008DE39DE00E9419F549895A896B897C8923
:10B2E00086E39DE00E9419F5AB85BC8513970CF4AD
:10B2F00087C0C701B6010F94374020E030E040E836
:10B3000050E40F9496404B015C012D853E854F859E
:10B31000588969897A898B899C890F9445472BEDD7
:10B320003FE049E450E40F94964020E030E040E0F4
:10B330005FE30F9496409B01AC01C501B4010F94EB
:10B3400040484B015C01C301B2010F9437402FE626
:10B3500032E143E85AE30F9496402B013C01B501DA
:10B36000A40180E39DE00E9419F5B301A2018AE2E5
:10B370009DE00E9419F52AE939E949E15FE3C50139
:10B38000B4010F9496404B015C019B01AC01C301D9
:10B39000B2010F94964020E030E040E05EE30F946D
:10B3A00096406D8F7E8F8F8F98A3A5019401C50164
:10B3B000B4010F944647A30192010F944048698F4E
:10B3C0007A8F8B8F9C8F88E09DE00E9446F4B501B8
:10B3D000A40184E29DE00E9419F5498D5A8D6B8D80
:10B3E0007C8D8EE19DE00E9419F54D8D5E8D6F8DF7
:10B3F00078A188E19DE00E9419F58AE00E94413819
:10B400008F819885A985BA858C0D9D1DAE1DBF1DA8
:10B41000B595A795979587958093390F2B853C8592
:10B420002F5F3F4F3C872B871D873D813E874E8195
:10B430004F87288A49805A806B807C8051E059A3CD
:10B440008ACD2F923F924F925F926F927F928F920E
:10B450009F92AF92BF92CF92DF92EF92FF920F93A3
:10B460001F93CF93DF93D62FC72FFC01808091804D
:10B47000A280B380C501B40120E831E541E050E08D
:10B480000F948646C9016DE671E00F9403476B0186
:10B490007C01C501B40120E13EE040E050E00F94A2
:10B4A0008646CA01B90128E130E040E050E00F943F
:10B4B0008646362E272E062F172F8CE3482E512C2A
:10B4C000612C712CC501B401A30192010F94864631
:10B4D000B62EA72ECA01B901A30192010F94864688
:10B4E000CB01C114D104D9F0AF92BF927F936F9377
:10B4F0002F923F92FF92EF92DF92CF928CE59CE0E9
:10B500009F938F93CF93DF930F94C83F8DB79EB7D0
:10B510000E960FB6F8949EBF0FBE8DBF5CC0E114AF
:10B52000F104C9F0AF92BF927F936F932F923F9235
:10B53000FF92EF9280E69CE09F938F93CF93DF93EF
:10B540000F94C83FEDB7FEB73C960FB6F894FEBF18
:10B550000FBEEDBF40C0012BB9F0AF92BF927F93F9
:10B560006F932F923F9284E69CE09F938F93CF93AB
:10B57000DF930F94C83F8DB79EB70A960FB6F89425
:10B580009EBF0FBE8DBF27C0892BA9F0AF92BF927F
:10B590007F936F9388E69CE09F938F93CF93DF9385
:10B5A0000F94C83FEDB7FEB738960FB6F894FEBFBC
:10B5B0000FBEEDBF10C0AF92BF928CE69CE09F9390
:10B5C0008F93CF93DF930F94C83F0F900F900F90FE
:10B5D0000F900F900F908D2F9C2FDF91CF911F9187
:10B5E0000F91FF90EF90DF90CF90BF90AF909F9022
:10B5F0008F907F906F905F904F903F902F90089525
:10B600008F929F92AF92BF92CF92DF92EF92FF9272
:10B610000F931F93CF93DF93CDB7DEB7E6970FB6A7
:10B62000F894DEBF0FBECDBF0091B9031091BA03ED
:10B63000F80101900020E9F731976F01C01AD10A93
:10B64000F801CF01801B910B8C159D0534F480818E
:10B650008F3209F410823196F4CF8BE1E9E5F2E103
:10B66000DE015C9601900D928A95E1F7E12CF12CB8
:10B67000EC14FD040CF07AC0F801EE0DFF1D808182
:10B68000811103C08FEFE81AF80A48018E0C9F1C45
:10B69000F4018081882309F469C0FFEFEF1AFF0AE3
:10B6A000F801EE0DFF1D7F01E01AF10A8191811171
:10B6B000FACFCE014C960E940DC58BE1FE017C961F
:10B6C000DE01119601900D928A95E1F7B401CE0149
:10B6D00001960E941E99CE0101960E9428F18FE2E8
:10B6E0000E9441388091F60D811103C082ED92E0F5
:10B6F00002C086EF9DE05C01F50181915F01882326
:10B7000019F00E944138F8CF80913C1284FF2EC07E
:10B7100019821C8221E0A401BE01645E7F4FCE012C
:10B7200001960E9492C281110FC08AE00E944138A6
:10B730000E944EF5B40182EA91E30E9437F5CE01F2
:10B7400001960E9428F112C0CE014C960E9489C237
:10B750008BE1FE013196DE015C9601900D928A9597
:10B76000E1F7CE0101960E9428F182CF8AE00E9483
:10B770004138CE014C960E9428F1E6960FB6F89417
:10B78000DEBF0FBECDBFDF91CF911F910F91FF9014
:10B79000EF90DF90CF90BF90AF909F908F900895E3
:10B7A000AB01BC01409338125093391260933A12A6
:10B7B00070933B128DE993E10C945FBCCF93DF93C0
:10B7C000EC01CB01BA010F94374020E030E0A90131
:10B7D0000F9446470F94B24879836883DF91CF91E5
:10B7E00008950C94604DCF92DF92EF92FF920F93E9
:10B7F0001F9387E5C82E86E3D82EE12CF12C0DEAA5
:10B8000019E121EF3BE54FEC56ED68E07BE384ED79
:10B8100099E10E94A4501F910F91FF90EF90DF904B
:10B82000CF9008950E94584D87EA99E19093DD04E6
:10B830008093DC0408950E9406F10E94C299109240
:10B8400031120C94584D9F92AF92BF92CF92DF92DB
:10B85000EF92FF920F931F93CF93DF9381E080933A
:10B860003A0D61E00E943F4CD091AE0DC0E09924AA
:10B8700093940BE11CE58DEAE82E89E1F82E92E124
:10B88000C92E9CE5D92E20ECA22E29E1B22ED11191
:10B890002BC09920D9F08091AD0D1816BCF04091C5
:10B8A000BF0D5091C00D6091C10D7091C20D4F5FE1
:10B8B0005F4F6F4F7F4F4093BF0D5093C00D60930C
:10B8C000C10D7093C20D8F5F8093AD0D80916E029C
:10B8D000882309F441C020E030E041E06AE478E1E7
:10B8E0008C2F0E94555438C0D13059F48091AD0D41
:10B8F0008130D1F48091A80D1092A80D81110EC055
:10B9000013C0D23049F58091AD0D8230A1F5809100
:10B91000A80D1092A80D811128C02DC00E94125CA4
:10B920008091CF0D811137C080916E02882399F0EC
:10B93000DF92CF92BF92AF92CF9381E09091AD0D05
:10B94000913039F58F930E94194C0F900F900F9002
:10B950000F900F900F90912CCF5FDF5FC53009F0F3
:10B9600096CF83E08093A90D16C00E941B5C809146
:10B97000CF0D811110C080916E02882361F31F9357
:10B980000F93FF92EF92CF9381E09091AD0D9230A3
:10B99000C9F280E0D7CFDF91CF911F910F91FF9037
:10B9A000EF90DF90CF90BF90AF909F900895EF926F
:10B9B000FF920F931F93CF93DF93CDB7DEB76597B9
:10B9C0000FB6F894DEBF0FBECDBF8091A80D1092C8
:10B9D000A80D882319F00E94604D7AC060E085E0D0
:10B9E0000E943F4C0091AE0D10E08AE3F82E90E2E9
:10B9F000E92E01110AC080916E02882361F120E0D6
:10BA000030E043E06FE670E323C0013051F48091F1
:10BA10006E02882301F120E030E041E067EE7FE232
:10BA200017C0023051F480916E028823A1F020E00B
:10BA300030E041E065E679E10BC00330E9F5809143
:10BA40006E02882341F020E030E041E06FE378E1CE
:10BA5000812F0E945554F982EA8242E150E06DEE56
:10BA60007FE2CE0103960F949F3F8C8987FD1C8A4D
:10BA7000053059F480916E028823A9F09E012F5F52
:10BA80003F4F41E069E97AE30BC0063061F48091F1
:10BA90006E02882341F020E030E041E063E579E187
:10BAA000812F0E9455541F5F0F5F153009F0A1CF01
:10BAB00087E08093A90D0CC0043069F680916E0276
:10BAC000882349F220E030E041E062ED7FE2C0CF20
:10BAD00065960FB6F894DEBF0FBECDBFDF91CF9154
:10BAE0001F910F91FF90EF900895EF92FF920F93A7
:10BAF0001F93CF93DF93CDB7DEB765970FB6F8945A
:10BB0000DEBF0FBECDBF8091A80D1092A80D882377
:10BB100019F00E94604D75C060E085E00E943F4CC6
:10BB20000091AE0D10E08AE3F82E90E2E92E0111AB
:10BB30000CC080916E02882341F020E030E043E0A9
:10BB400069E479E1812F0E945554F982EA8242E149
:10BB500050E062E479E1CE0103960F949F3F8C8917
:10BB600087FD1C8A013069F480916E02882349F0B8
:10BB70009E012F5F3F4F41E069E379E1812F0E94F1
:10BB80005554F982EA8242E150E065E379E1CE0161
:10BB900003960F949F3F8C8987FD1C8A023069F4BD
:10BBA00080916E02882349F09E012F5F3F4F41E054
:10BBB0006BE279E1812F0E945554F982EA8242E1D9
:10BBC00050E061E279E1CE0103960F949F3F8C89AA
:10BBD00087FD1C8A033069F480916E02882349F046
:10BBE0009E012F5F3F4F41E068E179E1812F0E9484
:10BBF00055541F5F0F5F153009F099CF84E0809393
:10BC0000A90D65960FB6F894DEBF0FBECDBFDF91CC
:10BC1000CF911F910F91FF90EF900895EF92FF92B7
:10BC20000F931F93CF93DF93CDB7DEB765970FB612
:10BC3000F894DEBF0FBECDBF8091A80D1092A80D65
:10BC4000882319F00E94604DB5C060E085E00E9435
:10BC50003F4C0091AE0D10E08AE3F82E90E2E92E01
:10BC600001110CC080916E02882341F020E030E089
:10BC700042E069E079E1812F0E945554F982EA821D
:10BC800042E150E060ED78E1CE0103960F949F3FD2
:10BC90008C8987FD1C8A013069F480916E028823AB
:10BCA00049F09E012F5F3F4F40E060E079E1812F36
:10BCB0000E945554F982EA8242E150E06CEF78E14B
:10BCC000CE0103960F949F3F8C8987FD1C8A02301A
:10BCD00059F480916E02882309F19E012F5F3F4F36
:10BCE00040E063EF78E117C0033051F480916E02B9
:10BCF0008823A1F020E030E040E061EE78E10BC065
:10BD0000043061F480916E02882341F020E030E03D
:10BD100042E062ED78E1812F0E945554F982EA8277
:10BD200042E150E060ED78E1CE0103960F949F3F31
:10BD30008C8987FD1C8A053069F480916E02882306
:10BD400049F09E012F5F3F4F40E060E079E1812F95
:10BD50000E945554F982EA8242E150E06EEC78E1AB
:10BD6000CE0103960F949F3F8C8987FD1C8A063075
:10BD700059F480916E028823A9F09E012F5F3F4FF6
:10BD800040E063EF78E10BC0073061F480916E0210
:10BD9000882341F020E030E040E061EE78E1812F3F
:10BDA0000E9455541F5F0F5F153009F059CF88E08E
:10BDB0008093A90D65960FB6F894DEBF0FBECDBF78
:10BDC000DF91CF911F910F91FF90EF9008952F92E7
:10BDD0003F924F925F926F927F928F929F92AF921B
:10BDE000BF92CF92DF92EF92FF920F931F93CF9368
:10BDF000DF93CDB7DEB7A1970FB6F894DEBF0FBEC5
:10BE0000CDBF8091A80D1092A80D882319F00E9433
:10BE1000604D19C18091C7049091C80499A388A36B
:10BE2000A091C904B091CA04BF8FAE8F4090CB04DB
:10BE30005090CC046090CD047090CE048091CF04DB
:10BE40009091D004A091D104B091D2048A8F9B8F9D
:10BE5000AC8FBD8F8090D3049090D404A090D50473
:10BE6000B090D60460E085E00E943F4C0091AE0D9A
:10BE700010E0DE0111967D018AE0C82ED12C9CE6EF
:10BE8000292E98E1392E01110DC080916E02882370
:10BE9000D9F188A199A10F94E7379C0140E06FEB9D
:10BEA00078E12FC0013069F480916E02882361F13E
:10BEB0008E8D9F8D0F94E7379C0140E06EEA78E10C
:10BEC00020C0023051F480916E028823E9F020E016
:10BED00030E040E06CE978E114C0033009F053C071
:10BEE00080916E02882381F04E8A5F8A688E798EF7
:10BEF000B701CE0146960E94215A9C0140E069E9B3
:10BF000078E1812F0E94555420E030E048EC52E463
:10BF1000C501B4010F9440480F94B248CB01B6015B
:10BF20000F9417479F938F9320E030E04AE754E443
:10BF3000C501B4010F9440480F94B2489F938F936A
:10BF40007F936F933F922F92FF92EF920F94C83F8F
:10BF50000FB6F894DEBF0FBECDBF073059F4809105
:10BF60006E02882339F0970140E069E978E1812F7A
:10BF70000E9455541F5F0F5F153009F084CF88E091
:10BF80008093A90D60C0043059F480916E0288231B
:10BF900009F4BACF20E030E040E066E878E118C06C
:10BFA0000530D1F480916E02882309F4ADCF8A8DDB
:10BFB0009B8DAC8DBD8D8E8B9F8BA88FB98FB7015C
:10BFC000CE0146960E94215A9C0140E069E978E141
:10BFD000812F0E9455540DC0063009F095CF8091F5
:10BFE0006E02882331F020E030E040E064E778E141
:10BFF00088CF20E030E048EC52E4C501B4010F9452
:10C0000040480F94B248CB01B6010F9417479F9355
:10C010008F9320E030E04AE754E4C501B4010F9467
:10C0200040480F94B2489F938F937F936F933F92B2
:10C030002F92FF92EF920F94C83F0FB6F894DEBF95
:10C040000FBECDBF97CFA1960FB6F894DEBF0FBE3F
:10C05000CDBFDF91CF911F910F91FF90EF90DF90B7
:10C06000CF90BF90AF909F908F907F906F905F9098
:10C070004F903F902F9008950F94374020E030E08C
:10C08000A9010F9446470F94B248CB010C9428D1D4
:10C090006EED7BE58CE390E60C94774D85EA9AE1B2
:10C0A0000C94BCDC8FE49AE10C94BCDC84E89AE14B
:10C0B0000C94BCDC8EEE9AE10C94BCDC8BEC9AE127
:10C0C0000C94BCDC8AE29AE10C94BCDC2F923F9287
:10C0D0004F926F927F928F929F92AF92BF92CF9228
:10C0E000DF92EF92FF920F931F93CF93DF930E9403
:10C0F000A636382E80913C1283FBDD27D0F983FFD2
:10C1000004C00E948937282E01C0212C61E081E003
:10C110000E943F4C1091AE0D412C8DEF682E8CEC9F
:10C12000782E91EAE92E96EDF92E27E1C22E2AE12A
:10C13000D22E30E0A32E3AE1B32E4AEE842E49E10E
:10C14000942E11110BC08091AD0D81113BC08091D7
:10C15000A80D1092A80D81112FC034C0332009F40E
:10C1600043C0113061F48091AD0D813009F090C170
:10C170008091A80D1092A80D811184C189C112303F
:10C1800061F48091AD0D823009F0A3C08091A80DBB
:10C190001092A80D811195C09CC0133009F092C176
:10C1A0008091AD0D833009F097C18091A80D109258
:10C1B000A80D811189C190C10E94604D8091CF0D61
:10C1C0008111D8C180916E02882361F081E0909145
:10C1D000AD0D911180E004E024E045E959E1642DC2
:10C1E0000E94555331106EC10E949737882371F019
:10C1F000113071F48091AD0D813009F083C18091CF
:10C20000A80D1092A80D811177C17CC1C1E001C0B9
:10C21000C2E0C11322C08091AD0D8C130EC080917D
:10C22000A80D1092A80D882341F08AE391E00E94A6
:10C23000C3908091CF0D81119DC180916E028823A2
:10C2400061F081E09091AD0D911380E003E02EE369
:10C250004EE35CE3642D0E945553CF5FC11322C0AF
:10C260008091AD0D8C130EC08091A80D1092A80D79
:10C27000882341F08BEB92E90E94C3908091CF0D0F
:10C28000811178C180916E02882361F081E09091E4
:10C29000AD0D911380E003E02EE34CED5BE0642DE7
:10C2A0000E94555381E08C0F811326C08091AD0D03
:10C2B00081134CC18091A80D1092A80D81113EC12F
:10C2C00045C183EF9BE50E94C3908091CF0D811102
:10C2D00051C180916E02882309F44AC181E0909196
:10C2E000AD0D923009F080E003E02EE34DEA59E114
:10C2F000642D0E945553C4E082E08C0F811322C04C
:10C300008091AD0D81130EC08091A80D1092A80DE3
:10C31000882341F086EE98ED0E94C3908091CF0D66
:10C32000811128C180916E02882361F081E0909193
:10C33000AD0D911380E003E02EE344EB5AE3642D4E
:10C340000E94555383E08C0F811322C08091AD0D64
:10C3500081130EC08091A80D1092A80D882341F082
:10C360008CEC92E60E94C3908091CF0D811102C1A6
:10C3700080916E02882361F081E09091AD0D911360
:10C3800080E003E02EE34EEE59E1642D0E94555308
:10C3900084E08C0F31106EC0DD2309F44CC02110F5
:10C3A00069C0811320C09091AD0D91130EC0809192
:10C3B000A80D1092A80D882341F09092DD04809280
:10C3C000DC048091CF0D8111D5C080916E0288234D
:10C3D00051F081E0911380E000E22EE349ED59E154
:10C3E000642D0E94555385E08C0F811322C08091EB
:10C3F000AD0D81130EC08091A80D1092A80D882359
:10C4000041F080ED91E00E94C3908091CF0D8111A9
:10C41000B1C080916E02882361F081E09091AD0DF2
:10C42000911380E003E02EE34FEA5CE3642D0E9469
:10C43000555386E01EC081131BC08091AD0D811342
:10C4400002C01092A80D90916E02992389F01F925C
:10C450001F92BF92AF924F9291E0811390E09F9311
:10C460000E94194C0F900F900F900F900F900F900B
:10C4700085E08C0F43941F5F95E0491262CE809354
:10C48000A90D78C00E94A1D68091CF0D811172C0F4
:10C4900080916E02882309F46BC0FF92EF92DF92C5
:10C4A000CF924F9281E09091AD0D913009F080E0F4
:10C4B0008F930E94194C0F900F900F900F900F9038
:10C4C0000F9056C0C4E0CACE81ED90E90E94C3909F
:10C4D0008091CF0D81114EC080916E02882309F4A6
:10C4E00047C081E09091AD0D933009F080E003E00A
:10C4F0002EE34CE05AE1FCCE0E94FDCC8091CF0DA2
:10C50000811138C080916E028823B1F07F926F92C2
:10C5100080EC99E19F938F934F9281E09091AD0DC4
:10C52000913009F080E08F930E94194C0F900F908A
:10C530000F900F900F900F90C2E08FCE84E59AED90
:10C540000E94C3908091CF0D811114C080916E0222
:10C55000882309F4D1CE81E09091AD0D911380E054
:10C5600003E02EE34EE558E1642D0E945553C4CEFE
:10C57000C4E098CEDF91CF911F910F91FF90EF9083
:10C58000DF90CF90BF90AF909F908F907F906F90F3
:10C590004F903F902F9008950F93CF93DF9361E0DA
:10C5A00081E00E943F4CD091AE0DC0E0D1110BC094
:10C5B0008091AD0D811129C08091A80D1092A80D18
:10C5C00081111DC022C0D13059F48091AD0D813050
:10C5D00091F58091A80D1092A80D811124C02BC057
:10C5E000D23009F041C08091AD0D823009F05EC0BB
:10C5F0008091A80D1092A80D811150C057C00E94C3
:10C60000604D8091CF0D811190C080916E02882382
:10C6100019F181E09091AD0D911180E004E024E0EA
:10C6200043E451E316C087ED9CE50E94C3908091DE
:10C63000CF0D81117AC080916E02882369F081E06C
:10C640009091AD0D913009F080E003E02EE34AE9CE
:10C6500059E16C2F0E945553CF5FDF5FC53009F061
:10C66000A5CFC093A90D61C0D33059F48091AD0D11
:10C67000833099F58091A80D1092A80D811125C0E5
:10C680002CC0D43049F78091AD0D8430F1F5809104
:10C69000A80D1092A80D811130C037C085E79DE527
:10C6A0000E94C3908091CF0D81113FC080916E0296
:10C6B000882391F281E09091AD0D923009F080E0F5
:10C6C00003E02EE34FE859E1C4CF8EE09EE50E94DF
:10C6D000C3908091CF0D811128C080916E02882374
:10C6E00009F4BACF81E09091AD0D933009F080E06C
:10C6F00003E02EE342E859E1ACCF87EE9EE50E94CD
:10C70000C3908091CF0D811110C080916E0288235B
:10C7100009F4A2CF81E09091AD0D943009F080E052
:10C7200003E02EE340E759E194CFDF91CF910F91E1
:10C7300008956111609302024093BC03082E000C1F
:10C74000990BAA0BBB0B8C30910570F5FC01882767
:10C75000EA55FF4F8F4F0D942B4782E590E61BC0A3
:10C7600083EF9DED16C08FEE9DED13C08AE590E638
:10C7700012C08EE590E60FC082E690E60CC08BEE0C
:10C780009DED07C01092E60D8AEB97ED02C087EF92
:10C790009DED009749F021E020933A0D20E040E024
:10C7A00060E070E00C94A84C0C94584D8EE490E638
:10C7B000F2CF86E590E6EFCFE091AC0D86E0E8029F
:10C7C000F0011124E15DFB4F8091B10D90E0958364
:10C7D000848308953F924F925F926F927F928F92DF
:10C7E0009F92AF92BF92CF92DF92EF92FF920F9300
:10C7F0001F93CF93DF93CDB7DEB728970FB6F8948A
:10C80000DEBF0FBECDBF3090AC0D61E081E00E9475
:10C810003F4C2091AE0D28871F8211E0232D30E080
:10C82000C901880F991FAC01405D534C5A8349835D
:10C8300046E0429FC001439F900D1124FC01E15D41
:10C84000FB4F3F019F012C5F3F4F3C832B832F0108
:10C8500032E0430E511CAC014F5C5B4F5E834D8355
:10C86000588551112CC01123D9F08091AD0D1816A7
:10C87000BCF04091BF0D5091C00D6091C10D709101
:10C88000C20D4F5F5F4F6F4F7F4F4093BF0D50936F
:10C89000C00D6093C10D7093C20D8F5F8093AD0D7D
:10C8A00080916E02882381F1E981FA81659174910A
:10C8B00020E030E043E08F810E94555425C08885F8
:10C8C000813011F58091AD0D813061F48091A80D1A
:10C8D0001092A80D882331F00E94604D8091CF0DF9
:10C8E00081112BC180916E02882369F081E09091C3
:10C8F000AD0D913009F080E004E024E04EE558E110
:10C900006F810E94555310E0EB81FC818081809300
:10C91000B10DF885F23071F43092AC0D8091AD0D0F
:10C92000823009F03EC08091A80D1092A80D8111AF
:10C930002EC037C02885233061F48091AD0D83303F
:10C9400009F07FC08091A80D1092A80D81114DC0F3
:10C9500078C0F885F43061F48091AD0D843009F031
:10C96000B2C08091A80D1092A80D81117EC0ABC0FD
:10C97000F885F53069F58091AD0D853009F0BEC0C0
:10C980008091A80D1092A80D8111B2C0B7C06CEDB6
:10C9900073E68EE291E30F941B398091CF0D8111E4
:10C9A000CCC080916E02882391F011E08091AD0D92
:10C9B000823009F010E08091B10D0E948DD100E02D
:10C9C0009C014EE251E36F81812F0E94585510E087
:10C9D0002F812F5F2F8338853F5F3887253009F0FF
:10C9E0003FCF86E08093A90DA8C0F30160817181DB
:10C9F00080E090E00F94354020E030E0A9010F94F2
:10CA0000464720E030E040EA50E40F9445470F9459
:10CA1000B948812C912C24EDA22E28EDB22E6B0169
:10CA2000E12CF12C8701EA9425E030E040E050E071
:10CA3000B30186E391E30F943E0A8091CF0D8111FB
:10CA40007CC080916E02882311F211E08091AD0DBF
:10CA5000833009F010E0F301808191810E945ED162
:10CA600000E09C0146E351E3AECFF20160817181A9
:10CA700080E090E00F94354020E030E0A9010F9471
:10CA8000464720E030E040EA50E40F9445470F94D9
:10CA9000B948812C912C84EDA82E88EDB82E6B011D
:10CAA0001EE6E12EF12C00E010E025E030E040E051
:10CAB00050E06D817E818BEF92E30F943E0A80916E
:10CAC000CF0D81113AC080916E02882309F47FCF87
:10CAD00011E08091AD0D843009F010E0F201808109
:10CAE00091810E945ED100E09C014BEF52E36BCF3D
:10CAF0000E94E0CC8091CF0D81111FC080916E0209
:10CB0000882309F464CF20EE3CEC3F932F9381EE11
:10CB100096E39F938F93FF81FF9381E09091AD0DFA
:10CB2000953009F080E08F930E94194C0F900F9080
:10CB30000F900F900F900F904ACF28960FB6F89451
:10CB4000DEBF0FBECDBFDF91CF911F910F91FF9040
:10CB5000EF90DF90CF90BF90AF909F908F907F909D
:10CB60006F905F904F903F90089581E080933A0DD1
:10CB70001092DA041092AE0420E040E060E070E031
:10CB80008BEC95E60E94A84C8BEA9CE39093DD0425
:10CB90008093DC04089580916E02882341F020E0A8
:10CBA00030E041E06BE57BE182E00E9455548091EA
:10CBB000AE048770873041F420E040E060E070E030
:10CBC0008EEF95E60C94A84C089520E040E060E0DC
:10CBD00070E081E496E60E94A84C81E08093BE0359
:10CBE0008091BF03811103C082E49BE102C080E316
:10CBF00092E49093DD048093DC04089580916E02AA
:10CC0000882341F020E030E041E069E47BE181E00D
:10CC10000E9455548091A80D1092A80D882321F0F0
:10CC20001092BF030C94E565089581E080933A0D5E
:10CC30008091DA048770873051F01092DA041092F4
:10CC4000AE048BEA9CE39093DD048093DC04809136
:10CC5000410E8093BD0380E00E94F1F220E040E0AD
:10CC600060E070E080E592E00C94A84C6091B10D1A
:10CC70007091B20D8091B30D9091B40D41E00C9480
:10CC80000CF30F931F93CF93DF93CDB7DEB72A97A3
:10CC90000FB6F894DEBF0FBECDBF80916E02882321
:10CCA000F1F01F9289E08F938091BF0390E001968D
:10CCB0009F938F938AE39BE19F938F938E010F5FE6
:10CCC0001F4F1F930F930F94C83FB80186E29BE15B
:10CCD0000E94D3540FB6F894DEBF0FBECDBF84E0E0
:10CCE00080936E028091BE03811108C020E040E075
:10CCF00060E070E089E896E60E94A84C2A960FB69C
:10CD0000F894DEBF0FBECDBFDF91CF911F910F9181
:10CD10000895CF92DF92EF92FF920F931F93CF93DC
:10CD2000DF9300D01F92CDB7DEB78091A80D10928F
:10CD3000A80D8823E1F08091BF038F5F8093BF032C
:10CD4000893090F081E08093BE0320E040E060E015
:10CD500070E08AE497E60E94A84C80E392E4909306
:10CD6000DD048093DC0489C00E94E56586C0609183
:10CD7000BF0D7091C00D8091C10D9091C20D6115D4
:10CD800071058105910509F448C00F9437402DECD9
:10CD90003CEC4CEC5CE30F9496402091591130919F
:10CDA0005A1140915B1150915C110F9446477B01E1
:10CDB0008C0120E030E040E050EC0F94304087FDE3
:10CDC0000FC020E030E040E050E4B701C8010F940C
:10CDD000A64918164CF4E12CF12C00E010E404C034
:10CDE000E12CF12C00E010ECC701D801809359111F
:10CDF00090935A11A0935B11B0935C118BE892E071
:10CE00000E94798982E080936E021092BF0D109289
:10CE1000C00D1092C10D1092C20D80916E02882338
:10CE200061F1C0905911D0905A11E0905B11F090CF
:10CE30005C1120E030E0A901C701B6010F94304039
:10CE400087FD05C027E137EB41ED58E304C027E13A
:10CE500037EB41ED58EBC701B6010F9446476983A4
:10CE60007A838B839C836BE2CE0101960E94BBCDBB
:10CE7000BC018EE39AE30E94D3540F900F900F9061
:10CE80000F90DF91CF911F910F91FF90EF90DF9066
:10CE9000CF9008958091BE03811104C00E943E4E40
:10CEA0000E942A4C80916E02882341F020E030E0FD
:10CEB00041E062E17BE181E00E94555482E0809391
:10CEC0006E0208952F923F924F925F926F927F92DF
:10CED0008F929F92AF92BF92CF92DF92EF92FF928A
:10CEE0000F931F93CF93DF9300D0CDB7DEB7809120
:10CEF000DA04877089830E94F5F3682E61E081E08F
:10CF00000E943F4C2091AE0D2A83712C45EF442E98
:10CF10004CEC542E51EE252E56E3352E8A8181118C
:10CF20000BC08091AD0D811195C18091A80D10921B
:10CF3000A80D811189C18EC19A81913061F48091CF
:10CF4000AD0D813009F09CC18091A80D1092A80D03
:10CF500081118EC195C12981273011F082E02FC047
:10CF60006620E1F39A81923049F52091410E2B839E
:10CF70008091AD0D823031F48091A80D1092A80DF2
:10CF8000811190C180916E02882309F4B1C181E0C2
:10CF90009091AD0D923009F080E09B81911103C01A
:10CFA00026E037E302C02AE037E301E04BE45CE32C
:10CFB000672D0E94585523E02B8302C083E08B83AA
:10CFC00080913D0E90913E0EA0913F0EB091400E8B
:10CFD0008093B10D9093B20DA093B30DB093B40DA7
:10CFE0009B812A8192133DC08091AD0D89131DC094
:10CFF0008091A80D1092A80D8823B9F00E9462F7C5
:10D0000026E3C22E26E6D22EE12CF12C08EC12E407
:10D0100020E030E0A90161EB7DE088E79BE10E9420
:10D02000C0F68091CF0D811176C180916E02882368
:10D03000C1F011E08091AD0D9A81891310E06091EB
:10D04000B10D7091B20D8091B30D9091B40D0E940D
:10D05000E04B00E09C0148E75BE1672D812F0E94D7
:10D0600058558B818F5F2A8182135CC08091AD0DF2
:10D0700082133CC08091A80D1092A80D8823B1F1B5
:10D0800020E030E04AE754E460913B0470913C04B6
:10D0900080913D0490913E040F94964020E030E052
:10D0A000A9010F94464720E030E04AE754E40F948A
:10D0B00046470F94B948812C912C82E1A82E81E03B
:10D0C000B82E6B0110EDE12E17E0F12E00E010E01C
:10D0D00028E13CEF4FEF5FEF6BE374E08CE391E30B
:10D0E0000F943E0A8091CF0D811115C180916E027F
:10D0F0008823C1F011E08091AD0D9A81891310E071
:10D1000060913B0470913C0480913D0490913E04F9
:10D110000E947E4700E09C014CE351E3672D812F84
:10D120000E9458558B818E5F2A81821323C0809183
:10D13000AD0D82130EC08091A80D1092A80D88230A
:10D1400041F085E196E60E94C3908091CF0D811158
:10D15000E2C080916E02882369F081E09091AD0D6C
:10D160002A81921380E003E02EE346E65BE1672D1F
:10D170000E9455538B818D5F9A8189132AC08091BB
:10D18000AD0D89130CC08091A80D1092A80D8823B5
:10D1900031F00E94F5CC8091CF0D8111BCC08091FF
:10D1A0006E028823B1F05F924F9283ED96E39F93D6
:10D1B0008F937F9281E09091AD0D2A81921380E050
:10D1C0008F930E94194C0F900F900F900F900F901B
:10D1D0000F908B818C5F9A8189132AC08091AD0D4D
:10D1E00089130CC08091A80D1092A80D882331F0EE
:10D1F0000E94E0CC8091CF0D81118DC080916E0294
:10D200008823B1F080EE9CEC9F938F933F922F92F6
:10D210007F9281E09091AD0D2A81921380E08F93EF
:10D220000E94194C0F900F900F900F900F900F903D
:10D2300073948A818F5F8A8395E079126FCE2B81F8
:10D240002B5F2093A90D67C00E94604D8091CF0D88
:10D25000811161C080916E02882399F181E09091E3
:10D26000AD0D911180E004E024E04EE35CE316C0D4
:10D2700085EB95E60E94C3908091CF0D81114BC044
:10D2800080916E028823E9F081E09091AD0D91309C
:10D2900009F080E003E02EE346E85BE1672D0E94A1
:10D2A00055530FC08B8191E089278B8323E0209316
:10D2B0006E020E9427498091CF0D882309F462CE27
:10D2C0002AC09981973009F44BCE80913D0E909100
:10D2D0003E0EA0913F0EB091400E8093B10D909301
:10D2E000B20DA093B30DB093B40D82E08B83B9CE91
:10D2F00080913D0E90913E0EA0913F0EB091400E58
:10D300008093B10D9093B20DA093B30DB093B40D73
:10D3100023E02B83A6CE0F900F900F90DF91CF913B
:10D320001F910F91FF90EF90DF90CF90BF90AF9043
:10D330009F908F907F906F905F904F903F902F9035
:10D3400008958F929F92AF92BF92CF92DF92EF9209
:10D35000FF92CF936B017C0120E030E0A9010F9494
:10D36000304087FD05C06DEB77E386E095E304C0B0
:10D370006DEB77E386E095EBA70196010F944647A6
:10D380006B017C0120E030E040E251E40F949640D4
:10D3900020E030E048EC52E40F9496404B015C01F1
:10D3A00020E030E0A901C701B6010F94304087FDAD
:10D3B00005C020E030E040EA50E404C020E030E066
:10D3C00040EA50ECC501B4010F94464720E030E03C
:10D3D00040E251E40F9440480F94B2486B017C0145
:10D3E00097FF0AC0F094E094D094C094C11CD11C63
:10D3F000E11CF11C8DE201C08BE280933B0DC70163
:10D40000B60120E137E240E050E00F94A8468AE000
:10D41000882E912CA12CB12CCA01B901A50194012F
:10D420000F94A846605D60933C0DC701B60128EEDD
:10D4300033E040E050E00F94A846CA01B901A501CD
:10D4400094010F94A846605D60933D0DC701B6013D
:10D4500024E630E040E050E00F94A846CA01B9014C
:10D46000A50194010F94A846605D60933E0D8EE285
:10D4700080933F0DC701B601A50194010F94A84602
:10D48000C62FCA01B901A50194010F94A846605D99
:10D490006093400DC05DC093410D8BE39DE0CF9143
:10D4A000FF90EF90DF90CF90BF90AF909F908F90C4
:10D4B00008957F928F929F92AF92BF92CF92DF9208
:10D4C000EF92FF920F931F93CF93DF9361E081E080
:10D4D0000E943F4CD091AE0DC0E0A3E07A2ED11156
:10D4E0000BC08091AD0D811129C08091A80D1092C3
:10D4F000A80D81111DC022C0D13059F48091AD0D0D
:10D500008130D1F58091A80D1092A80D811127C00E
:10D5100033C0D23009F04FC08091AD0D823009F098
:10D5200099C08091A80D1092A80D811164C092C07D
:10D530000E94604D8091CF0D8111BCC180916E021F
:10D54000882381F181E09091AD0D911180E004E09C
:10D5500024E04EE558E16C2F0E94555323C0809182
:10D560000D048D2780930D0470926E020E9414DECC
:10D570008091CF0D81119EC180916E02882391F020
:10D5800081E09091AD0D913009F080E090910D0413
:10D5900091111FC026E037E301E047EC5BE16C2FFF
:10D5A0000E945855CF5FDF5FC53009F098CF87E004
:10D5B0008093A90D7FC1D33079F48091AD0D833074
:10D5C00009F077C08091A80D1092A80D81115CC060
:10D5D00070C02AE037E3E0CFD43009F086C08091F4
:10D5E000AD0D843009F0CDC08091A80D1092A80D2A
:10D5F000811198C0C6C020E030E048EC52E4609150
:10D600000E0470910F0480911004909111040F94F6
:10D61000964020E030E0A9010F9446470F94B948A6
:10D62000812C912CE0EEAE2EE8EDBE2E6B0110E1C8
:10D63000E12E17E2F12E00E010E020E030E0A90139
:10D640006EE074E08DEB9BE10F943E0A8091CF0D6C
:10D65000811130C180916E02882309F4A3CF11E0BB
:10D660008091AD0D823009F010E060910E04709150
:10D670000F0480911004909111040E94A16900E0B0
:10D680009C014DEB5BE12EC0C12CD12CE12C10ECA8
:10D69000F12E09E714E420E030E040E85FE362E1C6
:10D6A00074E084EB9BE10E94C0F68091CF0D811164
:10D6B00001C180916E02882309F474CF11E080913A
:10D6C000AD0D833009F010E06091120470911304E5
:10D6D00080911404909115040E94E04B00E09C019D
:10D6E00044EB5BE16C2F812F5BCFD53061F48091EF
:10D6F000AD0D853009F095C08091A80D1092A80D50
:10D70000811159C08EC0D63009F04CCF8091AD0D3B
:10D71000863009F0B5C08091A80D1092A80D811136
:10D720009AC0AEC020E030E048EC52E460911604AC
:10D730007091170480911804909119040F949640E9
:10D7400020E030E0A9010F9446470F94B948812C9E
:10D75000912C30EEA32E38EDB32E6B011CE3E12E9D
:10D7600016E8F12E01E010E020E030E0A90166E1CA
:10D7700074E088EA9BE10F943E0A8091CF0D8111FD
:10D7800099C080916E02882309F40CCF11E080913A
:10D79000AD0D843009F010E060911604709117040B
:10D7A00080911804909119040E94A16900E09C01E5
:10D7B00048EA5BE197CF20E030E048EC52E460912A
:10D7C0001A0470911B0480911C0490911D040F9405
:10D7D000964020E030E0A9010F94464720E030E475
:10D7E0004CE156E40F9446470F94B948812C912C94
:10D7F00090EEA92E98EDB92E6B0110E2E12E1EE4F9
:10D80000F12E00E010E020EF38ED4FEF5FEF6AE11E
:10D8100074E08FE99BE10F943E0A8091CF0D811156
:10D8200049C080916E02882309F4BCCE11E080913A
:10D83000AD0D853009F010E060911A0470911B0461
:10D8400080911C0490911D040E94A16900E09C013C
:10D850004FE95BE147CFC12CD12CE12C10ECF12E2C
:10D8600009E714E420E030E040E85FE36EE174E0B3
:10D8700087E99BE10E94C0F68091CF0D81111AC00B
:10D8800080916E02882309F48DCE11E08091AD0D58
:10D89000863009F010E060911E0470911F048091A1
:10D8A0002004909121040E94E04B00E09C0147E994
:10D8B0005BE118CFDF91CF911F910F91FF90EF9017
:10D8C000DF90CF90BF90AF909F908F907F90089502
:10D8D0004F925F926F927F928F929F92AF92BF9280
:10D8E000CF92DF92EF92FF920F931F93CF93DF932C
:10D8F00000D01F92CDB7DEB70E9495FA4B015C01B4
:10D90000109109021F3FE9F10E9495FAC090F903B6
:10D91000D090FA03E090FB03F090FC03DC01CB0114
:10D920008C199D09AE09BF09B7FD2BC080919311D9
:10D93000909194118F5F8F70891719F1143060F5F1
:10D9400024E0129FF0011124ED57FD4F8081918159
:10D95000A281B38189839A83AB83BC83C12CD12CF0
:10D9600076018E010F5F1F4F2DE531E149E551E151
:10D9700065E571E181E591E10E9482B98FEF8093C5
:10D9800009020E9421D78091C803811191C1809121
:10D99000FE1582FD06C08CC180E090E0A8E4B2E4F0
:10D9A000D9CF8091040481110CC081E080930404DC
:10D9B0009091E70D89278093A80D1092E70D0F94A1
:10D9C0006C308091C4039091C503A091C603B091BF
:10D9D000C703A5019401281B390B4A0B5B0B57FFAA
:10D9E00005C08091C303882309F40DC2D501C40189
:10D9F0008C599F4FAF4FBF4F8093C4039093C50383
:10DA0000A093C603B093C7036091E00C062E000CF0
:10DA1000770B77FF03C07195619571099091E00CC8
:10DA200080910304981347C1633008F044C11092F9
:10DA3000E00C8091E00C80930304643028F4809122
:10DA4000A80D811187C097C08091B90D882309F472
:10DA50005AC0C090B50DD090B60DE090B70DF090C3
:10DA6000B80DC114D104E104F10409F43FC070E021
:10DA700080E090E00F94354020E030E040E85EE345
:10DA80000F9496402B013C01C501B4016C197D092E
:10DA90008E099F090F9435409B01AC01C301B2016F
:10DAA0000F94404820E030E04AE754E40F94964059
:10DAB0006B017C0120E030E040EA52E40F94A6497B
:10DAC00087FF0FC020E030E040EF51E4C701B6010E
:10DAD0000F94A64987FD0AC02AE030E040E050E0FC
:10DAE00009C024E630E040E050E004C021E030E02E
:10DAF00040E050E08092B50D9092B60DA092B70D27
:10DB0000B092B80D04C021E030E040E050E0A091B8
:10DB1000E00C0A2E000CBB0B0F94D24624E030E040
:10DB200040E050E00F94A8468091BF0D9091C00D49
:10DB3000A091C10DB091C20D820F931FA41FB51FFC
:10DB40008093BF0D9093C00DA093C10DB093C20DF3
:10DB50001092E00CD501C4018856954CAF4FBF4FD1
:10DB60008093FF0390930004A0930104B0930204F8
:10DB700081E080936E028091D5119091D6113FE69D
:10DB80008638930729F480915502882351F0C6C046
:10DB9000805D9140B9F480915502882309F49BC0BF
:10DBA000BDC08CE0809355028091FD039091FE03EF
:10DBB000009729F001979093FE038093FD0381E085
:10DBC00080936E020E94F484C0906C07D0906D0721
:10DBD000E0906E07F0906F0781110E940185D701D8
:10DBE000C6013AE0B695A795979587953A95D1F7EE
:10DBF000009751E0A507B10520F08FEF9FEFA0E05F
:10DC0000B0E09695879520916E02211105C0309164
:10DC1000C3033111F4C03FC0009739F04091FD03B8
:10DC20005091FE0348175907B0F58091C30388232C
:10DC300009F478C083E00E94D15281E08093FB1107
:10DC4000E091D511F091D61119951092C2038091EF
:10DC5000C303811174C01092A80D8091D5119091C9
:10DC6000D61186589F46F9F40E9495FADC01CB0143
:10DC700088199909AA09BB09C090FD03D090FE0339
:10DC8000E12CF12CC816D906EA06FB0620F4909385
:10DC9000FE038093FD038091D5119091D611865893
:10DCA0009F4609F49DC080913A0D811199C07EC0B4
:10DCB0001092040486CE633009F0BBCE8091E00C54
:10DCC00087FD02C081E001C08FEF880F880F80932D
:10DCD000E00C64E0AECE84E0809355028091D00DDC
:10DCE0008F5F8093D00D9091D10D981728F41092EA
:10DCF000D00D8CE08093550281E080936E02D501B7
:10DD0000C4018856954CAF4FBF4F8093FF0390934B
:10DD10000004A0930104B093020454CF8150809377
:10DD2000550250CF2230C0F0243028F02430A1F426
:10DD300010926E0211C081E080936E020DC08BEDD7
:10DD400091E10F94830E91E0811101C090E09093D6
:10DD5000C30381110BC07FCF87ED91E10F94562F44
:10DD600081E08093C2038093C30364CF8091D51177
:10DD70009091D61186589F4609F045C00E9495FAA9
:10DD8000DC01CB0188199909AA09BB09C090FD03E0
:10DD9000D090FE03E12CF12CC816D906EA06FB064A
:10DDA00090F59093FE038093FD032DC08091FF03B7
:10DDB00090910004A0910104B0910204881A990A7C
:10DDC000AA0ABB0AB7FE0E94584D8091C303811175
:10DDD0001AC080916E028130B1F410926E0213C0AD
:10DDE00058E9850E5AE3951EA11CB11C8092FF03D1
:10DDF00090920004A0920104B0920204E6CF009732
:10DE000009F418CF0BCF0F900F900F900F90DF9168
:10DE1000CF911F910F91FF90EF90DF90CF90BF9027
:10DE2000AF909F908F907F906F905F904F900895EC
:10DE3000CF92DF92EF92FF92CF93C82F0E9495FA74
:10DE40006B017C0124EA30E74DE75FE36091050256
:10DE50007091060280910702909108020F94304061
:10DE600087FD05C08AEF90E0A0E0B0E003C080E04D
:10DE700090E0DC01C80ED91EEA1EFB1EC092F90319
:10DE8000D092FA03E092FB03F092FC03C0930902E4
:10DE9000CF91FF90EF90DF90CF900895CF92DF92D7
:10DEA000EF92FF920F931F930E9495FA0091CA037D
:10DEB0001091CB032091CC033091CD036B017C01F9
:10DEC000C01AD10AE20AF30AF7FC13C02091C90371
:10DED00020952093C903DC01CB018A549C4FAF4F9E
:10DEE000BF4F8093CA039093CB03A093CC03B0930E
:10DEF000CD0381E09091C903911101C080E01F9191
:10DF00000F91FF90EF90DF90CF9008954F925F9226
:10DF10006F927F928F929F92AF92BF92CF92DF9239
:10DF2000EF92FF920F931F93CF93DF93CDB7DEB79E
:10DF30002C970FB6F894DEBF0FBECDBF1092B90D6F
:10DF40008091A80D1092A80D8823B1F020E040E048
:10DF500060E070E086E690E60E94A84C81E0809345
:10DF6000C00385ED9BE19093260F8093250F1092BF
:10DF7000280F1092270F0EC6209110023091110227
:10DF80004091BF0D5091C00DC901840F951F2436DB
:10DF9000310559F44730510514F0069723C04A3F24
:10DFA0005F4F0CF03AC306961DC0243631052CF4A1
:10DFB000853691050CF031C305C0843691050CF40B
:10DFC0002CC303C08A3091053CF0883EE3E09E07F5
:10DFD0002CF087EE93E002C08AE090E02817390722
:10DFE00031F411C08A30910584F78AE090E0909373
:10DFF0001102809310021092BF0D1092C00D10926A
:10E00000C10D1092C20D8091C203882309F419C278
:10E010006091370F7091380F072E000C880B990B09
:10E020000F94374011E02091330F3091340F40911D
:10E03000350F5091360F0F94A64918160CF010E0CA
:10E0400060914A0E70914B0E072E000C880B990BB5
:10E050000F9437402091460E3091470E4091480E64
:10E060005091490E0F94A64918160CF412601093A3
:10E07000F80320916511309166114091671150911C
:10E0800068116091551170915611809157119091BE
:10E0900058110F9446474B015C0120916911309152
:10E0A0006A1140916B1150916C11609159117091EE
:10E0B0005A1180915B1190915C110F9446476B014E
:10E0C0007C01209161113091621140916311509156
:10E0D000641160915111709152118091531190917E
:10E0E00054110F94464769837A838B839C838D8276
:10E0F0009E82AF82B886C986DA86EB86FC8620E0EF
:10E1000030E040E251E4C701B6010F94964020E0B0
:10E1100030E048EC52E40F9496404B015C0120E063
:10E1200030E0A901C701B6010F94304087FF05C058
:10E1300020E030E040EA50EC04C020E030E040EA6B
:10E1400050E4C501B4010F94464720E030E040E2BE
:10E1500051E40F9440480F94B2486B017C0197FF43
:10E160000AC0F094E094D094C094C11CD11CE11C6E
:10E17000F11C8DE201C080E280933B0DF0E1CF16EF
:10E18000F7E2DF06E104F10494F0C701B60120E1F3
:10E1900037E240E050E00F94A846CA01B9012AE0F6
:10E1A00030E040E050E00F94A846605D01C060E2BE
:10E1B00060933C0D28EEC21623E0D206E104F10480
:10E1C00094F0C701B60128EE33E040E050E00F9430
:10E1D000A846CA01B9012AE030E040E050E00F94BF
:10E1E000A846605D01C060E260933D0DC701B601C5
:10E1F00024E630E040E050E00F94A8466AE0862E26
:10E20000912CA12CB12CCA01B901A50194010F9444
:10E21000A846605D60933E0DC701B601A50194015B
:10E220000F94A846162F662381F08EE280933F0D4F
:10E23000CA01B901A50194010F94A846605D6093DD
:10E24000400D105D1093410D17C0CA01B901A50121
:10E2500094010F94A846662339F08EE280933F0D17
:10E26000605D6093400D05C080E28093400D809317
:10E270003F0D80E28093410D6BE37DE080EF93E002
:10E280000F94AB4ACE0101960E94D7CEBC018BEE13
:10E2900093E00F94AB4ACE0105960E94D7CEBC0105
:10E2A00086EE93E00F94AB4A1091C1031F7739F5C6
:10E2B0000E948937882319F1809134129091351288
:10E2C000A0913612B09137120097A105B105B9F0AF
:10E2D000BC01CD016D597F4F8F4F9F4F24E630E039
:10E2E00040E050E00F9486466091381270913912E8
:10E2F00080913A1290913B120F948646122F0E9401
:10E30000588B062F972E5C01F62E80910402811700
:10E3100009F43FC01093040238E4139FB0011124A4
:10E3200080E090E00F9435402AE037ED43E25CE373
:10E330000F9496400F94B9486093E503111103C000
:10E340001092E00326C0143630F0812F64E60F945B
:10E35000E946805D01C080E280933F0D1A3048F0AD
:10E360002AE0812F622F0F94E9460F94E946905DD1
:10E3700001C090E29093400D812F6AE00F94E9462E
:10E38000905D9093410D6FE37DE080EE93E00F94FC
:10E39000AB4A80910302F81609F453C000930302BC
:10E3A000602F792DC50120E13EE040E050E00F9460
:10E3B000864669017A014CE3442E512C612C712C64
:10E3C000602F792DC501A30192010F948646CA01E1
:10E3D000B901A30192010F94864644E6C416D10404
:10E3E000A8F47F936F93DF92CF9285ED9CE19F938A
:10E3F0008F9380ED93E09F938F930F94C83F0FB658
:10E40000F894DEBF0FBECDBF85E014C07F936F933D
:10E41000DF92CF928BEC9CE19F938F9380ED93E002
:10E420009F938F930F94C83F0FB6F894DEBF0FBE33
:10E43000CDBF86E09AEF899F802D1124805880936C
:10E44000CF030E944E6F182F81E00E94D15280911D
:10E450000F12843128F480911112883008F0E0C046
:10E460008091F803282F227081FF03C048E00CE060
:10E4700002C042E102E080910F1290E044977CF4E8
:10E4800080911112841758F02111D7C081E79CE1C7
:10E490007C0123E060E58BED91E10F94AF08809162
:10E4A0000F128431B8F480911112823098F0112348
:10E4B00009F4C6C080917007882309F4C1C08BE3BA
:10E4C0009CE17C0102E123E042E068E68BED91E112
:10E4D0000F94AF0880910F128C31B0F59091F80332
:10E4E0008090330F9090340FA090350FB090360F7E
:10E4F000C090370FD090380F843128F480911112DA
:10E50000883008F050C280910F12883008F42BC276
:10E5100080910F128C3108F42DC2C090460ED0901D
:10E52000470EE090480EF090490E80910F1288300F
:10E5300008F426C280910F128C3108F428C2809111
:10E540000F128C3108F429C20E948937882349F0C0
:10E5500080910F12843328F4809111128A3208F0CE
:10E5600072C080910F12853328F48091111281338B
:10E5700008F091C080910F12843328F48091111219
:10E58000823308F08FC080910F128033D8F48091CD
:10E5900011128832B8F08091E003882361F040EED8
:10E5A00053E060E387E30E94125665E270E080E08A
:10E5B00090E00E94E45240ED53E060E38091CF038D
:10E5C0000E94125680910F12883298F48091111295
:10E5D0008D3178F02BE040E86DE180E00F94010987
:10E5E00080910F12873228F4809111128F3108F038
:10E5F00063C080910F12833328F4809111128B3203
:10E6000008F016C180910F12813408F0C3C28091C6
:10E610001112863308F030C1BDC284E690E0D5CC3B
:10E620008BE9E82E8CE1F82E0CE024E048E060E075
:10E630008BED91E10F94AF0813CF87E79CE128CFD2
:10E6400085E09CE13ECF07E028E04AE26AE28BEDFC
:10E6500091E10F943B0905E022E04CE262E38BED8F
:10E6600091E10F943B0924E04AE061E38AE20F94D0
:10E6700001096091DD117091DE1182E38093F71141
:10E680008BE28093F81127EF31E142E38BED91E1CA
:10E690000E94DE9466CF24E04AE461E386E30F94AF
:10E6A000010968CF02E02091E50342E367E38BEDC7
:10E6B00091E10F943B0967CF83E08093121206E249
:10E6C0000093131268E570E080E090E00E94E4524D
:10E6D0008BE08093121200931312112329F08BEE1A
:10E6E00093E00E94CF5424C08091AE0480FD18C0F6
:10E6F0003BEEE32E33E0F32EF70161917F016623B9
:10E70000B9F06F3234F4062E000C770B880B990B9E
:10E7100004C06FE370E080E090E00E94E452ECCF30
:10E720008091DA0480FDDBCF84EE9CE10E94F353FC
:10E7300088E28093121206E20093131269E570E0FA
:10E7400080E090E00E94E45280E3809312120093F4
:10E750001312112329F086EE93E00E94CF5426C0B5
:10E760008091AE04869580FD18C026EEE22E23E04F
:10E77000F22EF70161917F016623C1F06F3234F40C
:10E78000062E000C770B880B990B04C06FE370E02A
:10E7900080E090E00E94E452ECCF8091DA0486950C
:10E7A00080FDD9CF84EE9CE10E94F3538DE48093E9
:10E7B000121206E2009313126AE570E080E090E026
:10E7C0000E94E45285E580931212009313121123E4
:10E7D00029F080EF93E00E94CF540BCF8091AE04DC
:10E7E0008695869580FD19C090EFE92E93E0F92E6D
:10E7F000F70161917F01662309F4FBCE6F3234F497
:10E80000062E000C770B880B990B04C06FE370E0A9
:10E8100080E090E00E94E452EBCF8091DA0486958C
:10E82000869580FDD6CF81EE9CE10E94F353E1CE28
:10E8300083E00E94D15283E08093121283E380939D
:10E84000131266E070E080E090E00E94E45281E004
:10E850000E94D15280911002909111020E9428D101
:10E86000AC0163E38CE00E94125665E270E080E048
:10E8700090E00E94E452C6CE109212128EE3809372
:10E88000131282EE9CE00E946050082F863178F4CB
:10E8900082EE9CE00E94CF54053109F47BC160E216
:10E8A00070E080E090E00E94E4520F5FF5CFE090CE
:10E8B000E10C8E2D90E09C012E51334F7901C9015E
:10E8C0000E946050082F60E870E0C7010E94F75373
:10E8D000053130F56EE270E080E090E00E94E45295
:10E8E0000431F1F06EE270E080E090E00E94E452CA
:10E8F0000331B1F0202F30E02E5F3F4F4AEF42034B
:10E90000B001439F700D112460587F4F82EE9CE050
:10E910000E94F75360E270E080E090E00E94E452D1
:10E920008091CE03181709F435C11093CE0382EEFF
:10E930009CE00E9460509091E10C981788F481E06F
:10E94000890F21E0280FE82FF0E0EE51F34F90817E
:10E95000907C903811F4822FF4CF8093E10C1AC18F
:10E960001092E10C17C111112FC08091081681116E
:10E97000CFCD2AC080911112843108F058C0CDCD7E
:10E98000111184C0809103168111D4CD7FC0809174
:10E990001112843108F0B1C0D2CD809111128431AE
:10E9A00008F0DAC0D1CD90FD0CC085ED9BE17C0173
:10E9B0000CE022E048E060E28BED91E10F94AF08BB
:10E9C000A2CD8DEE9BE1F3CFB601DD0C880B990B48
:10E9D0000F94374020E030E040E05FE30F9446477B
:10E9E0000F94B248CB010E9428D1FC018081803273
:10E9F000E1F48181803211F092E001C091E043E0C6
:10EA000050E0491B51094E0F5F1F892F880F980F47
:10EA1000892F819567E0895D0E94125669E070E058
:10EA200080E090E00E94E45273CD93E0E8CF20E0D4
:10EA300030E040E05FE3C501B4010F9446470F9416
:10EA4000B248CB010E9428D1FC0180818032E1F4E0
:10EA50008181803211F092E001C091E043E050E00A
:10EA6000491B51094E0F5F1F892F880F980F892F5F
:10EA700081956CE1895D0E94125669E070E080E04A
:10EA800090E00E94E45249CD93E0E8CF60914A0EB5
:10EA900070914B0E072E000C880B990B0F9437408A
:10EAA00020E030E040E05FE30F9446470F94B24827
:10EAB000CB010E9428D1FC0180818032E1F4818168
:10EAC000803211F092E001C091E043E050E0491B38
:10EAD00051094E0F5F1F892F880F980F892F81953D
:10EAE00067E0865A0E94125669E070E080E090E08C
:10EAF0000E94E4521FCD93E0E8CF20E030E040E0F8
:10EB00005FE3C701B6010F9446470F94B248CB01AB
:10EB10000E9428D1FC0180818032E1F48181803221
:10EB200011F092E001C091E043E050E0491B51092F
:10EB30004E0F5F1F892F880F980F892F81956CE1E9
:10EB4000865A0E94125669E070E080E090E00E94D0
:10EB5000E452F5CC93E0E8CF80917007882309F464
:10EB6000F3CCF4E68F9FC001112481589F4F6FEFC3
:10EB700070E00F941747CB010E9428D1AC016CE1E3
:10EB800087E60E94125665E270E080E090E00E9405
:10EB9000E452DACC2C960FB6F894DEBF0FBECDBF90
:10EBA000DF91CF911F910F91FF90EF90DF90CF9069
:10EBB000BF90AF909F908F907F906F905F904F909D
:10EBC00008950F930FB70F9300916E000F930B7F73
:10EBD00000936E0000916F000D7F00936F000F9304
:10EBE0000BB70F930CB70F921F922F933F934F9336
:10EBF0005F936F937F938F939F93AF93BF93EF93A5
:10EC0000FF9311240E945D76FF91EF91BF91AF9128
:10EC10009F918F917F916F915F914F913F912F9134
:10EC20001F900F900CBF0F910BBF0F910260F894D3
:10EC300000936F000F9100936E000F910FBF0F9123
:10EC400018958091D90480FF03C089988FEF02C086
:10EC5000899A81E0809364048091D904869580FF2D
:10EC600003C08F988FEF02C08F9A81E08093650474
:10EC70008091D9048695869580FF08C080910B010C
:10EC800080958270809309018FEF06C080910B01FF
:10EC900082708093090181E0809366048091D90499
:10ECA00086958695869580FF03C0169A8FEF02C0E1
:10ECB000169881E08093670408952F923F924F92B7
:10ECC0005F926F927F928F929F92AF92BF92CF92FC
:10ECD000DF92EF92FF920F931F93CF93DF9300D0B9
:10ECE0001F92CDB7DEB78FEF9FEF9093890080938F
:10ECF00088000AE00983212C312C78948091AA04A1
:10ED00009091AB04A091AC04B091AD04892B8A2BF7
:10ED10008B2B71F08091AA049091AB04A091AC046C
:10ED2000B091AD04892B8A2B8B2B09F063C5DAC116
:10ED30008091B9158823D1F01092B9158091B7153B
:10ED40009091B815892B91F01092B8151092B715C3
:10ED5000109263049091931180919411981731F05F
:10ED6000809194118F5F8F70809394118091B7156B
:10ED70009091B815892B71F2C090A604D090A70489
:10ED8000E090A804F090A9044091A2045091A3043B
:10ED90006091A4047091A5040091940410E020E017
:10EDA00030E0DB01CA018C199D09AE09BF090817C3
:10EDB00019072A073B0710F4D901C801E82F8C0D69
:10EDC0009D1DAE1DBF1D8093A6049093A704A09324
:10EDD000A804B093A9041B821A82F1E0C0906C04CD
:10EDE000D0906D04E0906E04F0906F0480917C04EC
:10EDF00090917D04A0917E04B0917F04C80ED91E2D
:10EE0000EA1EFB1EC0927C04D0927D04E0927E0438
:10EE1000F0927F04F7FC31C080916404082E000C4E
:10EE2000990BAA0BBB0B4091C6155091C715609169
:10EE3000C8157091C915840F951FA61FB71F809321
:10EE4000C6159093C715A093C815B093C9158091A6
:10EE5000680490916904A0916A04B0916B04A701C1
:10EE60009601281B390B4A0B5B0B20937C043093D3
:10EE70007D0440937E0450937F04009170041091B0
:10EE800071042091720430917304809180049091F8
:10EE90008104A0918204B0918304080F191F2A1FD6
:10EEA0003B1F0093800410938104209382043093CD
:10EEB000830437FD31C080916504082E000C990B46
:10EEC000AA0BBB0B4091CA155091CB156091CC1584
:10EED0007091CD15840F951FA61FB71F8093CA157B
:10EEE0009093CB15A093CC15B093CD158091680469
:10EEF00090916904A0916A04B0916B04B901A801D2
:10EF0000481B590B6A0B7B0B409380045093810480
:10EF1000609382047093830440917404509175044B
:10EF200060917604709177048091840490918504B7
:10EF3000A0918604B0918704480F591F6A1F7B1F58
:10EF400040938404509385046093860470938704EF
:10EF500077FD31C080916604082E000C990BAA0B36
:10EF6000BB0B8090CE159090CF15A090D015B0908F
:10EF7000D115880D991DAA1DBB1D8093CE159093A8
:10EF8000CF15A093D015B093D115809168049091BE
:10EF90006904A0916A04B0916B042A013B01481AEC
:10EFA000590A6A0A7B0A409284045092850460924E
:10EFB0008604709287048090780490907904A090E1
:10EFC0007A04B0907B048091880490918904A09188
:10EFD0008A04B0918B04880D991DAA1DBB1D8093D6
:10EFE000880490938904A0938A04B0938B04B7FD9E
:10EFF00031C080906704082C000C9908AA08BB084F
:10F000004090D2155090D3156090D4157090D515BE
:10F01000840C951CA61CB71C8092D2159092D31517
:10F02000A092D415B092D515809068049090690490
:10F03000A0906A04B0906B042C013D014818590857
:10F040006A087B08409288045092890460928A047E
:10F0500070928B04F1110CC0A0908400B0908500D8
:10F060006A807B80A618B708F2E0AF16B104A0F35F
:10F07000F7FE889A37FF8E9A77FD06C0F0910B0154
:10F08000F095F870F0930901B7FF149A409084004E
:10F09000509085005B824A82A0908400B0908500E9
:10F0A0006A807B80A618B708F2E0AF16B104A0F31F
:10F0B000F7FE889837FF8E9877FD05C020910B01E9
:10F0C000287020930901B7FF1498EE2331F0409087
:10F0D0008400509085005B824A82E150F0E009F0A4
:10F0E0007DCE18CEE091B715F091B815309709F4A0
:10F0F00007C58091A6049091A704A091A804B0919F
:10F10000A9044091A2045091A3046091A4047091B9
:10F11000A50484179507A607B707D0F01092B81575
:10F120001092B715109263049091931180919411ED
:10F13000981709F4E5C4809194118F5F8F708093C4
:10F140009411F0EDCF2EF7E0DF2EE12CF12C69C108
:10F1500040919E0450919F046091A0047091A1047D
:10F16000481759076A077B0708F470C040919A0452
:10F1700050919B0460919C0470919D0481A992A977
:10F18000A3A9B4A95524499F612C5A9F90016A9F55
:10F19000300D699F200D311D4A9F600C211D351DCA
:10F1A000599F600C211D351D689F600C211D351D68
:10F1B000589F610C251D351D6694251D351DB49F76
:10F1C000200D311DB59F300D112482AD93ADA4AD3E
:10F1D000B5AD820F931FA11DB11D8093960490932E
:10F1E0009704A0939804B093990406A917A920AD99
:10F1F00031AD081719072A073B0740F4009396041E
:10F200001093970420939804309399048090960467
:10F2100090909704A0909804B09099040090950461
:10F2200004C0880C991CAA1CBB1C0A94D2F786E067
:10F2300098E221E0FC01C590D590E590F490C814C7
:10F24000D904EA04FB0408F425C32FC340919004B9
:10F25000509191046091920470919304481759075A
:10F260006A077B0708F06CC040918C0450918D04B4
:10F2700060918E0470918F0481A992A9A3A9B4A969
:10F280004424499F512C5A9F90016A9F300D699FD9
:10F29000200D311D4A9F500C211D341D599F500CCB
:10F2A000211D341D689F500C211D341D589F510C89
:10F2B000241D341D5694241D341DB49F200D311D72
:10F2C000B59F300D1124C901A0E0B0E080909604F4
:10F2D00090909704A0909804B0909904FE96881599
:10F2E0009905AA05BB0580F4008111812281338133
:10F2F000881A990AAA0ABB0A80169106A206B306C2
:10F3000038F44801590104C080809180A280B38004
:10F310000090950404C0880C991CAA1CBB1C0A947C
:10F32000D2F786E098E221E0FC01C590D590E59007
:10F33000F490C814D904EA04FB0408F41EC328C3DB
:10F3400080910B0290910C02A0910D02B0910E02DF
:10F35000B7FF5FC086A997A9A0ADB1AD0090950495
:10F3600004C0880F991FAA1FBB1F0A94D2F726E07A
:10F3700038E241E0F901C590D590E590F490C816C7
:10F38000D906EA06FB0658F4B695A7959795879592
:10F39000440F2C5F3F4FF8E222323F0759F740936A
:10F3A000940480329105A105B10508F47CC38097CF
:10F3B000A109B109811508E09007A105B10508F47C
:10F3C0004FC314E0919F900111242A5F3B4DF90136
:10F3D000329645915491EE27859FB001849F610D2F
:10F3E0007E1F06946E1F7E1F1124CB01A0E0B0E0AB
:10F3F000F9014591549160E070E0481B590B6A0B8C
:10F400007B0B40930B0250930C0260930D027093A0
:10F410000E02C0900B02D0900C02E0900D02F09012
:10F420000E028091B7159091B815892B09F0DAC1B9
:10F430000E9435839093B8158093B715892B09F4F2
:10F44000D1C1E091B715F091B815808183FF44C018
:10F45000858D968DA78DB0A1418D528D638D748D54
:10F46000058916892789308D0093C6151093C71515
:10F470002093C8153093C9154093CA155093CB15E6
:10F480006093CC157093CD158093CE159093CF15C6
:10F49000A093D015B093D11581A192A1A3A1B4A13D
:10F4A0008093D2159093D315A093D415B093D5150E
:10F4B0001092B8151092B7151092630490919311A1
:10F4C00080919411981709F4B3CF809194118F5FB4
:10F4D0008F7080939411ACCFDF01A55BBF4F8D91EE
:10F4E0009D910D90BC91A02D80931A0F90931B0FAE
:10F4F000A0931C0FB0931D0F85889688A788B08CA9
:10F5000081E081149104A104B10409F480E0C18C6C
:10F51000D28CE38CF48CC114D104E104F10409F021
:10F520008260058D168D278D30A1011511052105ED
:10F53000310509F084608093630410928C0410926A
:10F540008D0410928E0410928F0410929A041092DF
:10F550009B0410929C0410929D0446A957A960AD8B
:10F5600071AD80E042389BE159076105710560F497
:10F57000440F551F661F771F4238ABE15A076105DC
:10F58000710580F78F5FEECF80939504482E512C44
:10F590005B824A8245A156A167A170A5082E04C0CE
:10F5A000440F551F661F771F0A94D2F74093A20499
:10F5B0005093A3046093A4047093A5044424552499
:10F5C0003201441A550A660A770A40927C04509226
:10F5D0007D0460927E0470927F0440928004509279
:10F5E0008104609282047092830440928404509259
:10F5F0008504609286047092870440928804509239
:10F60000890460928A0470928B0441A052A063A086
:10F6100074A0440C551C661C771C880C991CAA1CF1
:10F62000BB1C80926C0490926D04A0926E04B09208
:10F630006F04CC0CDD1CEE1CFF1CC0927004D09239
:10F640007104E0927204F0927304000F111F221FE4
:10F65000331F009374041093750420937604309341
:10F660007704409278045092790460927A04709200
:10F670007B04440F551F661F771F40936804509307
:10F68000690460936A0470936B041092A60410924C
:10F69000A7041092A8041092A90441A552A563A53D
:10F6A00074A5082E04C0440F551F661F771F0A94C7
:10F6B000D2F740939E0450939F046093A0047093EC
:10F6C000A10445A556A567A570A93A014B0104C040
:10F6D000660C771C881C991C8A95D2F7609290045E
:10F6E00070929104809292049092930485A99091D3
:10F6F000D904891721F08093D9040E942176809142
:10F70000D80481110E94C98A88248A94982C5401B3
:10F7100080920B0290920C02A0920D02B0920E0207
:10F72000E091B715F091B81582AD93ADA4ADB5AD2C
:10F730008093960490939704A0939804B0939904AF
:10F740000A8004C0880F991FAA1FBB1F0A94D2F712
:10F7500026E038E241E0F901C590D590E590F490BB
:10F76000C816D906EA06FB0670F4B695A7959795D4
:10F770008795440F2C5F3F4F62E2462E68E2562E7B
:10F780004216530641F74093940480329105A10537
:10F79000B10508F4B0C18097A109B109811508E04D
:10F7A0009007A105B10508F483C114E0919F900171
:10F7B00011242A5F3B4DF901329645915491EE2771
:10F7C000859FB001849F610D7E1F06946E1F7E1F72
:10F7D0001124F901C590D490E12CF12CC61AD70A56
:10F7E000E108F108C092AA04D092AB04E092AC0404
:10F7F000F092AD048091AA049091AB04A091AC0466
:10F80000B091AD048F3F2FEF9207A105B10528F00D
:10F810004FEF5FEF60E070E002C0AC01BD01841B00
:10F82000950BA60BB70B8093AA049093AB04A093FF
:10F83000AC04B093AD04F89480918400909185005D
:10F840004096098101500983002339F0240E351EAA
:10F850002816390608F451CA01C01C0130928900EB
:10F860002092880078940F900F900F900F90DF9166
:10F87000CF911F910F91FF90EF90DF90CF90BF90AD
:10F88000AF909F908F907F906F905F904F903F9040
:10F890002F900895B694A79497948794220F049676
:10F8A00018E28232910709F0C5CC2093940420E23B
:10F8B00082169104A104B10408F459C000E2801A30
:10F8C0009108A108B108811418E09106A104B104BF
:10F8D000F8F024E0929EC00111248A5F9B4DFC0148
:10F8E000329625913491F82DEE27F39FD001F29FA7
:10F8F000A10DBE1F0694AE1FBE1F1124FC01C590B2
:10F90000D490E12CF12CCA1ADB0AE108F10822C0DC
:10F91000D501C401B695A79597958795FC01EC7F15
:10F92000CF018A5F9F4DFC01C590D490FC013296B7
:10F9300025913491E82DE770E29FC001E39F900D7F
:10F940001124E3E096958795EA95E1F7C81AD90A5C
:10F95000E12CF12C4C0D5D1D6E1D7F1D40939A0412
:10F9600050939B0460939C0470939D045ACDA0E235
:10F970008A2E912CA12CB12CA1CFB694A794979448
:10F980008794220F049638E28232930709F0CCCC98
:10F990002093940480E288169104A104B10408F431
:10F9A00059C000E2801A9108A108B108811418E03A
:10F9B0009106A104B104F8F024E0929EC001112444
:10F9C0008A5F9B4DFC01329625913491F82DEE27EC
:10F9D000F39FD001F29FA10DBE1F0694AE1FBE1F64
:10F9E0001124FC01C590D490E12CF12CCA1ADB0A39
:10F9F000E108F10822C0D501C401B695A7959795F5
:10FA00008795FC01EC7FCF018A5F9F4DFC01C5907B
:10FA1000D490FC01329625913491E82DE770E29F55
:10FA2000C001E39F900D112423E0969587952A95B8
:10FA3000E1F7C81AD90AE12CF12C4C0D5D1D6E1DA1
:10FA40007F1D40938C0450938D0460938E047093BB
:10FA50008F04E7CCE0E28E2E912CA12CB12CA1CF0B
:10FA6000AC01BD017695679557954795FA01EC7FF6
:10FA70009F012A5F3F4DF90145915491F90132965A
:10FA8000659174918770869F9001879F300D112436
:10FA9000C90113E0969587951A95E1F7481B590B14
:10FAA00060E070E0AECC80E290E0A0E0B0E07FCC1F
:10FAB000AC01BD017695679557954795FA01EC7FA6
:10FAC0009F012A5F3F4DF901C590D490F90132960C
:10FAD000459154918770849F9001859F300D11242A
:10FAE000C90103E0969587950A95E1F7C81AD90AE6
:10FAF000E12CF12C77CE80E290E0A0E0B0E04BCE9C
:10FB000080EDC82E87E0D82EE12CF12C91CCAF925D
:10FB1000BF92CF92DF92EF92FF920F931F93CF93FA
:10FB2000C82F811102C00E944EF58FEE9FE10E9406
:10FB300046F489EE9FE10E9446F48AE00E94413833
:10FB4000C11102C00E944EF58CEC9FE10E9446F468
:10FB50008AE00E944138C11114C040E069EB7FE1A6
:10FB600080E00F94C8148091510E882321F08AE020
:10FB70000E94413804C08EEA9FE10E9446F40E9430
:10FB80004EF56091510E70E085EA9FE10E942AF5E2
:10FB900040914D0E50914E0E60914F0E7091500E4F
:10FBA00082EA9FE10E9419F58AE00E94413841E013
:10FBB00062E97FE18C2F0F94C8146FEF81E08C27EE
:10FBC0000F94B02441E065E77FE18C2F0F94C814B7
:10FBD000C11102C00E944EF54091990C50919A0CAF
:10FBE00060919B0C70919C0C8CE69FE10E9419F532
:10FBF00040919D0C50919E0C60919F0C7091A00CB7
:10FC000088EA9AE30E9419F54091A10C5091A20C48
:10FC10006091A30C7091A40C8DE49EE10E9419F5F3
:10FC20004091A50C5091A60C6091A70C7091A80C66
:10FC300083E29CE00E9419F58AE00E94413841E08D
:10FC40006BE47FE18C2F0F94C814C11102C00E9495
:10FC50004EF56091750C7091760C8091770C9091B7
:10FC6000780C0F943540AB01BC0182E49FE10E9407
:10FC700019F56091790C70917A0C80917B0C9091C0
:10FC80007C0C0F943540AB01BC0188EA9AE30E94DA
:10FC900019F560917D0C70917E0C80917F0C909194
:10FCA000800C0F943540AB01BC018DE49EE10E94B5
:10FCB00019F56091810C7091820C8091830C909168
:10FCC000840C0F943540AB01BC0183E29CE00E94A0
:10FCD00019F58AE00E94413841E069EF7EE18C2FFE
:10FCE0000F94C814C11102C00E944EF54091A90C96
:10FCF0005091AA0C6091AB0C7091AC0C80EF9EE11E
:10FD00000E9419F54091AD0C5091AE0C6091AF0C72
:10FD10007091B00C89EE9CE10E9419F54091B10CF4
:10FD20005091B20C6091B30C7091B40C8DEE9EE1C9
:10FD30000E9419F58AE00E94413841E069E97EE1BC
:10FD40008C2F0F94C814C11102C00E944EF560910F
:10FD5000850C7091860C8091870C9091880C0F9483
:10FD60003540AB01BC0180E99EE10E9419F540914C
:10FD7000B50C5091B60C6091B70C7091B80C8CE634
:10FD80009BE00E9419F54091B90C5091BA0C60911A
:10FD9000BB0C7091BC0C8DEE9EE10E9419F5409158
:10FDA00054075091550760915607709157078DE899
:10FDB0009EE10E9419F58AE00E94413841E060E826
:10FDC0007EE18C2F0F94C814C11102C00E944EF521
:10FDD00040915E0E50915F0E6091600E7091610EC9
:10FDE00087E79EE10E9419F54091620E5091630EE3
:10FDF0006091640E7091650E88EA9AE30E9419F58D
:10FE00004091660E5091670E6091680E7091690E78
:10FE10008DE49EE10E9419F58AE00E94413841E09C
:10FE200064E67EE18C2F0F94C814C11102C00E94B9
:10FE30004EF56091410E70E08BE59EE10E942AF53F
:10FE400040913D0E50913E0E60913F0E7091400EDC
:10FE50008DE49EE10E9419F58AE00E9441380E94DB
:10FE6000F5F3882309F44EC08FE3C82E84E0D82E22
:10FE700000E010E05601E12CF12CC11102C00E94FB
:10FE80004EF5B70180E59EE10E942AF5B8018DE8A4
:10FE90009EE10E942AF58DE49EE10E9446F4F50160
:10FEA000608171818281938145E00E94D1388AE02E
:10FEB0000E944138FFEFEF1AFF0A8CE0A80EB11C38
:10FEC000E3E0EE16F104C9F60F5F1F4FF4E0CF0E2A
:10FED000D11C0330110571F6C11102C00E944EF50C
:10FEE00085E49EE10E9446F460913B0470913C04DD
:10FEF00080913D0490913E0445E00E94D1388AE013
:10FF00000E94413841E069E27EE18C2F0F94C814D1
:10FF10000FE214E0E12CF12CC11102C00E944EF559
:10FF2000B70180E29EE10E942AF5F80160817181AB
:10FF30008DE19EE10E940CF5F8016281738186E9F2
:10FF40009EE10E940CF5F801648175818AE19EE1D1
:10FF50000E940CF58AE00E944138FFEFEF1AFF0A79
:10FF60000A5F1F4F82E0E816F104B1F641E06CE051
:10FF70007EE18C2F0F94C814C11102C00E944EF56F
:10FF800040913A0F50913B0F60913C0F70913D0FA3
:10FF900083E09EE10E9419F52CEA35EC47E25EE32E
:10FFA00060913E0F70913F0F8091400F9091410FF3
:10FFB0000F944048AB01BC0188E59EE10E9419F511
:10FFC0002CEA35EC47E25EE36091420F7091430FFB
:10FFD0008091440F9091450F0F949640AB01BC0166
:10FFE00082EA9FE10E9419F58AE00E94413841E0CF
:10FFF0006EEE7DE18C2F0F94C814C11102C00E94D7
:020000021000EC
:100000004EF560912E0470E085EE9DE10E942AF588
:100010008AE00E94413841E06FEB7DE18C2F0F9424
:10002000C814C11102C00E944EF540910E045091B7
:100030000F04609110047091110486EB9DE10E9401
:1000400019F5409122045091230460912404709189
:10005000250483EB9DE10E9419F520E030E040E7A4
:1000600052E46091120470911304809114049091F1
:1000700015040F949640AB01BC018AE19EE10E94F9
:1000800019F540911604509117046091180470916D
:1000900019048DE49EE10E9419F58AE00E9441381E
:1000A00041E065E97DE18C2F0F94C814C11102C0B5
:1000B0000E944EF540911A0450911B0460911C045B
:1000C00070911D048CE89DE10E9419F54091260471
:1000D00050912704609128047091290483EB9DE1DD
:1000E0000E9419F520E030E040E752E460911E04E0
:1000F00070911F0480912004909121040F949640E8
:10010000AB01BC018AE19EE10E9419F58AE00E94E0
:10011000413841E06FE37DE18C2F0F94C814C11189
:1001200002C00E944EF560910D0470E086E39DE1EF
:100130000E942AF58AE00E94413841E068E17DE1B1
:100140008C2F0F94C814C11102C00E944EF58CEE82
:100150009CE10E9446F44091090450910A04609188
:100160000B0470910C048DE397E30E9419F5409104
:10017000050450910604609107047091080485E11C
:100180009DE10E9419F58AE00E94413841E06DEF3F
:100190007CE18C2F0F94C814C11102C00E944EF54F
:1001A00060910A0270E084EF9CE10E942AF58AE0E7
:1001B000CF911F910F91FF90EF90DF90CF90BF9064
:1001C000AF900C944138CF92DF92EF92FF928091E2
:1001D000510E882371F1C0904D0ED0904E0EE090DC
:1001E0004F0EF090500E20E030E0A901C701B6019B
:1001F0000F9430408823E9F020E030E040E05FE3F6
:10020000C701B6010F9496409B01AC010F94964034
:100210002BED3FE049E450E40F9496409B01AC0184
:1002200060E070E080E89FE30F9440486B017C0140
:1002300006C0C12CD12C80E8E82E8FE3F82EC092A6
:10024000B704D092B804E092B904F092BA04609175
:10025000160270911702072E000C880B990B0F9451
:1002600037402AE037ED43E25CE30F949640A70164
:1002700096010F9496406093240270932502809318
:10028000260290932702FF90EF90DF90CF90089581
:10029000CF93C82FCB01009711F00E9446F482EE55
:1002A00092E40E9446F4C11103C086E298E202C0C3
:1002B0008BE298E20E9446F48AE0CF910C94413898
:1002C0004F925F926F927F928F929F92AF92BF9266
:1002D000CF92DF92EF92FF920F931F93CF93DF9312
:1002E000CDB7DEB768970FB6F894DEBF0FBECDBFAF
:1002F0008C015B015A834983DC01D6966D917D9117
:100300008D919C91D9970F9435406B017C01F5013B
:1003100020813181428153810F9496400F9424486B
:100320000F94B94869877A878B879C87A981BA819E
:100330002D913D914D915C91C701B6010F9496406E
:100340000F9424480F94B9486D877E878F87988BC8
:1003500029853A854B855C8528373105410551054E
:1003600040F488E790E0A0E0B0E089879A87AB8707
:10037000BC872D853E854F85588928373105410535
:10038000510540F488E790E0A0E0B0E08D879E87BB
:10039000AF87B88BF801EE5BFF4F2081318142813E
:1003A000538129833A834B835C83CA01B9010F943B
:1003B00037402B013C0169857A858B859C850F949C
:1003C0003540698B7A8B8B8B9C8B20E030E0A901C8
:1003D000C301B2010F943040882329F1A70196018F
:1003E000C701B6010F9496404B015C0129893A89F7
:1003F0004B895C89CA01B9010F9496409B01AC01FD
:10040000C501B4010F9445474B015C01A301920162
:10041000C301B2010F9446479B01AC01C501B40171
:100420000F94404803C060E070E0CB010F94244873
:100430000F94B9486D837E838F83988769817A8111
:100440008B819C8190958095709561957F4F8F4FA2
:100450009F4F0F9437404B015C016D857E858F85E2
:1004600098890F94354069837A838B839C8320E03D
:1004700030E0A901C501B4010F943040882349F14F
:1004800029813A814B815C81CA01B9010F94964060
:100490006D8B7E8B8F8B988FA7019601C701B6015C
:1004A0000F9496409B01AC016D897E898F89988D50
:1004B0000F9445476B017C01A5019401C501B4016E
:1004C0000F9446479B01AC01C701B6010F94404809
:1004D00003C060E070E0CB010F94E848D801959626
:1004E0008D909D90AD90BC909897750164012D8181
:1004F0003E814F815885C21AD30AE40AF50A0F9447
:10050000B948C61AD70AE80AF90AF7FE75C020E00A
:1005100030E0A901C301B2010F943040882309F4EF
:1005200043C0C501B4010F9435406B017C01A301A8
:100530009201C301B2010F9446479B01AC01C70170
:10054000B6010F9496406B017C0129893A894B8949
:100550005C89CA01B9010F9496409B01AC01C701A7
:10056000B6010F9445476B017C0129813A814B818B
:100570005C81CA01B9010F9496409B01AC01C7018F
:10058000B6010F9446476B017C0120E030E040E863
:1005900050E4C301B2010F9496409B01AC01C70126
:1005A000B6010F94404803C060E070E0CB010F94A7
:1005B00024487B018D83998320E030E0A9010F94CA
:1005C000A649181624F0E12CF12C1D821982B701DE
:1005D0008D8199810F94B9486D837E838F8398872D
:1005E00086169706A806B90620F48D829E82AF82F1
:1005F000B886C12CD12C76018D819E81AF81B885C2
:10060000F80181A792A7A3A7B4A7C80ED91EEA1E16
:10061000FB1EC5A6D6A6E7A6F0AA29853A854B8576
:100620005C8522AF33AF44AF55AFFE962D853E8536
:100630004F855889208331834283538368960FB650
:10064000F894DEBF0FBECDBFDF91CF911F910F9108
:10065000FF90EF90DF90CF90BF90AF909F908F90E2
:100660007F906F905F904F900895CF93DF9380912C
:10067000931190919411891B8F7009F445C090914A
:100680009011992351F0833030F48FEF890F19F0D6
:10069000809390113BC010929011E09194118FE4DF
:1006A000E89FF0011124EE57F84F808180FD2EC0A5
:1006B00080916C0790916D07A0916E07B0916F07C4
:1006C000EF01C95BDF4F488159816A817B81841BBF
:1006D000950BA60BB70B80936C0790936D07A093B7
:1006E0006E07B0936F07809194118F5F8F70809326
:1006F0009111909194118091921198130AC0809158
:1007000091118093921105C00E948AEB80E090E0E5
:1007100001C0CF01DF91CF9108952F923F924F9268
:100720005F926F927F928F929F92AF92BF92CF9281
:10073000DF92EF92FF920F931F93CF93DF93CDB78A
:10074000DEB762970FB6F894DEBF0FBECDBF788BD1
:100750006F87DC018D909D90AD90BC90139714969F
:100760002D913D914D915C9117972D833E834F8341
:10077000588720E030E040E251E4C501B4010F9415
:10078000454726ED39EB42EF5BE30F9496400F941B
:10079000B248161614F461E002C067FD60E0E62E70
:1007A000660FFF08F701EE0FFF1FEE0FFF1FEB5D57
:1007B000FD4E408051806280738087010F5F1F4F24
:1007C00020E030E040E251E46D817E818F819885A8
:1007D0000F94454725E338E74EE05CE30F949640DD
:1007E0000F94B248161614F461E002C067FD60E091
:1007F000E62F660FFF0BFA8BE98BEE0FFF1FEE0F54
:10080000FF1FEB5DFD4E20813181428153812983A1
:100810003A834B835C8329883A883FEF231A330A53
:10082000B701660F771FAB014E0D5F1D5A874987D1
:10083000FA0189899A89E80FF91FEE0FFF1FEE0F61
:10084000FF1FE15CFB4FC080D180E280F380F801A4
:10085000EE0FFF1FEE0FFF1FEB5DFD4EA301920198
:1008600060817181828193810F9445476B877C877A
:100870008D879E87A3019201C501B4010F9445475E
:100880002B013C01C801880F991F080F191FA98966
:10089000BA89A00FB11FAA0FBB1FAA0FBB1FA15C73
:1008A000BB4FA70196016D917D918D919C910F9405
:1008B00045472B853C854D855E850F944048A301B7
:1008C00092010F949640A70196010F9446476B0141
:1008D0007C01E985FA85E20DF31DEE0FFF1FEE0F97
:1008E000FF1FE15CFB4F80809180A280B380020DEE
:1008F000131DF801EE0FFF1FEE0FFF1FE15CFB4F12
:10090000A501940160817181828193810F94454793
:100910002B853C854D855E850F944048A30192014F
:100920000F949640A50194010F944647A7019601A4
:100930000F9445474B015C01F101EE0FFF1FEE0FD5
:10094000FF1FEB5DFD4E29813A814B815C81608107
:100950007181828193810F9445479B01AC01C50150
:10096000B4010F9440484B015C0129813A814B81CD
:100970005C816D817E818F8198850F9445479B01B5
:10098000AC01C501B4010F949640A70196010F94E4
:100990004647EF85F88920813181428153810F9448
:1009A000964020913B0430913C0440913D0450918D
:1009B0003E040F94464762960FB6F894DEBF0FBE12
:1009C000CDBFDF91CF911F910F91FF90EF90DF90FE
:1009D000CF90BF90AF909F908F907F906F905F90DF
:1009E0004F903F902F90089590916F0081E091FD7E
:1009F00002C080E0089590916F009D7F90936F00FA
:100A00000895EFE6F0E080818260808308958F9200
:100A10009F92AF92BF92CF92DF92EF92FF92CF93CD
:100A2000DF93EC0180903D0E90903E0EA0903F0E23
:100A3000B090400E20E030E0A901C501B4010F9450
:100A40003040882309F44AC0C880D980EA80FB80FE
:100A5000A7019601C501B4010F94304018160CF09F
:100A600042C02091B3043091B4044091B504509138
:100A7000B604C701B6010F943040882331F1C0920B
:100A8000B304D092B404E092B504F092B60420917D
:100A9000AF043091B0044091B1045091B204688128
:100AA00079818A819B810F9496409B01AC0160E023
:100AB00070E080E89FE30F944547609312027093C3
:100AC00013028093140290931502609112027091A8
:100AD0001302809114029091150208C060E070E04A
:100AE00080E89FE303C060E070E0CB01DF91CF912D
:100AF000FF90EF90DF90CF90BF90AF909F908F903E
:100B00000895CF93DF9324E0829FC0011124EC016C
:100B1000CF59DE4EFC01E25AF14FDC01AE5AB14F23
:100B20002D913D914D915C91608171818281938184
:100B30000F944647688379838A839B83DF91CF91A3
:100B4000089580FF04C09091AE0490FD8E7F81FFD8
:100B500004C09091AE0491FD8D7F82FF04C09091FE
:100B6000AE0492FD8B7F0895CF92DF92EF92FF92B9
:100B70001F93CF93DF9320910F02222309F48DC09E
:100B8000EC011091AE0410FF2CC0C0903902D0903F
:100B90003A02E0903B02F0903C02288139814A8180
:100BA0005B81C701B6010F94A649181624F4C882C8
:100BB000D982EA82FB82C0904502D0904602E09042
:100BC0004702F0904802288139814A815B81C70140
:100BD000B6010F94304087FF04C0C882D982EA82F0
:100BE000FB8211FF2CC0C0903D02D0903E02E090ED
:100BF0003F02F09040022C813D814E815F81C70110
:100C0000B6010F94A649181624F4CC82DD82EE8238
:100C1000FF82C0904902D0904A02E0904B02F090CF
:100C20004C022C813D814E815F81C701B6010F943A
:100C3000304087FF04C0CC82DD82EE82FF8212FF4B
:100C40002CC0C0904102D0904202E0904302F0904C
:100C50004402288539854A855B85C701B6010F9412
:100C6000A649181624F4C886D986EA86FB86C09061
:100C70004D02D0904E02E0904F02F0905002288535
:100C800039854A855B85C701B6010F94304087FFDF
:100C900004C0C886D986EA86FB86DF91CF911F9172
:100CA000FF90EF90DF90CF9008952F923F924F9258
:100CB0005F926F927F928F929F92AF92BF92CF92EC
:100CC000DF92EF92FF920F931F93CF93DF93CDB7F5
:100CD000DEB7A6970FB6F894DEBF0FBECDBF86ED88
:100CE0009DE00E94B4858091740C83FD83C02091A7
:100CF0005D1130915E1140915F11509160116091D2
:100D0000E20D7091E30D8091E40D9091E50D0F944B
:100D10003040882309F46EC080918107811119C089
:100D20006091330F7091340F8091350F9091360F91
:100D30000F94B2482091280230912902621773075C
:100D400044F40E944EF582E495E30E9446F411E0DB
:100D500001C010E020915D1130915E1140915F1152
:100D6000509160116091E20D7091E30D8091E40D5E
:100D70009091E50D0F9445476B017C0120E030E038
:100D8000A9010F94A64987FF04C0F7FAF094F7F879
:100D9000F094209124023091250240912602509136
:100DA0002702C701B6010F94964020E030E048E4E6
:100DB00053E40F94A64918163CF40E944EF583E2C2
:100DC00095E30E9446F402C01123A1F08091E20D48
:100DD0009091E30DA091E40DB091E50D80935D112C
:100DE00090935E11A0935F11B093601182EE9DE02D
:100DF0000E94DBEC2AE037ED43E25CE360915602AF
:100E00007091570280915802909159020F94964028
:100E10006B017C016091100270911102072E000C91
:100E2000880B990B0F9437409B01AC01C701B601A9
:100E30000F949640698B7A8B8B8B9C8B8091410EA3
:100E4000882309F48CC0C0903D0ED0903E0EE090F7
:100E50003F0EF090400E20E030E0A901C701B6013E
:100E60000F943040882379F02091DE0D3091DF0D12
:100E70004091E00D5091E10DC701B6010F94A649D4
:100E800018160CF06CC02091511130915211409104
:100E90005311509154116091D60D7091D70D8091DE
:100EA000D80D9091D90D0F9445476D8B7E8B8F8B0C
:100EB000988F2091551130915611409157115091B2
:100EC00058116091DA0D7091DB0D8091DC0D9091DD
:100ED000DD0D0F944547698F7A8F8B8F9C8F209102
:100EE000591130915A1140915B1150915C116091F0
:100EF000DE0D7091DF0D8091E00D9091E10D0F946A
:100F000045476D8F7E8F8F8F98A320915D11309113
:100F10005E1140915F11509160116091E20D7091EE
:100F2000E30D8091E40D9091E50D0F9445476B0121
:100F30007C0120E030E0A9016D897E898F89988D40
:100F40000F94304081113DC020E030E0A901698D4F
:100F50007A8D8B8D9C8D0F943040811132C0C12CC5
:100F6000D12C76018E010F5E1F4F22EE3DE04EED3B
:100F70005DE06AED7DE086ED9DE00E9482B980E152
:100F8000E6EDFDE0A1E5B1E101900D928A95E1F772
:100F9000A6960FB6F894DEBF0FBECDBFDF91CF91FE
:100FA0001F910F91FF90EF90DF90CF90BF90AF9087
:100FB0009F908F907F906F905F904F903F902F9079
:100FC00008952D893E894F89588DCA01B9010F9422
:100FD00096404B015C01298D3A8D4B8D5C8DCA0189
:100FE000B9010F9496409B01AC01C501B4010F9467
:100FF00046474B015C012D8D3E8D4F8D58A1CA0196
:10100000B9010F9496409B01AC01C501B4010F9446
:1010100046474B015C01A7019601C701B6010F9439
:1010200096409B01AC01C501B4010F9446470F9453
:10103000F4494B015C012DEB37E346E855E30F948F
:10104000304087FF0FC020E030E0A901C701B601A2
:101050000F94A6494601570187FF04C0B7FAB09420
:10106000B7F8B0942DEB37E346E855E3C501B4017A
:101070000F94304087FD83CF20E030E040EA50E419
:10108000C501B4010F9440480F94B9481B01672B68
:1010900019F422242394312CB10180E090E00F94C4
:1010A00035409B01AC0160E070E080E89FE30F9465
:1010B00040482B013C019B01AC01C501B4010F94D8
:1010C00096404B015C01A30192016D897E898F8955
:1010D000988D0F9496406D8B7E8B8F8B988FA3018C
:1010E0009201698D7A8D8B8D9C8D0F949640698FBE
:1010F0007A8F8B8F9C8FA30192016D8D7E8D8F8D4A
:1011000098A10F9496406D8F7E8F8F8F98A3A30127
:101110009201C701B6010F94964069A37AA38BA3ED
:101120009CA380E1E1E5F1E18E010F5F1F4FD80143
:1011300001900D928A95E1F70E9495FA2B013C01EE
:1011400028EC420E511C611C711C0DA31EA381E0F2
:10115000281A310819F47501640104CF0E9495FA28
:101160008B019C01041915092609370937FD0BC0AD
:101170002B013C0128EC420E511C611C711C80E0CB
:101180000E946D3902C00F94B72A2D893E894F897C
:10119000588D69817A818B819C810F944647698340
:1011A0007A838B839C83298D3A8D4B8D5C8D6D81E9
:1011B0007E818F8198850F9446476D837E838F83D0
:1011C00098872D8D3E8D4F8D58A169857A858B85A9
:1011D0009C850F94464769877A878B879C8729A1CE
:1011E0003AA14BA15CA16D857E858F8598890F946E
:1011F00046476D877E878F87988B750164018E01C6
:101200000F5E1F4F9E01235F3F4FAE01475F5F4F51
:10121000BE016B5F7F4F8DA19EA10E9482B981119B
:1012200096CF99CF8F929F92AF92BF92CF92DF923B
:10123000EF92FF92CF93DF938090560290905702E7
:10124000A0905802B0905902FC01C080D180E28089
:10125000F38020E030E0A901C701B6010F943040CF
:10126000882341F0C0925602D0925702E092580271
:10127000F0925902C0911002D091110284E690E0E0
:101280009093110280931002C0902402D090250206
:10129000E0902602F090270280E090E0A0E8BFE313
:1012A0008093240290932502A0932602B0932702F4
:1012B0000E9455868092560290925702A092580240
:1012C000B0925902D0931102C0931002C09224022E
:1012D000D0922502E0922602F0922702DF91CF9170
:1012E000FF90EF90DF90CF90BF90AF909F908F9046
:1012F0000895CF92DF92EF92FF920F931F93C12C2C
:10130000D12C76018C012DE531E149E551E165E50E
:1013100071E181E591E10E9482B91F910F91FF90E7
:10132000EF90DF90CF9008954F925F926F927F92EF
:101330008F929F92AF92BF92CF92DF92EF92FF92E5
:101340000F931F93CF93DF93CDB7DEB72C970FB6D4
:10135000F894DEBF0FBECDBF2B013C0129873A8731
:101360004B875C8747015801F601E080F1800281DC
:10137000138120E030E0A901B701C8010F9430408B
:1013800081110BC0E7EAF8E285919591A591B4919E
:10139000582F492F3A2F2B2F04C05E2D4F2D302F61
:1013A000212F852F942FA32FB22F89839A83AB836C
:1013B000BC8320E030E0A901B701C8010F943040A0
:1013C000811104C0E12CF12C08E412E4C701D8011A
:1013D0008D839E83AF83B887A501940160915911D5
:1013E00070915A1180915B1190915C110F94304073
:1013F00087FF0CC08092591190925A11A0925B11F4
:10140000B0925C11CE0101960E94798940925111EF
:1014100050925211609253117092541189859A859D
:10142000AB85BC858093551190935611A0935711AD
:10143000B0935811CE0105960E94798920915911D7
:1014400030915A1140915B1150915C11C501B4016A
:101450000F94304087FF0CC08092591190925A111E
:10146000A0925B11B0925C11CE0101960E94798925
:101470000E94CAEC2C960FB6F894DEBF0FBECDBF0B
:10148000DF91CF911F910F91FF90EF90DF90CF9060
:10149000BF90AF909F908F907F906F905F904F9094
:1014A0000895CF92DF92EF92FF920F931F936B01FB
:1014B000FC01E080F18002811381E1E5F1E124810A
:1014C00035814681578160817181828193810E943B
:1014D00094891F910F91FF90EF90DF90CF90089526
:1014E000EF92FF920F931F93CF93DF937C018B01B9
:1014F0000E94B1EEC1E5D1E1209124023091250294
:101500004091260250912702F7016081718182810A
:1015100093810F9440482C853D854E855F850F94BF
:1015200046476C877D878E879F87C8010E9479898F
:10153000DF91CF911F910F91FF90EF900C94CAEC27
:101540000D946E04CF93DF93CDB7DEB72C970FB613
:10155000F894DEBF0FBECDBF0F94C60A0E94F4847C
:101560009CE0E6ECF5E1DE01119601900D929A9572
:10157000E1F781110E940185CE0101960F941B2E87
:101580002C960FB6F894DEBF0FBECDBFDF91CF9182
:1015900008958091BB04659B02C0816001C08E7F6D
:1015A0008093BB04909103018091BB0491FF02C022
:1015B000826001C08D7F8093BB048091BB044B9BF4
:1015C00002C0846001C08B7F8093BB048091630460
:1015D00080FF10C08091D90480FF0CC08091BB04B3
:1015E00080FF08C08091A00681608093A00680E003
:1015F0000F944F2E80916304869580FF11C08091D7
:10160000D904869580FF0CC08091BB0481FF08C07F
:101610008091A00682608093A00681E00F944F2EF7
:10162000809163048695869580FF12C08091D904CD
:101630008695869580FF0CC08091BB0482FF08C010
:101640008091A00684608093A00682E00D944F2EC6
:10165000089580E598E20E9446F48CB16AE478E24D
:1016600085FB882780F90E9448818091030164E40A
:1016700078E2869581700E94488189B16EE378E2B4
:1016800083FB882780F90E94488182B365E378E272
:1016900085FB882780F90C9448818091D8048823A1
:1016A00031F062E070E080E090E00C9422F4089564
:1016B0000F931F938091380E813019F40E9495FA90
:1016C00008C06091800D7091810D8091820D909184
:1016D000830D0091780D1091790D20917A0D309144
:1016E0007B0D601B710B820B930B28EE33E040E007
:1016F00050E00F94864680917C0D90917D0DA091D5
:101700007E0DB0917F0DBC01CD01620F731F841F50
:10171000951F1F910F9108951092380E1092780D19
:101720001092790D10927A0D10927B0D1092800D0F
:101730001092810D1092820D1092830D10927C0DEB
:1017400010927D0D10927E0D10927F0D0895809164
:10175000380E813079F482E08093380E0E9495FA39
:101760006093800D7093810D8093820D9093830D13
:1017700081E0089580E00895CF92DF92EF92FF928A
:101780000F931F93CF93DF936C017A018B01C0E01D
:10179000D0E0CE15DF0581F0D8016D918D01D60125
:1017A000ED91FC910190F081E02DC6011995892BF6
:1017B00011F02196EECF7E01C701DF91CF911F91ED
:1017C0000F91FF90EF90DF90CF90089508950F94C0
:1017D000584A1F920F920FB60F9211242F933F93E6
:1017E0008F939F93AF93BF9380919A0D90919B0D90
:1017F000A0919C0DB0919D0D3091A40623E0230F84
:101800002D3720F40196A11DB11D05C026E8230F38
:101810000296A11DB11D2093A40680939A0D90936A
:101820009B0DA0939C0DB0939D0D80919E0D90916A
:101830009F0DA091A00DB091A10D0196A11DB11D0C
:1018400080939E0D90939F0DA093A00DB093A10D3A
:10185000BF91AF919F918F913F912F910F900FBEAC
:101860000F901F9018951F920F920FB60F92112490
:101870000BB60F922F933F934F935F936F937F938A
:101880008F939F93AF93BF93EF93FF938091BF0488
:101890009091C004A091C104B091C204892B8A2BFD
:1018A0008B2B59F19091BE04E091BC04F091BD04E2
:1018B0008081892780838091BF049091C004A0918A
:1018C000C104B091C204181619061A061B060CF0C2
:1018D00056C08091BF049091C004A091C104B09102
:1018E000C2040197A109B1098093BF049093C00479
:1018F000A093C104B093C20442C080911802EDEBE2
:10190000F8E2E4919FEF90931802E230C9F050F4AE
:10191000EE2399F0E13081F590916F009D7F9093D7
:101920006F002AC0E43019F1E0F0E53029F590911C
:1019300073009D7F909373001FC010926E001CC0B7
:10194000909170009D7F9093700091E09093B00013
:101950009091B100987F94609093B1001092B30081
:101960000BC0909171009D7F9093710005C0909184
:1019700072009D7F9093720060E00E9427F9FF91B2
:10198000EF91BF91AF919F918F917F916F915F91F7
:101990004F913F912F910F900BBE0F900FBE0F9064
:1019A0001F901895FC0130819281930F92832181C1
:1019B000921760F494819F5F94838381830F8217D1
:1019C00010F08FEF820F838381E0089580E0089507
:1019D000FC01128280818150838314820895FB016F
:1019E0004181DC0112962C911297421768F01396F0
:1019F0002C911397241740F0608115962C91621753
:101A000018F424810C94B1940895FC01A081B18153
:101A10001C92A281B3818C918F5F8C930280F381A1
:101A2000E02D90818CE0899F800D1124E7EDF1E19C
:101A300013AE84AF08956091160270911702072EBD
:101A4000000C880B990B0F9437402AE037ED43E2E6
:101A50005CE30F9496402091B7043091B804409114
:101A6000B9045091BA040F94964060932402709385
:101A70002502809326029093270208958091AC0D51
:101A8000811104C08091B10D8093700708958091F9
:101A9000AC0D811104C08091B10D80937007089541
:101AA00020E040E060E070E084E69DE80E94A84C01
:101AB00081E080933A0D1092A6061092A506089533
:101AC0000D944B0E0D944B0E8F929F92AF92BF923E
:101AD000CF92DF92EF92FF92CF938091A80D109258
:101AE000A80D882359F0CF91FF90EF90DF90CF9011
:101AF000BF90AF909F908F900C943E4EC090BF0DC2
:101B0000D090C00DE090C10DF090C20DC114D10471
:101B1000E104F10421F11092BF0D1092C00D10925A
:101B2000C10D1092C20D81E080936E0284E00E948C
:101B3000A185811119C08091A5069091A6068C0DF2
:101B40009D1D9093A6068093A5068091D50C90913B
:101B5000D60CC80ED91ED092D60CC092D50C80914E
:101B60006E02882309F4B0C06091A5067091A606A4
:101B7000072E000C880B990B0F94374020917907A2
:101B800030917A0740917B0750917C070F949640E3
:101B90006B017C0120E030E040E251E40F9496407C
:101BA00020E030E04AE754E40F9496404B015C019A
:101BB00020E030E0A901C701B6010F94304087FD55
:101BC00005C020E030E040EA50E404C020E030E00E
:101BD00040EA50ECC501B4010F94464720E030E0E4
:101BE00040E251E40F9440480F94B2486B017C01ED
:101BF00097FF0AC0F094E094D094C094C11CD11C0B
:101C0000E11CF11C8DE201C08BE280933B0DC7010A
